:020000040800F2
:1080000028EE0020A1810008A981000889AB0008A2
:10801000AD810008AF810008B181000800000000B8
:10802000000000000000000000000000B381000814
:10803000B581000800000000B7810008B981000880
:10804000BB810008BB810008BB810008BB81000820
:10805000BB810008BB810008199E0008299E00080A
:10806000BB810008BB810008BB810008BB81000800
:10807000BB810008BB810008AB990008B3990008D8
:10808000BB810008BB990008BB810008BB810008C8
:10809000BB810008BB810008BB810008BB810008D0
:1080A000BB810008BB810008BB810008BB810008C0
:1080B00035440308BB810008BB810008BB81000870
:1080C000BB810008BB810008BB810008BB810008A0
:1080D000BB810008575303085F5303086753030825
:1080E000219E0008BB810008BB810008BB810008FD
:1080F000BB810008BB810008BB810008C399000850
:10810000BB810008BB810008BB810008BB8100085F
:10811000475303084F530308BB810008BB81000885
:10812000BB810008BB810008BB810008BB8100083F
:10813000BB810008BB810008BB810008BB8100082F
:10814000BB810008BB810008BB810008BB8100081F
:10815000BB810008CB990008D39900086F5303082E
:10816000BB810008BB810008BB810008BB810008FF
:10817000BB810008BB810008BB810008BB810008EF
:10818000BB810008BB810008DFF810D000F058FC6C
:1081900000480047B1710308AFF3008028EE0020CB
:1081A0000648804706480047FEE7FEE7FEE7FEE791
:1081B000FEE7FEE7FEE7FEE7FEE7FEE7CD43030846
:1081C000898100082DE9F0410024061B254671F144
:1081D000000605DA01240027D0EB070067EB010158
:1081E000161E73F1000605DA0027D2EB07020125FF
:1081F00067EB030300F0C1FA86460E4617469C461D
:10820000AC4204D00025D0EB050E65EB010624B18D
:108210000020D2EB000760EB030C704631463A4673
:108220006346BDE8F081202A06DBCB17203A41FAED
:1082300002F043EAE07306E041FA02F3D040C2F1F3
:108240002002914008431946704740EA01039B070A
:1082500003D009E008C9121F08C0042AFAD203E0BB
:1082600011F8013B00F8013B521EF9D27047421E43
:1082700012F8013F002BFBD111F8013B02F8013B42
:10828000002BF9D17047421C10F8011B0029FBD1CB
:10829000801A704730B505460020034600E05B1C9D
:1082A000934205D2EC5CC85C201A01D1002CF6D1B7
:1082B00030BD2DE9FE4F804681EA0300C00F0C4619
:1082C000009021F0004123F00045B8EB0200A941E5
:1082D00005D24046214690461C460B46024623F0F6
:1082E0000040104347D0270DC7F30A00C3F30A51DB
:1082F0000290401A019040286BDAC3F3130040F457
:10830000801B0098924620B10023D2EB030A63EB56
:108310000B0B01985946C0F14002504600F05EFA3E
:1083200006460D4650465946019AFFF77CFF10EB72
:1083300008006141002487EA115284EAE7731A4376
:1083400040D0009A62B3019A012A4FEA075215DC25
:10835000001B61EB02014FF0004202EA0752CDE937
:108360000042001C41F5801132462B4600F0EAFA2B
:1083700003B0BDE8F08F40462146F9E7001B61EBF2
:108380000201001C41F5801300185B412018A2F582
:10839000001747EB030140EAD570B6196D4111E0B3
:1083A0006D084FEA360645EAC0754FEA0752001BD2
:1083B00061EB0201001C41F5801149084FEA3000D1
:1083C0000019514132462B4603B0BDE8F04F00F092
:1083D000AABA0098012240000023D0EB020263EB0E
:1083E000E073009821464FEAE074B8EB000061EBBF
:1083F0000401E9E783F000435BE781F0004158E7BF
:108400002DE9FE4F81EA030404F0004421F000410D
:1084100000944FF0000B23F0004350EA01045ED0BB
:1084200052EA03045BD0C3F30A54C1F30A552C4447
:10843000A4F2F3340194A0FB0254C1F3130141F4FC
:108440008011C3F3130343F4801301FB024400FBC8
:10845000034E840A970A44EA815447EA8357A4FBEF
:10846000076802958D0A05FB07854FEA932C04FBEC
:108470000C542705029D4FEA065847EA1637B5EB1C
:1084800008056EEB070C870E920E47EA811742EA49
:108490008312A7FB0201B6EB0B0164EB00042B0D6A
:1084A00043EA0C335E1844EB1C50DA465146E7FBB6
:1084B0000201C5F313044FEA0B3343EA14534FEAA6
:1084C0000432019C43EA0603A4F10C040294009CCC
:1084D000CDE900B400F036FA03B0BDE8F08F00201B
:1084E0000146F9E72DE9F04D81EA030404F0004B61
:1084F00021F0004514464FF0000A23F0004150EAF5
:10850000050220D054EA01021DD0C5F30A570246E5
:10851000C5F31303C1F31300C1F30A5640F48015E9
:1085200043F48013A7EB0608101BD64608F2FD386B
:1085300073EB050002D308F1010801E092185B41DA
:10854000B8F1000F03DA00200146BDE8F08D0020ED
:108550004FF48011064684460EE0171B73EB0507A7
:1085600005D3121B63EB050306434CEA010C4908D3
:108570004FEA300092185B4150EA0107EDD152EA10
:10858000030012D082EA040083EA0501084305D003
:10859000101BAB4106D20122002306E000224FF05F
:1085A000004302E06FF0010253101AEB06004CEB9F
:1085B000085110EB0A0041EB0B01BDE8F04D00F053
:1085C000B2B9F0B4CA17CB0F50405140C61841F1B0
:1085D00000054FEAC372314628004FF0960303D0DE
:1085E000B623F0BC00F071B930460021F9E70EB5B2
:1085F000C10F80EAE0700844CA07002140F233430B
:108600008DE80E000A460B4600F09CF903B000BD51
:108610000EB540F2334102910021CDE900110A4626
:108620000B4600F08FF903B000BD3EB5CA17CB0F63
:10863000002450405140C0186141DA0740F23343F2
:108640000094CDE901232246234600F07BF903B0D4
:1086500030BD10B500F0004420F00040C20DC0F362
:10866000160040F400007F2A02DA0020014610BD07
:108670000021962A03DCC2F19602D04002E0963A2D
:1086800000F0ACF8002CF2D00023D0EB030063EB39
:10869000010110BD70B5C1F30A5201F0004500247C
:1086A000C1F3130140F2FF3341F480119A4201DA21
:1086B000002070BD40F233439A42A2F2334203DC01
:1086C000524200F09AF800E090402C43F1D0404232
:1086D00070BD70B5C1F30A5201F000450024C1F32A
:1086E000130140F2FF3341F480119A4202DA002074
:1086F000014670BD40F233439A42A2F2334203DC9A
:10870000524200F07AF801E000F068F82C43F0D013
:108710000023D0EB030063EB010170BD00F00042C9
:1087200030F000400AD0C10D01F56071C0F31600B1
:1087300042EA0151C2084007114370470020014638
:10874000704701F0004330B421F0004150EA0102CB
:1087500006D00A0DA2F56072C1F31301002A02DCF3
:1087600030BC00207047440F44EAC104C100E01847
:1087700030BC00EBC25000F09FB82DE9F05F054619
:10878000002092469B4688460646814640241BE0D0
:10879000284641464746224600F02FF853465A469F
:1087A000C01A914110D311461846224600F016F81F
:1087B0002D1A67EB01084F4622460120002100F0E8
:1087C0000DF817EB00094E41201EA4F10104DFDC77
:1087D000484631462A464346BDE8F09F202A04DB3E
:1087E000203A00FA02F1002070479140C2F12003C4
:1087F00020FA03F3194390407047202A04DB203A03
:1088000021FA02F00021704721FA02F3D040C2F1B0
:108810002002914008431946704700000FB400231E
:1088200000B589B00CA900910B996FF00042CB60A4
:108830001E4B06931E4B07930423CDE901321D4ABC
:10884000089202466B46002000F0A6F909B05DF8D8
:1088500014FB70B586B006464FF0FF300091CDE9AD
:108860000101002015460C4604903246694604A8D2
:10887000FFF7D4FF02460498211825B108B1084635
:1088800000E020462860049800280DD0002A02DD70
:108890000098884208D0081B0094CDE901043246B4
:1088A000694604A8FFF7BAFF06B070BDD18D000875
:1088B000EF8D0008658A00080029A8BF7047401C9A
:1088C000490008BF20F00100704710B4B0FA80FCE6
:1088D00000FA0CF050EA010404BF10BC704749B123
:1088E000CCF1200421FA04F411FA0CF118BF012193
:1088F00021430843A3EB0C01CB1D4FEA00614FEA73
:10890000102042BF002010BC704700EBC350104441
:108910000029A4BF10BC7047401C490008BF20F0CC
:10892000010010BC704710B5141E73F1000408DA82
:10893000401C41F1000192185B411A4301D120F023
:10894000010010BD2DE9F04D92469B4611B1B1FAE0
:1089500081F202E0B0FA80F220329046FFF73EFF4B
:1089600004460F4640EA0A0041EA0B0153465A46C4
:10897000084313D0114653EA010019D0C8F1400250
:108980005046FFF73AFF05460E46504659464246C6
:10899000FFF724FF084305D0012004E020463946B4
:1089A000BDE8F08D0020054346EAE0762C433743CE
:1089B0000A986305E40AA0EB08000022FD0A44EAD5
:1089C00047540A3002D500200146E9E70105101995
:1089D0006941DDE9084500196941BDE8F04DA2E7AC
:1089E00070B521F0004303430CD0C1F30A550024B5
:1089F000D5EB040564EB0403D617AD1AB34102DBD3
:108A00000020014670BD201841EB025170BD0000EE
:108A100030B5041E71F1000404DB4FF00044404205
:108A200064EB0101141E73F1000405DB1C464FF0DA
:108A30000043524263EB0403994208BF904230BDA9
:108A4000064C074D06E0E06840F0010394E807009B
:108A500098471034AC42F6D3FFF79AFBA8F7030807
:108A6000C8F70308C0B24FF4F05100F03BBA000061
:108A70002DE9FF4F087883B09946FF2805D0491C9F
:108A80002D2804D00024002008E000200BE0012461
:108A9000F9E700EB800003EB4000491C0B78FF2B4B
:108AA000F7D104B1404200230293147819461D46C1
:108AB0002D2C01D02B2C04D1521C2D2C13D0002492
:108AC0000294AA461478FF2C0FD00A25A3FB057840
:108AD00001FB05814FF0000C03FB0C11521CE31944
:108AE0004AEB0101EEE70124EAE7814453EA010081
:108AF00002D019F5C87F06DA03980021C0E90011F9
:108B000007B0BDE8F08F0025AE4E2F46DFF8B882E3
:108B1000184600F0FBF9CDE90001B9F1000002DAD6
:108B2000C9F1000400E004460023A74A1AEB030B36
:108B300042EB045A12E0E00707D02A463346384693
:108B40004146FFF75DFC074688462A4633461046F5
:108B50001946FFF755FC05460E466410002CEAD175
:108B6000DDE90001B9F1000F5A46534606DAFFF776
:108B7000B9FC3A464346FFF7B5FC05E0FFF740FC79
:108B80003A464346FFF73CFC029A0AB181F00041A5
:108B9000039AC2E90001B3E72DE9FF4F1F468DB0EC
:108BA000D7E901464FF0FF382E2045464FF0000927
:108BB0000B90B9696D1C0E988847396A82468847C0
:108BC0000028F6D1BAF1FF3F0AD024F4D064002E79
:108BD00011DDBAF12B0F08D0BAF12D0F0BD102E045
:108BE000404611B08DE744F48064B9696D1C0E985D
:108BF00088478246761E6946600501D52D2000E033
:108C00002B208DF8000001F1010B0DF1200809E087
:108C1000B9696D1C0E98884782460F9844F4007419
:108C2000761E0560002E02DDBAF1300FF0D00B99F0
:108C30008A453ED144F0800406E00F99681CA9F1F2
:108C4000010944F400740860B9696D1C761E0E9821
:108C5000884782463028F0D02BE00B998A4505D111
:108C6000200603D444F08004761E18E050462DF010
:108C7000B9FE08B30DF11301761E44F400748B4560
:108C800008D2AAF130000BF8010B200607D5A9F194
:108C9000010003E0200602D409F101008146A0058D
:108CA00002D50F99681C0860B9696D1C0E98884739
:108CB0008246002ED1DC53E0002E51DDBAF1650F63
:108CC00002D0BAF1450F4BD1A00549D5B9696D1C49
:108CD00024F44074761E0E9888478246002E0CDDE0
:108CE0002B2804D0BAF12D0F07D144F48074B96950
:108CF0006D1C0E9888478246761EE00501D52D2111
:108D000000E02B2108F8011BCDF82C8021E00DF1AB
:108D10002901761E44F4007488450CD2AAF1300073
:108D200010F0FF0088F8000002D10B99884509D99E
:108D300008F1010806E0E00501D5244801E042F20F
:108D40000F708146B9696D1C0E98884782460F984E
:108D50000560002E04DD50462DF044FE0028D6D1DB
:108D6000F9690E988847FF208BF8000088F800000A
:108D70000020069007904B466A4608A906A8FFF710
:108D800077FEA00502D46FF001002AE714F0240F4B
:108D90000AD0E00714D1DDE906123868031D3B60F4
:108DA0000068C0E900120BE0DDE90601FFF7C9FC2D
:108DB0000146E00704D13868021D3A60006801608E
:108DC00028460EE7000014400000F03FF1D8FFFFF6
:108DD000426842B1016811F8013B23B1521EC0E95B
:108DE0000012184670470121C160881E7047426812
:108DF0005AB1C368016843B983688B4205D0491EE4
:108E0000521CC0E90012002070474FF0FF3070473D
:108E10002DE9F04D00231A461B1A8A4103DB00207E
:108E20000146BDE8F08DC1F30A52C1F3130141F4CC
:108E300080154FF0000BD10702D100186D41521E72
:108E40000027044640F2FF11384601EB620A3E4615
:108E50008046024600204FF48011FFF7CEFCC21975
:108E60007141BB1846EB0100B4EB030C75EB000C31
:108E700004D3E41A65EB000517460E46241908F1E1
:108E800001006D4180463428E3DDF91946EB060008
:108E9000091BA84103D24FF0FF32134601E0002224
:108EA00013461BEB070046EB0A51BDE8F04DFFF7F8
:108EB0003ABD000030B5041E71F1000404DB4FF030
:108EC0000044404264EB0101141E73F1000405DB11
:108ED0001C464FF00043524263EB04038B4208BF31
:108EE000824230BD7F2801D9002208E0064A02EB09
:108EF0005002C007127800D1120902F00F020120BF
:108F0000904008407047000068F703080EB540F233
:108F1000334202920022CDE900221346FFF712FDF0
:108F200003B000BD70B58C1810F8015B15F0070395
:108F300001D110F8013B2A1106D110F8012B03E0F2
:108F400010F8016B01F8016B5B1EF9D12B0705D4FA
:108F50000023521E0DD401F8013BFAE710F8013B43
:108F6000CB1A921C03E013F8015B01F8015B521E5F
:108F7000F9D5A142D8D3002070BD10B502461078B3
:108F800003E012F8014B2318D8B20B1EA1F1010423
:108F9000A1B2F6D110BD000070B5ADF5287D044634
:108FA0000D460020A790A690002604EB44004549FA
:108FB00001EBC000408AA84203DC00200DF5287DAB
:108FC00070BD0020A69077E004EB44003D4B03EB1E
:108FD000C000028A04EB440003EBC00080892844EF
:108FE00081B2394800F010F90020A79011E004EB9D
:108FF0004400344901EBC0004068BDF89C12405C5D
:1090000001A9BDF89C228854BDF89C02401C80B286
:10901000A79004EB44002B4901EBC000008ABDF887
:109020009C128842E3DC04EB4400264A02EBC000B9
:10903000008A401E81B201A8FFF79FFF23490870F4
:1090400004EB44001F4901EBC000008A401E01A947
:10905000085C1E490978884226D10020A79016E0B6
:1090600004EB4400174901EBC0004068BDF89C12B6
:10907000405C04EB4401134A02EBC1018968BDF86E
:109080009C228854BDF89C02401C80B2A79004EB3F
:1090900044000C4901EBC000008A401EBDF89C1240
:1090A0008842DDDC012089E764202DF0D9FEBDF87F
:1090B0009802401C80B2A690BDF89802062883DB77
:1090C00000207BE7A4CF030890A70020310A0020EE
:1090D0002DE9F043ADF5257D04460E460025002719
:1090E000A846A94604EB4400324901EBC000408A7F
:1090F000B04204DC00200DF5257DBDE8F08300259D
:1091000018E004EB44002B4901EBC0008068405D8F
:1091100004EB4401274A02EBC1014968485504EBBE
:109120004400114601EBC0004068405D0DF80500A9
:10913000681C85B204EB44001E4901EBC000008AA4
:10914000401EA842DDDC04EB44000A4602EBC000EE
:10915000008A401E81B26846FFF70FFF04EB44010E
:10916000144A02EBC101098A491E0DF801000027CB
:109170001BE004EB44000F4B03EBC000028A04EB3E
:10918000440003EBC0008089304481B2684600F09F
:109190004FF931462046FFF7FFFE012800D1AAE72C
:1091A00064202DF05DFE781C87B2062FE1DB0020E5
:1091B000A1E70000A4CF030808B50020009028F024
:1091C000B9FB0F49087000F09BF80D48007824287F
:1091D00004D0272807D028280FD109E0002109480A
:1091E00080F8081D09E00121064880F8081D04E008
:1091F0000221044880F8081D00BF00BF08BD000020
:109200002C0A0020BC2200202DE9F04106460D4624
:109210001746002401202DF0DBFB002028490880A0
:109220000DE028F069FB00F0800000B10BE00120A8
:109230002DF016FE22480088401C21490880204855
:109240000088C828EDDB00BF1D480088C82832DA36
:1092500010211C4801F08CFC08211A4801F08AFCFE
:10926000E82000F031F8C5F3871000F02DF8A906CA
:10927000080E00F029F8002000F026F8002404E091
:10928000002000F021F8601C84B2042CF8DB0024DC
:1092900005E0FF2000F018F83055601C84B2BC4295
:1092A000F7DB1021074801F065FC00202DF090FB52
:1092B0000120BDE8F08100202DF08AFB0020F8E7B6
:1092C0002E0A00200000024010B5044600BF022113
:1092D0000A4828F03FFC0028F9D02146074828F02A
:1092E00045FC00BF0121054828F034FC0028F9D0D6
:1092F000024828F038FCC0B210BD00000030014028
:1093000010B501202DF064FB00201E4908800DE0FF
:1093100028F0F2FA00F0800000B10BE001202DF0FF
:109320009FFD18480088401C164908801548008891
:10933000C828EDDB00BF13480088C8281CDA1021BC
:10934000114801F015FC08210F4801F013FC3D20E5
:10935000FFF7BAFF2A20FFF7B7FF8020FFF7B4FF1F
:10936000A720FFF7B1FF1021074801F003FC002000
:109370002DF02EFB012010BD00202DF029FB002038
:10938000F9E700002E0A00200000024070B50546F3
:109390000E46002401202DF01BFB002022490880EE
:1093A0000DE028F0A9FA00F0800000B10BE00120E8
:1093B0002DF056FD1C480088401C1B4908801A48A7
:1093C0000088C828EDDB00BF17480088C82825DAC8
:1093D0001021164801F0CCFB0821144801F0CAFB0B
:1093E0008420FFF771FF0020FFF76EFF0020FFF7DA
:1093F0006BFF0020FFF768FF002404E0285DFFF703
:1094000063FF601C84B2B442F8DB1021074801F00E
:10941000B1FB00202DF0DCFA012070BD00202DF002
:10942000D7FA0020F9E700002E0A002000000240D1
:1094300070B506460C46154601202DF0C9FA29469E
:109440003046FFF7A3FF08B9002070BD00201F4978
:1094500008800DE028F050FA00F0800000B10BE029
:1094600001202DF0FDFC19480088401C1749088098
:1094700016480088C828EDDB00BF14480088C828BB
:109480001EDA1021124801F073FB0821104801F088
:1094900071FB8320FFF718FFC4F38710FFF714FF59
:1094A000A106080EFFF710FF0020FFF70DFF1021A7
:1094B000074801F05FFB00202DF08AFA0120C4E785
:1094C00000202DF085FA0020BFE700002E0A0020C2
:1094D0000000024030B502460020002304E012F8EC
:1094E000014B60405C1CE3B28B42F8DB30BD70B5D1
:1094F00004460D46164632462946204600F001F83D
:1095000070BDF8B503460C460020002100BF06E000
:10951000C50022FA05F5EDB20DF80050401C0428F4
:10952000F6DB00201AE0064600EBD6777F100FB975
:10953000012701E04FF0FF373D4600210BE01E5CA4
:10954000012D01D10F4601E0C1F103071DF807709D
:109550007E401E54491C0429F1DB401CA042E2D38A
:10956000F8BD000010B5044639202DF0BBFEE0B276
:109570002DF0D8FEC4F307202DF0D4FEC4F307402D
:109580002DF0D0FE200E2DF0CDFE4FF4805103487B
:1095900001F0F0FA2CF02EF810BD0000000402409B
:1095A0002DE9F04107460E4614463A202DF09AFE6A
:1095B000F0B22DF0B7FE30122DF0B4FE4FF4805112
:1095C0000F4801F0D7FA19E02CF014F805461D2DCC
:1095D00011D1384600F0ACF805463B202DF082FE54
:1095E0004FF48051064801F0C5FA2F4434B1208869
:1095F0002844208002E02846BDE8F081E4E700002E
:10960000000402402DE9F04107460E4614463C2076
:109610002DF068FEF0B22DF085FE30122DF082FEA6
:109620004FF48051104801F0A5FA0CB100202080C1
:1096300019E02BF0DFFF05461E2D11D1384600F052
:109640002BF905463D202DF04DFE4FF48051064884
:1096500001F090FA2F4434B120882844208002E0A1
:109660002846BDE8F081E4E70004024010B528F088
:109670003BF808B100F02EF8302000F0A9F810BD3A
:1096800010B504462146362000F08EF810BD10B506
:10969000044614B1204600F0ABF8342000F098F8EE
:1096A00010BD10B50446204600F0A2F820785C28D2
:1096B00002D020782F2803D10021642000F008F97F
:1096C000322000F085F810BD10B5682000F04CF88D
:1096D00010BD000010B522202DF004FE2DF0F7FD86
:1096E00004464FF48051024801F044FA204610BD70
:1096F000000402402DE9F0412DF0E9FD04462DF073
:10970000E6FD05462DF0E3FD06462DF0E0FD07469B
:109710004FF48051054801F02DFA44EA052040EA53
:10972000064040EA0760BDE8F08100000004024006
:1097300070B5044627202DF0D5FD2DF0C8FD064656
:10974000054646B100BF2DF0C2FD2070641C701E9E
:10975000C0B2061EF7D14FF48051024801F00AFA58
:10976000284670BD0004024010B504460C202DF0C0
:10977000B9FD20462DF0D6FDFFF7BCFF10BD00005F
:1097800070B504460A202DF0ADFD20462DF0CAFD2F
:109790002DF09DFD05464FF48051024801F0EAF995
:1097A000284670BD0004024070B505460C462846A8
:1097B0002DF098FD20462DF0B5FD4FF48051034863
:1097C00001F0D8F92BF016FF70BD00000004024034
:1097D00010B5044620462DF085FD4FF48051034816
:1097E00001F0C8F92BF006FF10BD00000004024094
:1097F0002DE9F041064601202DF074FD2DF067FDA6
:1098000043282BDA2B20FFF7BBFF102826DA2F2066
:109810002DF068FD00202DF085FD3220FFF7D8FFE8
:109820000446142C1AD1CF20FFF7AAFF0446ACB18E
:109830004C20FFF799FF00EB042739464C2000F03D
:1098400047F85020FFF790FF00EB042739465020DF
:1098500000F03EF80021702000F03AF82F202DF0A3
:1098600041FD357828462DF05DFD09E0761C357800
:109870005C2D01D02F2D00D1002528462DF052FD62
:10988000002DF3D14FF48051024801F073F9BDE887
:10989000F08100000004024070B504462D202DF038
:1098A00021FD2DF014FD0646054646B100BF207887
:1098B0002DF038FD641C701EC0B2061EF7D14FF4A7
:1098C0008051024801F056F9284670BD000402405C
:1098D00070B505460C460D202DF004FD28462DF0F0
:1098E00021FDE0B22DF01EFDC4F307202DF01AFD7E
:1098F000C4F307402DF016FD200E2DF013FD4FF49C
:109900008051024801F036F970BD000000040240A9
:1099100070B502460C46FF25FF2309E012F8010B43
:1099200080EA05010648405C80EA03050548435C7F
:10993000201EA4F10106B4B2F0D145EA032070BDA7
:109940000CCD03080CCE03082DE9F04103460C466C
:1099500000200146024606E013F8010B411842F1CF
:109960000002601E84B2002CF6DC080C40EA024CB7
:10997000100C8DB21CEB050140F10002080C40EA0E
:10998000024041186FEA010080B2BDE8F08130B5B5
:1099900002460020002305E012F8015B2C18E0B21B
:1099A0005C1CE3B28B42F7DB30BD10B51DF0A4FAAE
:1099B00010BD10B51DF03EFA10BD10B51DF00AFA2D
:1099C00010BD10B51DF066FA10BD10B51FF080FD7A
:1099D00010BD10B527F0C4F910BD00000246094BB8
:1099E0009A4201D2084801E00648103801F00053BD
:1099F0001BB1064B0B40C36002E0044B0B4083607D
:109A00007047000010640240006002407D0F7D0F2F
:109A100021B1026842F00102026003E0026822F014
:109A20000102026070470000016821F0010101603D
:109A30000021016041608160C160016121214161BB
:109A40004A49884204D13D21484A103A91608CE04D
:109A500046491831884205D14FF47461434A103A9F
:109A6000916082E041493031884205D14FF4741150
:109A70003E4A103A916078E03C494831884205D12D
:109A80004FF07461394A103A91606EE037496031A5
:109A9000884204D13649354A103AD16065E03349ED
:109AA0007831884204D13349304A103AD1605CE0C1
:109AB0002E499031884204D12F492C4A103AD16066
:109AC00053E02A49A831884205D14FF03D51274A39
:109AD000103AD16049E02949884204D13D21274A02
:109AE000083A116041E025491831884205D14FF408
:109AF0007461224A083A116037E0204930318842C7
:109B000005D14FF474111D4A083A11602DE01B492C
:109B10004831884205D14FF07461184A083A116003
:109B200023E016496031884204D11149134A121FBB
:109B300011601AE011497831884204D10D490F4A69
:109B4000121F116011E00D499031884204D10A4979
:109B50000A4A121F116008E00849A831884204D15E
:109B60004FF03D51054A121F1160704710600240CE
:109B70003D000020400F002000003D201064024006
:109B800010B501F080034BB122B1436943F080036B
:109B9000436103E0436923F08003436180290BD0D4
:109BA0002AB1036801F01E042343036004E0036844
:109BB00001F01E04A343036010BD000010B5002295
:109BC0000268134B1A40CC680B6823434C6923434B
:109BD0008C692343CC6923430C6A23434C6A234397
:109BE0008C6A23434C6B23438C6B23431A430260E0
:109BF000426922F00702D1E90B3423431A43426140
:109C00000B6943604B6883608B68C36010BD0000C4
:109C10003F801CF01CB500240121202027F070FD9E
:109C20003020009001208DF8040000208DF80600FF
:109C300003208DF8050000208DF8070069461748BD
:109C400000F022FF3021154800F094FF0021144855
:109C500080F8841600201349887001204870C8706D
:109C60004FF4FA70886000F021F80F4890F80B0F5D
:109C7000592811DD24200A49F53948710820087156
:109C80003020C870142088702020487000210648B9
:109C900080F80B1F00F04EF81CBD000000140240BD
:109CA000BC32002040390020BC2200201CB52DF021
:109CB000DFF9D0202DF0A8F92DF00EFA00202DF0BC
:109CC000A3F92DF009FA2DF0D3F9D1202DF09CF94C
:109CD0002DF002FA00240EE0062C05DA01202DF00A
:109CE00063F90DF8040004E000202DF05DF90DF893
:109CF0000400601CC4B2072CEEDB2DF0D3F99DF8F4
:109D000006000A4948719DF8050008719DF8040095
:109D1000C8709DF8020088709DF8010048709DF899
:109D20000010034880F80B1F1CBD0000C731002045
:109D3000BC2200201CB500241B4890F80B0F8DF8A6
:109D400000001A4840788DF80100184880788DF896
:109D5000020001208DF803001448C0788DF804003B
:109D6000124800798DF80500104840798DF80600FA
:109D70002DF07EF9D0202DF047F92DF0ADF900201F
:109D80002DF042F92DF0A8F900BF07E01DF80400FE
:109D90002DF03AF92DF0A0F9601CC4B2072CF5DBC8
:109DA0002DF080F91CBD0000BC220020C73100202E
:109DB00070B502460C460025002309E012F8010B9D
:109DC00080EA05010648405C80EA03050548435CDB
:109DD000201EA4F10106B4B2F0D145EA032070BD03
:109DE0000CCD03080CCE030810B504460B46002129
:109DF000072A00DD072244EA042001462BB901FAB4
:109E000002F081B20912084610BD012B02D11141A6
:109E1000C8B2F9E700BFF7E710B527F095FA10BD13
:109E200010B527F091FA10BD10B527F08DFA10BDCE
:109E30000149086070470000143C014001460020C1
:109E40000022074B1B6803EA0102054B14331B6811
:109E50000B4013B10AB1012000E000207047000060
:109E6000003C0140002123498279002A3AD00A4669
:109E7000126803689A430B461A600A1D1268036849
:109E80009A430B1D1A60027911440A6803681A4349
:109E90000A60184A0832126803689A43154B08335F
:109EA0001A601A1D126803689A43124B0C331A6029
:109EB0004279102A0ED11A1F126803681A430D4BFB
:109EC00008331A601A1D126803681A43094B0C33D1
:109ED0001A600DE00749427911440A6803681A4381
:109EE0000A6005E0027911440A6803689A430A602F
:109EF00070470000003C014010B504460B460021AD
:109F0000072A00DD072244EA0420014613B9114163
:109F1000C8B210BD012B05D101FA02F081B20912BD
:109F20000846F6E700BFF4E7F0B5ADF21C5D044665
:109F30000D460020CDF81805CDF81405002604EBD9
:109F40004400584901EBC000408AA84203DC0020CD
:109F50000DF21C5DF0BD0020CDF814059AE05148CB
:109F60000122C168504800F0A9FA4E4840680078C4
:109F70008DF800009DF8000038287DD104EB4400E6
:109F8000484B03EBC000C06804EB4403454F07EBAC
:109F9000C3031B8A03FB050104EB44003B4603EBB0
:109FA000C000028A404800F089FA0020CDF8180568
:109FB00012E004EB44003B4901EBC0004068BDF8EF
:109FC0001815405CBDF818250DF80200BDF81805FD
:109FD000401C80B2CDF8180504EB4400314901EB78
:109FE000C000008ABDF818158842E2DC04EB44008A
:109FF0002C4A02EBC000008A401E81B2684600F085
:10A0000023FB064604EB4400264901EBC000008A0E
:10A01000401E1DF80000B04233D10020CDF81805D5
:10A0200020E004EB44001F4901EBC0004068BDF88C
:10A030001815415C04EB44001A4A02EBC00080682A
:10A04000BDF81825024404EB4400164B03EBC00096
:10A05000008A401E68431154BDF81805401C80B2A8
:10A06000CDF8180504EB44000E4901EBC000008A4E
:10A07000401EBDF8181500E003E08842D1DC012045
:10A0800066E764202CF0ECFEBDF81405401C80B29D
:10A09000CDF81405BDF814050628FFF660AF0020C2
:10A0A00056E70000F87D0308E07900202DE9F04133
:10A0B000ADF5A36D04460E4600250027A8460020F6
:10A0C000009004EB4400494901EBC000408AB042D3
:10A0D00004DC00200DF5A36DBDE8F0814448807BD1
:10A0E000002878D100210846FFF71EFF01287AD109
:10A0F000002520E004EB44003C4901EBC0008068EF
:10A10000411904EB4400394A02EBC000008A401EAA
:10A110007043085C04EB440102EBC10149684855F7
:10A1200004EB4400114601EBC0004068405D01A90A
:10A130004855681C85B204EB44002C4901EBC00073
:10A14000008AA842D6DC00274BE004EB4400274BF2
:10A1500003EBC000C06804EB4403DFF890C00CEBD5
:10A16000C3031B8A03FB060104EB4400634603EBB5
:10A17000C000008A401E82B21E4800F021FA04EBA3
:10A1800044001A4A02EBC000008A401E81B201A8B6
:10A1900000F05AFA009004EB4400144A02EBC000AD
:10A1A000C06804EB4402114B03EBC202128A104454
:10A1B00004EB440203EBC202128A02FB0600411EBA
:10A1C0000122684600F0FCF931462046FFF7ACFE5C
:10A1D000012801D17EE706E064202CF041FE781CC6
:10A1E00087B2062FB1DB002074E70000F87D03087A
:10A1F000BC120020E0790020F0B5ADF21C5D002516
:10A20000002400200190002600210120FFF78CFE91
:10A210004B4890F8FC6C00204A49088080E00025FB
:10A220006FE0002414E04748008800EB40004649F6
:10A2300051F83000005D4349098801EB4101424A71
:10A2400002EBC1014968085502A90855601C84B297
:10A250003C48008800EB40003B4901EBC000008A0D
:10A26000401EA042DFDC3748008800EB40000A4671
:10A2700002EBC000008A401E81B202A800F0E4F99F
:10A2800001903048008800EB40002F4B03EBC000EA
:10A29000C0682C4B1B8803EB43032B4F07EBC30316
:10A2A0001B8A03FB05012748008800EB40003B4662
:10A2B00003EBC000008A401E82B2244800F080F9FF
:10A2C0002048008800EB40003A4602EBC000C0681E
:10A2D0001C4A128802EB42023B4603EBC202128A7E
:10A2E0001044184A128802EB420203EBC202128A9F
:10A2F00002FB0500411E012201A800F061F9681C63
:10A3000085B21048008800EB40000F4901EBC00007
:10A31000408AA84285DC0B480088401C0949088017
:10A32000084800880D28FFF67AAF054880F8FC6CD5
:10A3300000210120FFF7BAFE0DF21C5DF0BD000008
:10A34000BC22002010000020F87D0308E0790020E6
:10A350001CB50121084627F0D3F901208DF804002F
:10A3600002208DF8050000208DF8060001208DF8F0
:10A370000700182000906946144800F085FB05226C
:10A380001146124800F0C8FB052206210F4800F0D4
:10A39000C3FB052207210D4800F0BEFBA020009062
:10A3A00002208DF8040003208DF8050000208DF8B0
:10A3B00006008DF807006946044800F065FB402060
:10A3C00000906946014800F05FFB1CBD00000240A0
:10A3D0002DE9F84300240025002700200090804646
:10A3E000FFF7B6FF00F0BCF80A202CF039FD6E46EE
:10A3F00008212D4800F0BCFB10212B4800F0BAFBCF
:10A40000062000F091F80821274800F0B3FB08214E
:10A41000254800F0ADFB1021234800F0ABFB0120E4
:10A4200000F082F8002000F07FF808211E4800F0BC
:10A43000A1FB1E48D0F82C11B0F83021B0F8320141
:10A4400002FB0010B0F5003F02D900BE00BFFEE7DE
:10A450001748006808B9FFF7CFFE002015490880AB
:10A4600017E0002406E0134908782146FFF75CFD59
:10A47000601C84B20F48008800EB40000B4901EBE0
:10A48000C000408AA042EEDC0A480088401C09490E
:10A490000880084800880D28E3DB0748D0F80C0244
:10A4A0000549C873BDE8F88300000240F87D030841
:10A4B0001C02434210000020BC1200202DE9F04194
:10A4C00005460C461646002701202CF07EFA08218E
:10A4D000144800F04DFB1021124800F04BFB032004
:10A4E00000F022F8C4F3074000F01EF8C4F3072080
:10A4F00000F01AF8E0B200F017F800BF06E0002004
:10A5000000F012F828706D1C781C87B2B742F6DB99
:10A510000821044800F02EFB00202CF056FABDE87C
:10A52000F08100000000024010B5044600BF022187
:10A530000A4827F00FFB0028F9D02146074827F0EA
:10A5400015FB00BF0121054827F004FB0028F9D0C6
:10A55000024827F008FBC0B210BD000000300140E7
:10A5600000B585B00121080327F01AF9134827F038
:10A57000C5FA0020ADF80000ADF80400ADF8060003
:10A58000ADF808004FF40070ADF80A000820ADF8EF
:10A590000C000020ADF80E000720ADF810004FF4BD
:10A5A0008270ADF802006946044827F0E1FA012103
:10A5B000024827F097FA05B000BD000000300140C6
:10A5C0002DE9F04105460C461646002701202CF0E7
:10A5D000FCF908211B4800F0CBFA1021194800F0C3
:10A5E000C9FA0620FFF7A0FF0821164800F0C2FABA
:10A5F0000821144800F0BCFA1021124800F0BAFA01
:10A600000220FFF791FFC4F30740FFF78DFFC4F36B
:10A610000720FFF789FFE0B2FFF786FF00BF05E0E4
:10A620002878FFF781FF6D1C781C87B2B742F7DBF3
:10A630000821044800F09EFA00202CF0C6F9BDE87D
:10A64000F08100000000024010B50246107803E0DF
:10A6500012F8014B2318D8B20B1EA1F10104A1B2CC
:10A66000F6D110BD2C48807F012854D100212A4802
:10A6700081772A480078C0B9012028490870284805
:10A680000068C0002749D1F8301240EA810025490E
:10A69000D1F82C1240EA41002249D1F8281208438F
:10A6A0000F2181432048017017E000201B490870EA
:10A6B0001B480068C0001B49D1F8301240EA8100F5
:10A6C0001849D1F82C1240EA41001649D1F8281255
:10A6D00008430F218143154801701348007813493E
:10A6E0000978884217D11048007811490870084647
:10A6F00000781049097888420DD00D480078064945
:10A7000008760B4800780B4908700948007810B1AA
:10A7100001200149C8757047BC120020DE0A0020E4
:10A720003402424200004242DF0A0020E00A0020D8
:10A73000E10A0020DD0A002010B5ADF57C7D002483
:10A740007DA00068FB9000200090FEF78FFF14288A
:10A750007CD17A48FEF7A5FF794908700846007851
:10A76000142874D1FEF7B0FF0021764A03C2BDF869
:10A770000000FEF7F7FE6A464FF4FA7101A8FEF7F3
:10A780000FFF71A101A82CF049FD7149088008460E
:10A79000008810B300BF04E000216E480155601C22
:10A7A00084B2282CF8DB01A9694A128888186AA1AA
:10A7B0002CF034FD69490880002409E064480088D1
:10A7C000C01C204401A9095C62480155601C84B288
:10A7D00062480088001FA042F0DC61A101A82CF0B3
:10A7E0001DFD5B4908800846008820B3002405E071
:10A7F0000021584828300155601C84B2282CF7DB12
:10A8000001A9534A1288881853A12CF007FD534917
:10A81000088000240AE04E4800880830204401A93E
:10A82000095C4C4828300155601C84B24B480088B4
:10A830000938A042EFDC4DA101A82CF0EFFC4449FF
:10A8400008800846008830B3002407E06BE05BE036
:10A850000021404850300155601C84B2142CF7DBB5
:10A8600001A93B4A128888183BA12CF0D7FC3B4930
:10A87000088000240AE0364800880C30204401A9F2
:10A88000095C344850300155601C84B2334800885C
:10A890000D38A042EFDC39A101A82CF0BFFC2C49F7
:10A8A00008800846008820B3002405E000202949DC
:10A8B00046390855601C84B2322CF7DB01A9244AC2
:10A8C0001288881824A12CF0A9FC244908800024AF
:10A8D0000AE01F480088801D204401A9085C1D492A
:10A8E00046390855601C84B21C480088C01FA0422D
:10A8F000EFDC00210320FFF7D9FB0120FEF7C0FEAB
:10A9000001200DF57C7D10BD0D480078422803D153
:10A910000A48FEF7BCFE0CE00120FEF7B1FE002065
:10A920000749087005E00021164880F80A1F2CF03E
:10A9300009FC00BFE5E700000D0A0000480A0020FE
:10A94000380A0020400A002041504E3D000000001F
:10A950005E0A0020203A00203B0000005C0A002034
:10A96000574946494E414D453D000000574946492B
:10A9700050415353574F52443D00000053455256E7
:10A9800045523D00BC22002010B5044635488442A3
:10A9900008D10121084626F0C3FE0021012026F03F
:10A9A000BFFE5EE03048844208D10121022026F03B
:10A9B000B7FE0021022026F0B3FE52E02B4884426D
:10A9C00008D10121042026F0ABFE0021042026F04E
:10A9D000A7FE46E02648844208D10121082026F03F
:10A9E0009FFE0021082026F09BFE3AE02148844289
:10A9F00008D10121102026F093FE0021102026F01E
:10AA00008FFE2EE01C48844208D10121202026F030
:10AA100087FE0021202026F083FE22E01748844292
:10AA200008D10121402026F07BFE0021402026F0A5
:10AA300077FE16E01248844208D10121802026F0DA
:10AA40006FFE0021802026F06BFE0AE00D48844254
:10AA500007D10121801526F063FE0021A01526F004
:10AA60005FFE10BD000002400004024000080240EA
:10AA7000000C024000100240001402400018024086
:10AA8000001C024000200240F0B50A4600210023CD
:10AA9000002400BF3DE0012505FA01F3156805EA31
:10AAA00003049C4234D105684F000326BE40B543E1
:10AAB000056015794E00B540066835430560157987
:10AAC000012D02D01579022D16D185684F0003267D
:10AAD000BE40B543856055794E00B5408668354324
:10AAE0008560456801268E40B54345604568967986
:10AAF0008E40B6B235434560C5684F000326BE4060
:10AB0000B543C560D5794E00B540C6683543C560CC
:10AB1000491C1029BFD3F0BDF0B5002300244D0718
:10AB2000ED0E02FA05F3CE1000F1200555F826507F
:10AB30004E07F70E0F26BE40B543CF1000F120069A
:10AB400046F82750CE1000F1200555F8265045EA6A
:10AB50000304CE1000F1200545F82640F0BD024662
:10AB6000002013690B400BB1012000E0002070476A
:10AB700041837047018370470249087E0021014AE2
:10AB800011767047BC1200200E48006800F00100EA
:10AB900000B100BE012080F3138800BF00BFBFF3E7
:10ABA0004F8F0848E438006800F4E0600649084325
:10ABB000001D0449E4390860BFF34F8F00BF00BF98
:10ABC000FEE70000F0ED00E00000FA054AF6AA20DA
:10ABD00001490860704700000030004030B502466F
:10ABE0000024002305E012F8015B2819C4B2581CA8
:10ABF000C3B28B42F7DB6042C0B230BD10B5002457
:10AC00002CF0A0FA64202CF02BF910BD2DE9F043B4
:10AC1000ADF2DC7D07460D46164698460024A14657
:10AC20008EA00068CDF8D80700200190042E7CDCAF
:10AC30008B480079302101EB101006EBC60101EBC7
:10AC40000611884A114408718548007900F00F0008
:10AC5000303006EBC60101EB061111444871804803
:10AC6000C078302101EB101006EBC60101EB061194
:10AC7000114488717A48C07800F00F00303006EB3C
:10AC8000C60101EB06111144C871FEF7EFFC142850
:10AC900071D175480078142809D006EBC60101EB84
:10ACA0000611704A8818FEF7FCFC6F4908706E4860
:10ACB0000078142872D1B5F57A7F01DD4FF47A75EA
:10ACC000FEF702FD0021694A03C268480068FEF7EA
:10ACD00049FC6348C078302101EB10108DF8080062
:10ACE0005F48C07800F00F0030308DF809005C48F4
:10ACF000807801EB10108DF80A005948807800F038
:10AD00000F0030308DF80B005548407801EB1010E3
:10AD10008DF80C005248407800F00F0030308DF86C
:10AD20000D00534890F80B0F00E093E001EB10107A
:10AD30008DF80E004E4890F80B0F00F00F003030E9
:10AD40008DF80F00B8F1020F16D13A208DF81000DF
:10AD5000002406E0395D02AA04F109001154601CC8
:10AD600084B2AC42F6DB05F1090081B201AA02A867
:10AD7000FEF748FC47E067E0B8F1000F03D154202C
:10AD80008DF8100005E0B8F1010F02D152208DF8C6
:10AD900010003A208DF81100002429E040E0204600
:10ADA00004EBD0714910795C4FEA21190A2099FB14
:10ADB000F0F0C0EBC00109F130000844C1B202AAB2
:10ADC00004F10A001154204604EBD0714910795C5B
:10ADD00001F00F090A2099FBF0F0C0EBC00109F166
:10ADE00030000844C1B204F10B001154A01C84B21D
:10ADF000B4EB450FD3DB0A2000EB450081B201AA7A
:10AE000002A8FEF7FFFB01AA02210DF5FB60FEF789
:10AE1000F9FB0120FEF734FC00201349087019E00B
:10AE200011480078422808D106EBC60101EB061153
:10AE30000C4A8818FEF72BFC0CE00120FEF720FCE2
:10AE400000200949087005E00021094880F80A1F20
:10AE50002CF078F90DF2DC7DBDE8F0830D0A0000DE
:10AE6000C7310020600A0020380A0020400A002074
:10AE7000BC22002070B5BAB00021399138913791C9
:10AE80003691359134913391329100223092319242
:10AE90002E922F922D912C912B912A9129912891CC
:10AEA0002791269125912491239115911491139125
:10AEB0001291119110910F919FEDFE0A8DED0E0AE6
:10AEC000FDA006C8CDE90C12FDA006C8CDE90A1206
:10AED000BAE0FD48807858B30020FB498870FB48F1
:10AEE000B0F8C406FA490968C1F57A7188421FD1E1
:10AEF000F7480068C0F57A7081B2F448A0F8BC1633
:10AF00000021F348001FFEF783FDF249F048001FBF
:10AF1000FEF764FD0120F04908704FF47A70EC49A7
:10AF20008C39C1F88C000121E948001FFEF770FD43
:10AF3000E548807B50B30021E3488173E7484088AF
:10AF4000E3498C39496CC1F57A7188421ED1E048D9
:10AF50008C38406CC0F57A70E0490839488000218F
:10AF6000DB484C38FEF754FDDD49D9484C38FEF734
:10AF700035FD0120DB4908704FF47A70D4498C39D3
:10AF800048640121D2484C38FEF742FDCE48807E0D
:10AF900050B30021CC488176D0488088CC498C3988
:10AFA0004969C1F57A7188421ED1C9488C38406917
:10AFB000C0F57A70C949083988800021C4487C38B6
:10AFC000FEF726FDC849C2487C38FEF707FD012080
:10AFD000C64908704FF47A70BD498C394861012127
:10AFE000BB487C38FEF714FDB74890F8260058B3EC
:10AFF0000021B54880F82610B848C088B4498C397B
:10B00000C96AC1F57A7188421ED1B1488C38C06ACC
:10B01000C0F57A70B1490839C8800021AC4864385D
:10B02000FEF7F6FCB249AA486438FEF7D7FC0120C7
:10B03000B04908704FF47A70A5498C39C862012173
:10B04000A3486438FEF7E4FC9F488178807B014484
:10B050009D48807E01449C4890F8260008440028C2
:10B060007FF437AF13F056BA9B48007820B1002028
:10B07000994908702D9019E09A48007828B100206D
:10B080009849087001202D9010E09848007828B168
:10B0900000209649087002202D9007E0954800781E
:10B0A00020B100209349087003202D909DF8B41022
:10B0B00001EB4100C0EBC1108F4911F83000C128ED
:10B0C00036D19DF8B41001EB4100C0EBC1108A49A4
:10B0D00001EBC000807808282AD101217B4880F844
:10B0E00014179DF8B40030B101280AD002280ED000
:10B0F000032818D111E04FF480418048FFF738FD54
:10B1000011E04FF400517D48FFF732FD0BE04FF4A2
:10B1100080517A48FFF72CFD05E04FF40061774835
:10B12000FFF726FD00BF00BF00207549086099E7C2
:10B1300065480C389DF8B41010F811000121B1EBEE
:10B14000D01F53F042806F4890F80A0FB8B163499E
:10B1500008399DF8B40031F8101009919DF8B40039
:10B1600000EB4001C1EBC011634800EBC1010123BA
:10B1700008919DF8B420DDE90801FFF747FD9DF82F
:10B18000B41001EB410000EB01105F4901EB00102E
:10B1900081792C919DF8B0000C2892F0FB87DFE8B4
:10B1A00010F0BD960C001A17C62AE63A1A3D314136
:10B1B000E94F485E056E8F83BE969DF8B41001EB93
:10B1C0004100C0EBC1104C4901EBC000417808467A
:10B1D000099100211BF01CFDC1B22891002136917C
:10B1E0001CE09DF8B41001EB410000EB0110464952
:10B1F00001EB00113031BDF8D80001EB00104178AF
:10B200009DF8A000814204D1BDF8D800C1B22891B8
:10B2100012E0BDF8D800401C81B236919DF8B41000
:10B2200001EB410000EB0110374901EB0010C1793F
:10B23000BDF8D8008142D4DC00BF9DF8B40000EB1B
:10B240004001C1EBC0102C4901EBC000807800F038
:10B25000F000A0280DD19DF8B41001EB4100C0EB27
:10B26000C110254901EBC000807800F00F01299141
:10B270000AE09DF8B41001EB4100C0EBC1111E487B
:10B2800000EBC10081782991BDF8A40008B9102015
:10B2900029909DF8B41001EB4100C0EBC110164994
:10B2A00001EBC001BDF8A400401C095C2591BDF86C
:10B2B000A4002BE000000000016932303130300082
:10B2C0000169323045303000283E0020BC72002039
:10B2D0008C6002400088002012000020807900204D
:10B2E0000080201013000020208000101400002097
:10B2F0000088001015000020F88700200018024088
:10B3000088024242BC22002098400020401C81B2AA
:10B3100009919DF8B41001EB4100C0EBC111FE484A
:10B3200000EBC1010891DDE908011CF001F937903B
:10B330009DF8B41001EB4100C0EBC110F64901EBE0
:10B34000C001BDF8A400801C095CBDF8DC0081428E
:10B3500042F03F869DF8B41001EB4100C0EBC110F4
:10B36000ED4901EBC0004078002842F332869DF899
:10B37000B41001EB4100C0EBC110E74901EBC00183
:10B38000BDF8A400C01C0A5C9DF8B40040F2A111F5
:10B3900010FB01F0E14901EBC00101F562719DF87C
:10B3A000A00000EB400303EB001001EBC00080F8AD
:10B3B00044200021DA4A9DF8B40002EB00129DF807
:10B3C000A0001154D74890F82800012840D19DF8DA
:10B3D000B40000EB400101EB0010D34901EB001079
:10B3E00030309DF8A01000EB0110801C099000780F
:10B3F00020F08000803009990870BDF89400B628CC
:10B4000014D0C52819D0D52802D0D9281CD106E0DF
:10B41000BDF8A400032801DA0020259017E0BDF84C
:10B42000A400032801DA0020259010E0BDF8A40054
:10B43000032801DA0020259009E0BDF8A4000328C4
:10B4400001DA0020259002E00020259000BF00BF17
:10B45000BDF89400C3287DD01DDCB32801F08083A3
:10B460000DDC112802F08084122802F0C584132814
:10B4700002F05785B22842F0AB8501F0C8BDB5286F
:10B4800001F08483B62801F07884B92801F0FD83A7
:10B49000BA28F0D1FDE3D9287ED00ADCC52801F016
:10B4A000EE85CA2879D0CE2802F05283D528E2D181
:10B4B00009E0E12802F06283E52802F07583E728BD
:10B4C000D9D102F037BC9DF8B41001EB4100C0EBBC
:10B4D000C110914901EBC000C178944880F8021D69
:10B4E0009DF8B41040F2A11011FB00F08B4901EB64
:10B4F000C00101F562719DF8A00000EB400202EB73
:10B50000001011F830109DF8B40040F2A11210FBA9
:10B5100002F0824A02EBC000407981427DDA9DF858
:10B52000B41001EB410000EB01107F4901EB00106A
:10B5300030309DF8A01000EB0110801C09907B4872
:10B5400090F8021D0120A0EBD1120998007862F357
:10B55000000000E0FEE309990870744890F8020DBD
:10B56000C0F34010F0BB9DF8B40000EB400101EBCC
:10B5700000106D4901EB001030309DF8A01000EB79
:10B5800001108078C0F3401060B39DF8B40000EB68
:10B59000400101EB001001E0FEE3FEE3624901EB34
:10B5A000001030309DF8A01000EB0110801C0990B5
:10B5B000007820F00200801C099908709DF8B410F2
:10B5C00040F2A11011FB00F0544901EBC00000F55E
:10B5D00062709DF8A01001EB410202EB011100EB3B
:10B5E000C10000E00CE018300990007820F0020063
:10B5F000801C099908709DF8B4100220FEF756FDD2
:10B6000000219DF8B40040F2A11210FB02F0434A61
:10B6100002EBC0000171022200E028E09DF8B400B6
:10B6200040F2A11110FB01F03C4901EBC00101F512
:10B6300062719DF8A00000EB400303EB001001F8DD
:10B640003020B6229DF8B40040F2A11110FB01F0A9
:10B65000324901EBC00000F562709DF8A01001EBCB
:10B66000410303EB011100EBC1004271FDE32F48E0
:10B6700090F8020DC0F3C000A8B9E5229DF8B4000F
:10B6800040F2A11110FB01F0244901EBC00000F5CC
:10B6900062709DF8A01001EB410303EB011100EB78
:10B6A000C1004271E2E79DF8B41001EB410000EBEC
:10B6B00001101D4901EB001030309DF8A01000EB87
:10B6C0000110801C0990194890F8021D0120A0EB80
:10B6D000D11009990A7860F300020A709DF8B4103D
:10B6E00001EB410000EB01100F4901EB001030307D
:10B6F0009DF8A01000EB0110801C09900B4890F8F9
:10B70000020D42090998007862F341000999087016
:10B710009DF8B4100CE00000F88700205845002088
:10B72000883E0020BC12002098400020BC2200204F
:10B7300001EB410000EB0110FE4901EB001030303D
:10B740009DF8A01000EB01108078C0F340029DF836
:10B75000B40040F2A11110FB01F0F74901EBC00069
:10B7600000F562709DF8A01001EB410303EB01119D
:10B7700000EBC100007EC0F3400082427BD09DF808
:10B78000B41040F2A11011FB00F0EB4901EBC00036
:10B7900000F562709DF8A01001EB410202EB01116F
:10B7A00000EBC100183009909DF8B40000EB400197
:10B7B00001EB0010DF4901EB001030309DF8A010C4
:10B7C00000EB0110807842080998007862F341008C
:10B7D000099908709DF8B41001EB410000EB0110CD
:10B7E000D44901EB001030309DF8A01000EB01109F
:10B7F0008078C0F34000E8B3D9229DF8B40040F24D
:10B80000A11110FB01F0CC4901EBC00000F5627002
:10B810009DF8A01001EB410303EB011100EBC10007
:10B820004271C64890F8E00700287CD19DF8B4101A
:10B8300040F2A11011FB00F0BF4901EBC00000F580
:10B8400062709DF8A01001EB410202EB011100EBC8
:10B85000C10090F87F00002865D011239DF8B40046
:10B8600040F2A11110FB01F0B34901EBC00101F559
:10B87000627101E06EE088E19DF8A00000EB4002FB
:10B8800002EB001001EBC00090F8800040F2A11123
:10B8900010FB01F0A84901EBC00101F562719DF8B0
:10B8A000B40040F2A11210FB02F0A34A02EBC00266
:10B8B00002F562729DF8A00000EB400404EB00105A
:10B8C00002EBC00090F8810000EB400202EB001098
:10B8D00001EBC00080F87E30F3239DF8B40040F205
:10B8E000A11110FB01F0944901EBC00101F5627157
:10B8F0009DF8A00000EB400202EB001001EBC0003D
:10B9000090F8800040F2A11110FB01F08A4901EB90
:10B91000C00101F562719DF8B40040F2A11210FB64
:10B9200002F0854A00E096E002EBC00000F562708C
:10B930009DF8A02002EB420404EB021200EBC200CF
:10B9400090F8810000EB400202EB001001EBC00018
:10B95000437115E101229DF8B40040F2A11110FBE2
:10B9600001F0754901EBC00101F562719DF8A0007D
:10B9700000EB400303EB001001EBC0004273D9223F
:10B980009DF8B40040F2A11110FB01F06A4901EBEF
:10B99000C00101F562719DF8A00000EB400303EBCC
:10B9A000001001EBC000427101229DF8B40040F28A
:10B9B000A11110FB01F0604901EBC00000F56270BD
:10B9C0009DF8A01001EB410303EB011100EBC10056
:10B9D00080F84620594890F8E007E0BB9DF8B40095
:10B9E00040F2A11110FB01F0534901EBC00000F53A
:10B9F00062709DF8A01001EB410202EB011100EB17
:10BA0000C10090F87F0030B39DF8B41040F2A1104F
:10BA100011FB00F0484901EBC00101F562719DF88E
:10BA2000A00000EB400202EB001001EBC00090F818
:10BA3000801001EB410000EB01103E4901EB0011C9
:10BA400030319DF8B40040F2A11210FB02F03A4AE6
:10BA500002EBC00200E093E002F562729DF8A000E4
:10BA600000EB400303EB001002EBC00090F88100F4
:10BA700001EB0010801C0990007820F00402099866
:10BA8000027000239DF8B40040F2A11110FB01F0F8
:10BA9000294901EBC00000F562709DF8A01001EB90
:10BAA000410202EB011100EBC10090F8800040F26E
:10BAB000A11110FB01F0204901EBC00000F56270FC
:10BAC0009DF8B41040F2A11211FB02F11A4A02EBE8
:10BAD000C10202F562729DF8A01001EB410404EB73
:10BAE000011102EBC10191F8811001EB410202EB5F
:10BAF000011100EBC10080F87E30F3239DF8B40003
:10BB000040F2A11110FB01F00B4901EBC00000F560
:10BB100062709DF8A01001EB410202EB011100EBF5
:10BB2000C10090F8800040F2A11110FB01F0024921
:10BB300006E000009840002058450020BC3200205C
:10BB400001EBC00000F562709DF8B41040F2A11244
:10BB500011FB02F1FE4A02EBC10101F562719DF891
:10BB6000A02002EB420404EB021201EBC20191F8A7
:10BB7000811001EB410202EB011100EBC1004371A6
:10BB80009DF8B4100220FEF791FA9DF8B40000EB86
:10BB9000400101EB0010EF4901EB001130319DF83D
:10BBA000A00001EB0010807800F001029DF8B400C5
:10BBB00040F2A11110FB01F0E54901EBC00000F5D6
:10BBC00062709DF8A01001EB410303EB011100EB43
:10BBD000C100007E00F0010082427AD09DF8B400DE
:10BBE00040F2A11110FB01F0D94901EBC00000F5B2
:10BBF00062709DF8A01001EB410202EB011100EB15
:10BC0000C100183009909DF8B40000EB400101EB31
:10BC10000010D04901EB001030309DF8A01000EB6F
:10BC20000110807809990A7860F300020A709DF883
:10BC3000B41001EB410000EB0110C64901EB00100C
:10BC400030309DF8A01000EB0110807800F001006A
:10BC5000F0BB9DF8B41001EB410000EB0110BD49B1
:10BC600001EB001030309DF8A01000EB011080783F
:10BC7000C0F3401070B39DF8B41040F2A11011FB56
:10BC800000F0B34901EBC00000F562709DF8A01010
:10BC900000E0E8E301EB410202EB011100EBC1001F
:10BCA00090F84600B0B99DF8B41040F2A11011FB15
:10BCB00000F0A74901EBC00000F562709DF8A010EC
:10BCC00001EB410202EB011100EBC100407B02E0FD
:10BCD00071E0AAE23FE0F0BB9DF8B41001EB410037
:10BCE00000EB01109B4901EB001030309DF8A010D3
:10BCF00000EB01108078C0F3400060BB01229DF88A
:10BD0000B40040F2A11110FB01F0914901EBC00118
:10BD100001F562719DF8A00000EB400303EB0010F9
:10BD200001EBC0004273D9229DF8B40040F2A1118A
:10BD300010FB01F0864901EBC00101F562719DF82D
:10BD4000A00000EB400303EB001001EBC0004271C8
:10BD5000012201E0F1E314E09DF8B40040F2A111EA
:10BD600010FB01F07A4901EBC00000F562709DF80C
:10BD7000A01001EB410303EB011100EBC10080F8BF
:10BD8000462000229DF8B40040F2A11110FB01F002
:10BD90006F4901EBC00001E0FDE3FDE300F56270D7
:10BDA0009DF8A01001EB410303EB011100EBC10072
:10BDB00080F8452034E29DF8B41040F2A11011FB48
:10BDC00000F0634901EBC00000F562709DF8A0101F
:10BDD00001EB410202EB011100EBC10090F84600BB
:10BDE000B0B901229DF8B40040F2A11110FB01F09E
:10BDF000574901EBC00000F562709DF8A01001EBFF
:10BE0000410303EB011100EBC10080F845202AE05B
:10BE100000229DF8B40040F2A11110FB01F04C4942
:10BE200001EBC00101F562719DF8A00000EB400339
:10BE300003EB001001EBC00080F845209DF8B41022
:10BE400001EB410000EB0110424901EB00113031E0
:10BE50009DF8A00001EB0010801C0990007820F0F4
:10BE60000102099802703C4800E06AE290F8E0079D
:10BE700080B19DF8B41001EB410000EB0110354991
:10BE800001EB001030309DF8A01000EB0110807A1B
:10BE900002288FD1314890F8290001288AD12F48F3
:10BEA000D0F80C022D49498D88427DD29DF8B4000E
:10BEB00040F2A11110FB01F0254901EBC00000F593
:10BEC00062709DF8A01001EB410202EB011100EB42
:10BED000C10090F84500012839D19DF8B40040F226
:10BEE000A11110FB01F01A4901EBC00000F56270CE
:10BEF0009DF8A01001EB410202EB011100EBC10023
:10BF000090F87F0018BB9DF8B40000EB400101EBF6
:10BF10000010104901EB001130319DF8A00001EB39
:10BF2000001001789DF8B40040F2A11210FB02F05D
:10BF3000074A02EBC0004170C3229DF8B40040F2F2
:10BF4000A11110FB01F0024901EBC00108E082E001
:10BF50005845002098400020BC320020BC12002030
:10BF600001F562719DF8A00000EB400303EB0010A7
:10BF700001EBC000427100229DF8B40000EB4001CB
:10BF800001EB0010FE4901EB001130319DF8A000DB
:10BF900001EB0010426001229DF8B40000EB40016B
:10BFA00001EB0010F64900E0EAE001EB001130314E
:10BFB0009DF8A00001EB0010C2729DF8B4100220A1
:10BFC000FEF774F8002139911CE000229DF8B400BE
:10BFD00040F2A11110FB01F0EA4901EBC00101F5AB
:10BFE00062719DF8A00000EB400303EB001001EB31
:10BFF000C0014731BDF8E4000A54BDF8E400401C1C
:10C0000081B23991BDF8E4000628DEDB00203990CA
:10C010001CE000229DF8B40040F2A11110FB01F0D9
:10C02000D84901EBC00101F562719DF8A00000EB59
:10C03000400303EB001001EBC0016331BDF8E400E5
:10C040000A54BDF8E400401C81B23991BDF8E40007
:10C050000F28DEDBE4E09DF8B41040F2A11011FBE4
:10C0600000F0C84901EBC00000F562709DF8A01017
:10C0700001EB410202EB011100EBC10090F8450019
:10C0800001287DD19DF8B41040F2A11011FB00F001
:10C09000BC4901EBC00101F562719DF8A00000EB05
:10C0A000400202EB001001EBC00090F8801040F25B
:10C0B000A11011FB00F0B34901EBC00101F5627161
:10C0C0009DF8B40040F2A11210FB02F0AD4A02EB61
:10C0D000C00000F562709DF8A02002EB420303EB64
:10C0E000021200EBC20090F8810000EB400202EB6C
:10C0F000001001EBC00090F87E00032840D100231F
:10C100009DF8B40040F2A11110FB01F09D4901EB34
:10C11000C00101F562719DF8A00000EB400202EB46
:10C12000001001EBC00090F8800040F2A11110FB5C
:10C1300001F0944901EBC00101F562719DF8B40072
:10C1400040F2A11210FB02F08E4A02EBC00202F58F
:10C1500062729DF8A00000EB400404EB001002EBBB
:10C16000C00090F8810000EB400202EB001001EBF0
:10C17000C00080F87E309DF8B41001EB410000E073
:10C180004EE000EB01107E4901EB001130319DF8CB
:10C19000A00001EB001001789DF8B40040F2A1125C
:10C1A00010FB02F0774A02EBC0004170C3229DF8F9
:10C1B000B40040F2A11110FB01F0724901EBC00183
:10C1C00001F562719DF8A00000EB400303EB001045
:10C1D00001EBC000427100229DF8B40000EB400169
:10C1E00001EB0010664901EB001130319DF8A00011
:10C1F00001EB0010426002229DF8B40000EB400108
:10C2000001EB00105E4901EB001130319DF8A000F8
:10C2100001EB0010C2729DF8B4100220FDF746FF3A
:10C220009DF8B4100220FDF741FF9DF8B41001EB1A
:10C23000410000EB0110524901EB001030309DF835
:10C24000A01000EB01108078C0F3400050B39DF8BF
:10C25000B41040F2A11011FB00F04A4901EBC000FC
:10C2600000F562709DF8A01001EB410202EB011194
:10C2700000EBC1004079D52814D1D9229DF8B40033
:10C2800040F2A11110FB01F03E4901EBC00000F5A6
:10C2900062709DF8A01001EB410303EB011100EB6C
:10C2A000C10042719DF8B41040F2A11011FB00F0E2
:10C2B000344901EBC00000F562709DF8A01001EB5D
:10C2C000410202EB011100EBC1008078B22838D1A5
:10C2D0009DF8B41001EB410000EB0110284901EB7F
:10C2E000001030309DF8A01000EB01108078C0F3F2
:10C2F000400030BB9DF8B40000EB400101EB0010A2
:10C300001F4901EB001030309DF8A01000EB011028
:10C310008078C0F34010A0B9E5229DF8B40040F247
:10C32000A11110FB01F0174901EBC00000F562708C
:10C330009DF8A01001EB410303EB011100EBC100DC
:10C3400042719DF8B40000EB400101EB00100C4974
:10C3500001EB001030309DF8A01000EB0110807848
:10C360000121B1EBD01F7DD19DF8B40000EB40015D
:10C3700001EB0010024901EB0010303004E0000036
:10C3800098400020584500209DF8A01000EB0110B7
:10C39000807800F00100002864D19DF8B40040F2DC
:10C3A000A11110FB01F0F84901EBC00000F562702B
:10C3B0009DF8A01001EB410202EB011100EBC1005E
:10C3C00090F8460000284DD19DF8B40000EB4001E4
:10C3D00001EB0010ED4901EB001030309DF8A0108A
:10C3E00000EB01108078C0F3C000D8BB9DF8B4000A
:10C3F00000EB400101EB0010E44901EB001030308C
:10C400009DF8A01000EB0110407A00F0010048B345
:10C410009DF8B40040F2A11110FB01F0DA4901EBE4
:10C42000C00000F562709DF8A01001EB410202EB24
:10C43000011100EBC10090F8900000F0010088B9F4
:10C440009DF8B40040F2A11110FB01F0CE4901EBC0
:10C45000C00000F562709DF8A01001EB410202EBF4
:10C46000011101E040E05AE300EBC10090F88200C6
:10C47000D0B3002039902CE09DF8B40040F2A11117
:10C4800010FB01F0C04901EBC00101F562719DF89C
:10C49000A00000EB400202EB001001EBC00000F135
:10C4A0008301BDF8E4000A5C9DF8B40000EB400194
:10C4B00001EB0010B54901EB00100E30BDF8E4109F
:10C4C000405C824200D008E0BDF8E400401C81B22C
:10C4D0003991BDF8E4000628CEDB00BFBDF8E400CA
:10C4E00006286CD139902EE069E09DF8B41040F236
:10C4F000A11011FB00F0A44901EBC00101F562712C
:10C500009DF8A00000EB400202EB001001EBC00020
:10C5100000F18301BDF8E4000A5C9DF8B40000EB73
:10C52000400101EB0010994901EB00100E30BDF8FD
:10C53000E410405C824201D009E09EE2BDF8E400D4
:10C54000401C81B23991BDF8E4000A28CDDB00BF60
:10C55000BDF8E4000A2832D09DF8B41040F2A110D2
:10C5600011FB00F0884901EBC00000F562709DF8F6
:10C57000A01001EB410202EB011100EBC100903071
:10C580000990007820F00100401C099908701222DF
:10C590009DF8B40001E014E0ABE240F2A11110FB01
:10C5A00001F0794901EBC00000F562709DF8A01020
:10C5B00001EB410303EB011100EBC100427101F0FB
:10C5C00007BD9DF8B41001EB410000EB01106F496D
:10C5D00001EB0010007BD0BBBDF8A400082800D000
:10C5E000EDE70020399028E09DF8B41001EB410000
:10C5F000C0EBC110664901EBC001BDF8E400C01CEE
:10C60000085C00F00F00092800DD1AE09DF8B41066
:10C6100001EB4100C0EBC1105D4901EBC001BDF869
:10C62000E400C01C085C00F0F000902800DD08E089
:10C63000BDF8E400401C81B23991BDF8E400062841
:10C64000D2DB00BFBDF8E400062801DAB7E76EE0F0
:10C650009DF8B41001EB4100C0EBC1104C4901EB57
:10C66000C000C07801049DF8B40000EB4002C2EBAA
:10C67000C010474A02EBC000007941EA00219DF852
:10C68000B40000EB4002C2EBC010414A02EBC00014
:10C69000407901439DF8B40040F2A11210FB02F072
:10C6A000394A02EBC00202F562729DF8A00000EB6D
:10C6B000400303EB001002EBC000C0F81A109DF815
:10C6C000B41001EB4100C0EBC110314901EBC000D7
:10C6D000807901049DF8B40000EB4002C2EBC01069
:10C6E0002B4A02EBC000C07941EA00219DF8B4005A
:10C6F00000EB4002C2EBC010254A02EBC000007AFA
:10C7000001439DF8B40040F2A11210FB02F01E4A52
:10C7100002EBC00000F562709DF8A02002EB42031E
:10C7200003EB021200EBC200C0F81E10C7E0BDF818
:10C73000A4000A2800D042E7002039902FE09DF89D
:10C74000B40000EB4001C1EBC010114901EBC00186
:10C75000BDF8E400C01C085C00F00F00092800DDF3
:10C7600021E09DF8B40000EB4001C1EBC010084986
:10C7700001EBC001BDF8E400C01C085C00F0F00053
:10C78000902807DD0FE00000584500209840002069
:10C79000F8870020BDF8E400401C81B23991BDF853
:10C7A000E4000828CBDB00BFBDF8E400082800DA6D
:10C7B00005E79DF8B40000EB4001C1EBC010FE4955
:10C7C00001EBC000C07801069DF8B40000EB400208
:10C7D000C2EBC010F84A02EBC000007941EA004108
:10C7E0009DF8B40000EB4002C2EBC010F24A02EB2D
:10C7F000C000407941EA00219DF8B40000EB4002FE
:10C80000C2EBC010EC4A02EBC000807901439DF8F6
:10C81000B40040F2A11210FB02F0E84A02EBC002A1
:10C8200002F562729DF8A00000EB400303EB0010DC
:10C8300002EBC000C0F81A109DF8B40000EB4001F4
:10C84000C1EBC011DC4800EBC100C07901069DF8C6
:10C85000B40000EB4002C2EBC010D74A02EBC000AC
:10C86000007A41EA00419DF8B40000EB4002C2EBBF
:10C87000C010D14A02EBC000407A41EA00219DF885
:10C88000B40000EB4002C2EBC010CB4A02EBC00088
:10C89000807A01439DF8B40040F2A11210FB02F02F
:10C8A000C64A02EBC00000F562709DF8A02002EBC2
:10C8B000420303EB021200EBC200C0F81E109DF809
:10C8C000B40040F2A11110FB01F0BC4901EBC00122
:10C8D00001F562719DF8A00000EB400202EB001030
:10C8E00011F830109DF8B40040F2A11210FB02F0D4
:10C8F000B24A02EBC0004079814234DA00219DF84F
:10C90000B40040F2A11210FB02F0AC4A02EBC000EE
:10C91000017104229DF8B40040F2A11110FB01F056
:10C92000A64901EBC00101F562719DF8A00000EB82
:10C93000400303EB001001F83020C5229DF8B4003D
:10C9400040F2A11110FB01F09C4901EBC00000F581
:10C9500062709DF8A01001EB410303EB011100EBA5
:10C96000C100427188E09DF8B41001EB410000EB7A
:10C970000110934901EB001030309DF8A01000EB3E
:10C9800001108078C0F3400058B39DF8B41040F215
:10C99000A11011FB00F0894901EBC00000F56270A5
:10C9A0009DF8A01001EB410202EB011100EBC10068
:10C9B0004079D92815D1D5229DF8B40040F2A111B3
:10C9C00010FB01F07D4901EBC00000F562709DF89D
:10C9D000A01001EB410303EB011100EBC100427118
:10C9E0004AE09DF8B41040F2A11011FB00F0734929
:10C9F00001EBC00000F562709DF8A01001EB410250
:10CA000002EB011100EBC100807B012834D1002230
:10CA10009DF8B40040F2A11110FB01F0674901EB51
:10CA2000C00101F562719DF8A00000EB400303EB2B
:10CA3000001001EBC0008273B6229DF8B40040F2F2
:10CA4000A11110FB01F05D4901EBC00101F562711C
:10CA50009DF8A00000EB400303EB001001EBC000C9
:10CA6000427100219DF8B40040F2A11210FB02F0C7
:10CA7000524A02EBC0000171A1E5D5229DF8B40035
:10CA800040F2A11110FB01F04C4901EBC00101F58E
:10CA900062719DF8A00000EB400303EB001001EB76
:10CAA000C000427101219DF8B40040F2A11210FBB8
:10CAB00002F0424A02EBC00001719DF8B41001EB94
:10CAC000410000EB01103E4901EB001130319DF8AF
:10CAD000A00001EB0010801C0990007820F02000DD
:10CAE0002030099908709DF8B4100220FDF7DEFA95
:10CAF00065E5D5229DF8B40040F2A11110FB01F0CC
:10CB00002E4901EBC00000F562709DF8A01001EB0A
:10CB1000410303EB011100EBC10042714FE5D52247
:10CB20009DF8B40040F2A11110FB01F0234901EB84
:10CB3000C00101F562719DF8A00000EB400303EB1A
:10CB4000001001EBC000427101219DF8B40040F2D9
:10CB5000A11210FB02F0194A02EBC00001712EE590
:10CB6000D5229DF8B40040F2A11110FB01F0134949
:10CB700001EBC00000F562709DF8A01001EB4103CD
:10CB800003EB011100EBC100427118E59DF8B410F0
:10CB900040F2A11011FB00F0084901EBC00000F5C4
:10CBA0006270BDF8D81001EB410202EB011100EBFD
:10CBB000C1008079012805E0F88700205845002051
:10CBC0009840002040D100229DF8B40040F2A1110D
:10CBD00010FB01F0FA4901EBC00101F56271BDF8EB
:10CBE000D80000EB400303EB001001EBC0008271A2
:10CBF000D5229DF8B40040F2A11110FB01F0F049DC
:10CC000001EBC00101F562719DF8A00000EB40034B
:10CC100003EB001001EBC00042719DF8B41001EB72
:10CC2000410000EB0110E74901EB001130319DF8A4
:10CC3000A00001EB0010801C0990007820F0040097
:10CC4000001D099908701FE0C3229DF8B40040F24E
:10CC5000A11110FB01F0DA4901EBC00101F562718D
:10CC60009DF8A00000EB400303EB001001EBC000B7
:10CC7000427100219DF8B40040F2A11210FB02F0B5
:10CC8000CF4A02EBC000017199E49DF8B41040F264
:10CC9000A11011FB00F0CA4901EBC00000F5627061
:10CCA000BDF8D81001EB410202EB011100EBC1000D
:10CCB0008079012840D100229DF8B40040F2A111F2
:10CCC00010FB01F0BE4901EBC00101F56271BDF836
:10CCD000D80000EB400303EB001001EBC0008271B1
:10CCE000D5229DF8B40040F2A11110FB01F0B44927
:10CCF00001EBC00101F562719DF8A00000EB40035B
:10CD000003EB001001EBC00042719DF8B41001EB81
:10CD1000410000EB0110AB4901EB001130319DF8EF
:10CD2000A00001EB0010801C0990007820F00400A6
:10CD3000001D099908701FE0C3229DF8B40040F25D
:10CD4000A11110FB01F09E4901EBC00101F56271D8
:10CD50009DF8A00000EB400303EB001001EBC000C6
:10CD6000427100219DF8B40040F2A11210FB02F0C4
:10CD7000934A02EBC000017121E49DF8B41001EB6D
:10CD8000410000EB01108F4901EB0010007B50BB0C
:10CD90009DF8B41001EB4100C0EBC1108A4901EBD2
:10CDA000C00001799DF8B40000EB4002C2EBC01056
:10CDB000854A02EBC000C07841EA00229DF8B40029
:10CDC00040F2A11110FB01F07D4901EBC00000F51C
:10CDD00062709DF8A01001EB410303EB011100EB21
:10CDE000C100426335E09DF8B41001EB4100C0EB97
:10CDF000C110754901EBC000C07801049DF8B40072
:10CE000000EB4002C2EBC0106F4A02EBC000007999
:10CE100041EA00219DF8B40000EB4002C2EBC010D3
:10CE2000694A02EBC000407901439DF8B40040F22A
:10CE3000A11210FB02F0624A02EBC00000F5627022
:10CE40009DF8A02002EB420303EB021200EBC200AC
:10CE500041639DF8B41040F2A11011FB00F0584955
:10CE600001EBC00101F562719DF8A00000EB4002EA
:10CE700002EB001011F830109DF8B40040F2A1123E
:10CE800010FB02F04E4A02EBC0004079814234DAD6
:10CE900000219DF8B40040F2A11210FB02F0484AB4
:10CEA00002EBC000017103229DF8B40040F2A11111
:10CEB00010FB01F0424901EBC00101F562719DF8E0
:10CEC000A00000EB400303EB001001F83020D92252
:10CED0009DF8B40040F2A11110FB01F0384901EBBC
:10CEE000C00000F562709DF8A01001EB410303EB58
:10CEF000011100EBC100427188E09DF8B40040F2DE
:10CF0000A11110FB01F02E4901EBC00000F5627089
:10CF1000BDF8D81001EB410202EB011100EBC1009A
:10CF20008079012852D100229DF8B40040F2A1116D
:10CF300010FB01F0224901EBC00101F56271BDF85F
:10CF4000D80000EB400303EB001001EBC00082713E
:10CF5000D9229DF8B40040F2A11110FB01F018494C
:10CF600001EBC00101F562719DF8A00000EB4003E8
:10CF700003EB001001EBC00042719DF8B40000EB20
:10CF8000400101EB00100F4901EB001130319DF819
:10CF9000A00001EB0010801C0990007820F0040034
:10CFA000001D0999087001209DF8B41040F2A112EB
:10CFB00011FB02F1024A02EBC101087126E00000F8
:10CFC0005845002098400020F8870020C5229DF891
:10CFD000B40040F2A11110FB01F0FE4901EBC001C9
:10CFE00001F562719DF8A00000EB400303EB001017
:10CFF00001EBC000427100219DF8B40040F2A11283
:10D0000010FB02F0F34A02EBC000017134E500218D
:10D010009DF8B40040F2A11210FB02F0ED4A02EBC1
:10D02000C00001719DF8B41001EB410000EB01104C
:10D03000A2F5986101EB001130319DF8A00001EBE1
:10D040000010801C0990007820F00400001D099950
:10D050000870D5229DF8B40040F2A11110FB01F038
:10D06000DC4901EBC00000F562709DF8A01001EBF7
:10D07000410303EB011100EBC1004271FCE49DF898
:10D08000B41001EB410000EB0110D34901EB00109B
:10D09000007BD0BBBDF8A4000C2800D0ECE400213C
:10D0A000399128E09DF8B41001EB4100C0EBC110AC
:10D0B000CA4901EBC001BDF8E400C01C085C00F0E7
:10D0C0000F00092800DD1AE09DF8B41001EB4100C3
:10D0D000C0EBC110C14901EBC001BDF8E400C01CA8
:10D0E000085C00F0F000902800DD08E0BDF8E400E6
:10D0F000401C81B23991BDF8E4000A28D2DB00BFA0
:10D10000BDF8E4000A2801DAB6E482E000202E909F
:10D110002F90002139911EE0DDE92E10000240EA37
:10D1200011620902CDE92E129DF8B41001EB410005
:10D13000C0EBC110A94901EBC001BDF8E400C01C5F
:10D14000085CDDE92E341843CDE92E04BDF8E40077
:10D15000401C80B23990BDF8E4000528DCDB9DF866
:10D16000B400DDE92E1240F2A11310FB03F399483D
:10D1700000EBC30303F562739DF8A00000EB4004CD
:10D1800004EB001003EBC00040F8221F42600022B5
:10D190002E922F92002139911EE0DDE92E1000021F
:10D1A00040EA11620902CDE92E129DF8B41001EB9C
:10D1B0004100C0EBC110894901EBC001BDF8E4009A
:10D1C0000830085CDDE92E341843CDE92E04BDF8A3
:10D1D000E400401C80B23990BDF8E4000528DCDB97
:10D1E0009DF8B400DDE92E1240F2A11310FB03F00C
:10D1F000784B03EBC00000F562709DF8A03003EBA4
:10D20000430404EB031300EBC30022308160C260CF
:10D21000BCE0BDF8A4000E2800D02DE40020399019
:10D2200028E09DF8B41001EB4100C0EBC1106B4940
:10D2300001EBC001BDF8E400C01C085C00F00F0069
:10D24000092800DD1AE09DF8B41001EB4100C0EBA5
:10D25000C110624901EBC001BDF8E400C01C085CCC
:10D2600000F0F000902800DD08E0BDF8E400401C6C
:10D2700081B23991BDF8E4000C28D2DB00BFBDF8C3
:10D28000E4000C2800DA33E400202E902F900021D7
:10D2900039911EE0DDE92E10000240EA1162090218
:10D2A000CDE92E129DF8B41001EB4100C0EBC11086
:10D2B0004A4901EBC001BDF8E400C01C085CDDE98F
:10D2C0002E341843CDE92E04BDF8E400401C80B292
:10D2D0003990BDF8E4000628DCDB9DF8B400DDE9F8
:10D2E0002E1240F2A11310FB03F03A4B03EBC003E4
:10D2F00003F562739DF8A00000EB400404EB0010FE
:10D3000003EBC00040F8221F426000222E922F92B1
:10D31000002139911EE0DDE92E10000240EA116281
:10D320000902CDE92E129DF8B41001EB4100C0EBCB
:10D33000C1102A4901EBC001BDF8E4000930085CC6
:10D34000DDE92E341843CDE92E04BDF8E400401C7D
:10D3500080B23990BDF8E4000628DCDB9DF8B4000B
:10D36000DDE92E2140F2A11310FB03F0194B03EB72
:10D37000C00000F562709DF8A03003EB430404EB9D
:10D38000031300EBC30022308260C1609DF8B4102B
:10D3900040F2A11011FB00F00E4901EBC00101F5B4
:10D3A00062719DF8A00000EB400202EB001011F842
:10D3B00030109DF8B40040F2A11210FB02F0054AB3
:10D3C00002EBC000407981427ED19DF8B4009DF807
:10D3D000A01005E05845002098400020F887002064
:10D3E00001EB0010C217CDE92E02FE4890F8E007CD
:10D3F00008B39DF8B41001EB410000EB0110FA49AD
:10D4000001EB001030309DF8A01000EB0110807A85
:10D41000022810D09DF8B41001EB410000EB011080
:10D42000F14901EB001030309DF8A01000EB011025
:10D43000C07A00287DDD00229DF8B40000EB400199
:10D4400001EB0010E84901EB001030309DF8A0100E
:10D4500000EB0110C272E548D0F80C020521B0FBC8
:10D46000F1F201FB120000EB4001E0482C3000EB30
:10D4700041100D3009909DF8B40040F2A11110FB4D
:10D4800001F0DB4901EBC00000F562709DF8A010CF
:10D4900001EB410202EB011100EBC100223010222E
:10D4A000014608900998FAF7D0FED048D0F80C024F
:10D4B0000521B0FBF1F201FB120000EB4001CB486B
:10D4C0002C3000EB411200E0D8E29DF8B40040F2AD
:10D4D000A11110FB01F0C64901EBC00101F5627119
:10D4E0009DF8A00000EB400303EB001001EBC0002F
:10D4F00050F81A1F42F8011F40685060BB48D0F82E
:10D500000C020521B0FBF1F201FB120000EB40011F
:10D51000B6482C3000EB41129DF8B40000EB4001FE
:10D5200001EB0010B04901EB001130319DF8A00073
:10D5300000E094E101EB001000781070AB48D0F8E7
:10D540000C020521B0FBF1F201FB120000EB4001DF
:10D55000A6482C3000EB4111A248F538026841F88A
:10D560001D2F80888880A148D0F80C020521B0FBCF
:10D57000F1F201FB120000EB40019C482C3000EB63
:10D5800041129DF8B40040F2A11110FB01F098493E
:10D5900001EBC00101F562719DF8A00000EB4003B2
:10D5A00003EB001001EBC000406BC2F809008F488C
:10D5B000D0F80C020521B0FBF1F201FB120000EBE8
:10D5C00040018A482C3000EB41129DF8B40000EB7A
:10D5D000400101EB0010844901EB001130319DF84E
:10D5E000A00001EB00104068C2F8230000229DF863
:10D5F000B40000EB400101EB00107B4901EB00118E
:10D6000030319DF8A00001EB0010426000213991FB
:10D6100054E07648D0F80C020521B0FBF1F201FB92
:10D62000120000EB400171482C3000EB4111273112
:10D63000BDF8E4409DF8B40040F2A11210FB02F0E6
:10D640006B4A02EBC00202F562729DF8A00000EB8B
:10D65000400303EB001002EBC00090F8800040F2A2
:10D66000A11210FB02F0624A02EBC00202F56272E4
:10D670009DF8B40040F2A11310FB03F05C4B03EBE8
:10D68000C00303F562739DF8A00000EB400505EBB5
:10D69000001003EBC00090F8810000EB400303EBA7
:10D6A000001002EBC0024732BDF8E400001D105C20
:10D6B0000855BDF8E400401C81B23991BDF8E40082
:10D6C0000628A6DB0021399142E000239DF8B40032
:10D6D00040F2A11110FB01F0454901EBC00101F539
:10D6E00062719DF8A00000EB400202EB001001EB1C
:10D6F000C00090F8800040F2A11110FB01F03C49FD
:10D7000001EBC00101F562719DF8B40040F2A11275
:10D7100010FB02F0364A02EBC00202F562729DF87D
:10D72000A00000EB400404EB001002EBC00090F8F6
:10D73000810000EB400202EB001001EBC001473119
:10D74000BDF8E4000B54BDF8E400401C81B23991EF
:10D75000BDF8E4000A28B8DB2448D0F80C02052103
:10D76000B0FBF1F080B2014609900220FBF7B0FC5B
:10D7700000210620FCF79AFC1C48D0F80C021B493B
:10D78000498D884206D21948D0F80C02401C17492E
:10D79000C1F80C0200210520FCF788FC9DF8B410AC
:10D7A00001EB410000EB01100F4901EB001030309C
:10D7B0009DF8A01000EB0110801C0990007820F06B
:10D7C0000400001D099908700848D0F80C020521D2
:10D7D000B0FBF1F201FB120000EB400103482C30DA
:10D7E00008E00000BC32002098400020BC1200205D
:10D7F0005845002000EB4110D0F823202E9800EB74
:10D800004001FE4800EB4110C0F823200020399071
:10D8100020E0FB48D0F80C020521B0FBF1F201FB3F
:10D82000120000EB4001F6482C3000EB411027308D
:10D83000BDF8E410425C2E9800EB4001EF4800EB8D
:10D8400041112731BDF8E4000A54BDF8E400401C42
:10D8500081B23991BDF8E4000628DADB59E09DF881
:10D86000B40000EB400101EB0010E64901EB0010B1
:10D8700030309DF8A01000EB0110801C099000785A
:10D8800020F008000830099908709DF8B40000EBFA
:10D89000400101EB0010DB4901EB001030309DF836
:10D8A000A01000EB011042682E9800EB4001D34815
:10D8B00000EB4110C0F823200020399025E09DF8AE
:10D8C000B40040F2A11110FB01F0CF4901EBC001FF
:10D8D00001F562719DF8A00000EB400202EB001020
:10D8E00001EBC0014731BDF8E4000A5C2E9800EB63
:10D8F0004001C24800EB41112731BDF8E4000A5451
:10D90000BDF8E400401C81B23991BDF8E40006285E
:10D91000D5DB9DF8B40000EB400101EB0010B949E4
:10D9200001EB001030309DF8A01000EB0110801CBE
:10D930000990007820F02002099802709DF8B41038
:10D940000220FCF7B3FB9DF8B40040F2A11110FBDC
:10D9500001F0AD4901EBC00000F562709DF8A01028
:10D9600001EB410202EB011100EBC10022300990F2
:10D970002E9800EB4001A14800EB41100D30102221
:10D9800008900999FAF761FC9DF8B40040F2A111E2
:10D9900010FB01F09C4901EBC00101F562719DF89B
:10D9A000A00000EB400202EB001001EBC0012E983A
:10D9B00000EB4002914800EB421051F81A2F40F85A
:10D9C000012F496841609DF8B40000EB400101EB74
:10D9D00000108C4901EB001130319DF8A00001EBE3
:10D9E000001001782E9800EB4002844800EB4210B2
:10D9F00001702E9800EB4001804800EB41118348F4
:10DA0000026841F81D2F808888809DF8B40040F29C
:10DA1000A11110FB01F07C4901EBC00101F562711D
:10DA20009DF8A00000EB400202EB001001EBC000EB
:10DA3000416B2E9800EB4002704800EB4210C0F89A
:10DA400009102E9881B208200991FCF72FFB0022C3
:10DA50009DF8B40040F2A11110FB01F06A4901EBFE
:10DA6000C00000F562709DF8A01001EB410303EBCC
:10DA7000011100EBC10080F8462053E09DF8B4008E
:10DA800000EB400101EB00105E4901EB001030306B
:10DA90009DF8A01000EB0110801C0990007820F088
:10DAA0000400001D099908709DF8B40000EB4001C6
:10DAB00001EB0010534901EB001030309DF8A0102D
:10DAC00000EB0110801C0990007820F0800080306D
:10DAD0000999087001209DF8B41040F2A11211FBC1
:10DAE00002F1494A02EBC10108719DF8B40040F20D
:10DAF000A11110FB01F0114601EBC00042799DF825
:10DB0000B40040F2A11110FB01F03F4901EBC0004D
:10DB100000F562709DF8A01001EB410303EB0111C9
:10DB200000F83120D5229DF8B40040F2A11110FB7D
:10DB300001F0354901EBC00000F562709DF8A010BE
:10DB400001EB410303EB011100EBC10042713FE225
:10DB5000D5229DF8B40040F2A11110FB01F02A4932
:10DB600001EBC00000F562709DF8A01001EB4103CD
:10DB700003EB011100EBC100427129E2D5229DF8AF
:10DB8000B40040F2A11110FB01F01F4901EBC000ED
:10DB900000F562709DF8A01001EB410303EB011149
:10DBA00000EBC100427113E201211848F53080F802
:10DBB00004179DF8B41040F2A11011FB00F01249B7
:10DBC00001EBC00101F562719DF8A00000EB40027D
:10DBD00002EB001011F830109DF8B40040F2A112D1
:10DBE00010FB02F0084A02EBC000407981423FDAA4
:10DBF00000219DF8B40040F2A11209E0D8140020E1
:10DC0000BC1200209840002058450020C731002059
:10DC100010FB02F0FE4A02EBC000017101229DF8E8
:10DC2000B40040F2A11110FB01F0F94901EBC00171
:10DC300001F562719DF8A00000EB400303EB0010BA
:10DC400001F8302011229DF8B40040F2A11110FB20
:10DC500001F0EF4901EBC00000F562709DF8A010E3
:10DC600001EB410303EB011100EBC100427160E0E5
:10DC70009DF8B41040F2A11011FB00F0E44901EB53
:10DC8000C00000F562709DF8A01001EB410202EBAC
:10DC9000011100EBC1008078B22835D100219DF838
:10DCA000B40040F2A11210FB02F0D94A02EBC0000E
:10DCB0000171B2229DF8B40040F2A11110FB01F0F5
:10DCC000D34901EBC00101F562719DF8A00000EBA2
:10DCD000400303EB001001EBC000427100229DF8ED
:10DCE000B40040F2A11110FB01F0C94901EBC000E2
:10DCF00000F562709DF8A01001EB410303EB0111E8
:10DD000000EBC100827014E0D5229DF8B40040F20F
:10DD1000A11110FB01F0BE4901EBC00000F56270DB
:10DD20009DF8A01001EB410303EB011100EBC100D2
:10DD300042714DE10021B74880F80417D5229DF8C3
:10DD4000B40040F2A11110FB01F0B14901EBC00099
:10DD500000F562709DF8A01001EB410303EB011187
:10DD600000EBC100427133E101229DF8B40040F2A2
:10DD7000A11110FB01F0A64901EBC00101F5627190
:10DD80009DF8A00000EB400303EB001001EBC00086
:10DD900080F882200021399129E09DF8B41001EB30
:10DDA0004100C0EBC1109C4901EBC001BDF8E4008B
:10DDB000C01C0A5C9DF8B40040F2A11110FB01F0F8
:10DDC000934901EBC00101F562719DF8A00000EBE1
:10DDD000400303EB001001EBC00000F18301BDF82C
:10DDE000E4000A54BDF8E400401C81B23991BDF84A
:10DDF000E4000A28D1DBEBE09DF8B41001EB410010
:10DE0000C0EBC110844901EBC000C07801049DF84B
:10DE1000B40000EB4002C2EBC0107F4A02EBC0002E
:10DE2000007941EA00209DF8B41001EB4102C2EBF9
:10DE3000C111794A02EBC10149790843B0F5E13FCC
:10DE40006ED19DF8B41001EB410000EB0110734955
:10DE500001EB001030309DF8A01000EB0110801C89
:10DE60000990007820F004020998027000229DF8C1
:10DE7000B40040F2A11110FB01F0654901EBC000B4
:10DE800000F562709DF8A01001EB410303EB011156
:10DE900000EBC100A0F88E2013229DF8B40040F2E0
:10DEA000A11110FB01F05A4901EBC00000F56270AE
:10DEB0009DF8A01001EB410303EB011100EBC10041
:10DEC00042719DF8B41001EB410000EB0110534981
:10DED00001EB0010407903464FF480524FF4E131DA
:10DEE00009909DF8B40019F035FB9DF8B41040F28C
:10DEF000A11011FB00F0464901EBC00101F5627170
:10DF00009DF8A00000EB400202EB001001EBC00006
:10DF100090300990007820F00800083009990870C6
:10DF200056E09DF8B41001EB4100C0EBC1103A4936
:10DF300001EBC00001799DF8B40000EB4002C2EB98
:10DF4000C010354A02EBC000C07841EA00229DF8BB
:10DF5000B40040F2A11110FB01F02D4901EBC0010A
:10DF600001F562719DF8A00000EB400303EB001087
:10DF700001EBC000A0F88E209DF8B40040F2A11182
:10DF800010FB01F0224901EBC00101F562719DF81F
:10DF9000A00000EB400202EB001001EBC000B0F863
:10DFA0008E109DF8B40000EB400202EB00101B4AFB
:10DFB00002EB0010408B814209DB0621A2F50472BE
:10DFC0009DF8B40002EB00129DF8A000115400BFB0
:10DFD00000BF10F0DFB89DF8B40000EB4001C1EBCA
:10DFE000C0100D4911F83000042801D125900BE034
:10DFF0009DF8B40000EB4001C1EBC010064911F8D8
:10E000003000152800D125909DF8B40008E00000EC
:10E0100058450020BC320020F8870020984000209E
:10E0200000EB4001C1EBC010F84901EBC0004178A2
:10E030009DF8B40000EB4002C2EBC010F34A12F8A6
:10E04000300041EA002041F23001884202D1A6208E
:10E0500025903DE09DF8B40000EB4001C1EBC010FD
:10E06000EA4901EBC00041789DF8B40000EB4002A2
:10E07000C2EBC010E54A12F8300041EA002041F23C
:10E080003101884202D1A720259021E09DF8B400FB
:10E0900000EB4001C1EBC010DC4911F83000022850
:10E0A00016D19DF8B40000EB4001C1EBC010D74978
:10E0B00001EBC00001799DF8B40000EB4002C2EB17
:10E0C000C010D24A02EBC000C07841EA002125917D
:10E0D0009DF8B41040F2A11011FB00F0CC4901EB07
:10E0E000C000817828910021CA4A9DF8B40002EB53
:10E0F00000129DF8A0001154C74890F8280001288C
:10E1000015D19DF8B40000EB400101EB0010C349AC
:10E1100001EB001030309DF8A01000EB0110801CC6
:10E120000990007820F08000803009990870BDF8CF
:10E13000941043F23002881A91427CD009DC042901
:10E140007AD0152979D0A62910D0A72942F0EC82DF
:10E1500066E1B0F5C06F71D0A0F2016000286ED00A
:10E1600001286DD00428F1D101F074BE00219DF882
:10E17000B40040F2A11210FB02F0A54A02EBC0006D
:10E1800001719DF8B40040F2A11110FB01F011469D
:10E1900001EBC00000F562709DF8A01001EB410298
:10E1A00002EB011110F83100052829DC06229DF848
:10E1B000B40040F2A11110FB01F0954901EBC00140
:10E1C00001F562719DF8A00000EB400303EB001025
:10E1D00001F83020A8229DF8B40040F2A11110FBF4
:10E1E00001F08B4901EBC00000F562709DF8A010B2
:10E1F00001EB410303EB011100EBC100427103E1AC
:10E200009DF8B40040F2A11110FB01F0804901EB30
:10E21000C00000F562709DF8A01001EB410202EB16
:10E22000011110F831000A2830DC0B229DF8B400EF
:10E2300040F2A11105E0B9E137E2F3E3F3E3F3E3E0
:10E24000F3E310FB01F0724901EBC00101F56271CB
:10E250009DF8A00000EB400303EB001001F8302014
:10E26000A9229DF8B40040F2A11110FB01F0684909
:10E2700001EBC00000F562709DF8A01001EB4103B6
:10E2800003EB011100EBC1004271BDE09DF8B40049
:10E2900040F2A11110FB01F05D4901EBC00000F557
:10E2A00062709DF8A01001EB410202EB011110F821
:10E2B00031000F2829DC10229DF8B40040F2A11192
:10E2C00010FB01F0524901EBC00101F562719DF8AC
:10E2D000A00000EB400303EB001001F83020A22265
:10E2E0009DF8B40040F2A11110FB01F0484901EB88
:10E2F000C00000F562709DF8A01001EB410303EB34
:10E30000011100EBC10042717EE09DF8B40040F2C3
:10E31000A11110FB01F03E4901EBC00000F5627055
:10E320009DF8A01001EB410202EB011100EBC100CE
:10E330004079A52815D19DF8B40000EB400101EB10
:10E340000010364901EB001030309DF8A01000EBB2
:10E350000110801C0990007820F00400001D09992C
:10E3600008709DF8B40040F2A11110FB01F028499B
:10E3700001EBC00000F562709DF8A01001EB4102B6
:10E3800002EB011100EBC1008078A1283CD09DF880
:10E39000B40040F2A11110FB01F01D4901EBC001D6
:10E3A00001F562719DF8A00000EB400202EB001045
:10E3B00001EBC00082789DF8B40040F2A11110FB7F
:10E3C00001F0134901EBC00101F562719DF8A00055
:10E3D00000EB400303EB001001EBC0004271A122EF
:10E3E0009DF8B40040F2A11110FB01F0084901EBC7
:10E3F000C00000F562709DF8A01001EB410303EB33
:10E40000011100EBC100827002F08EB9F887002084
:10E4100058450020883E0020BC1200209840002073
:10E4200000219DF8B40040F2A11210FB02F0FE4A58
:10E4300002EBC00001719DF8B41040F2A11011FB75
:10E4400000F0114601EBC00000F562709DF8A010CD
:10E4500001EB410202EB011110F8310008281FDC2A
:10E4600000219DF8B40040F2A11210FB02F0EE4A28
:10E4700002EBC000017108229DF8B40040F2A11126
:10E4800010FB01F0E84901EBC00000F562709DF857
:10E49000A01001EB410303EB011100F8312028E04B
:10E4A0009DF8B41040F2A11011FB00F0DE4901EB21
:10E4B000C00000F562709DF8A01001EB410202EB74
:10E4C000011110F831000B2813DC0C229DF8B40068
:10E4D00040F2A11110FB01F0D34901EBC00000F59F
:10E4E00062709DF8A01001EB410303EB011100F8ED
:10E4F00031209DF8B41040F2A11011FB00F0CA4980
:10E5000001EBC00000F562709DF8A01001EB410224
:10E5100002EB011100EBC1004079A42830D19DF835
:10E52000B41001EB410000EB0110C04901EB0010F9
:10E5300030309DF8A01000EB0110801C099000788D
:10E5400020F0200020300999087000229DF8B400C6
:10E5500040F2A11110FB01F0B34901EBC00000F53E
:10E5600062709DF8A01001EB410303EB011100EB79
:10E57000C10080F845209DF8B4100220FBF796FDFD
:10E58000A1229DF8B40040F2A11110FB01F0A649B0
:10E5900001EBC00000F562709DF8A01001EB410393
:10E5A00003EB011100EBC10042712DE7002139910D
:10E5B00015E09DF8B41001EB4100C0EBC1109C497F
:10E5C00001EBC001BDF8E400C01C0A5C16A9BDF84F
:10E5D000E4000A54BDF8E400401C81B23991BDF852
:10E5E000E4000628E5DB062116A828F07DFC0021C2
:10E5F000CDE93001DDE93021100A40EA0164A218BA
:10E6000041EB2120CDE908204FF480724FF0000348
:10E61000DDE90801F9F7D6FD9DF8B40040F2A1113B
:10E6200010FB01F0804901EBC00000F562709DF81D
:10E63000A01001EB410303EB011100EBC1000271DB
:10E6400000209DF8B41040F2A11211FB02F1764AAD
:10E6500002EBC101087104229DF8B40040F2A1113F
:10E6600010FB01F0704901EBC00000F562709DF8ED
:10E67000A01001EB410303EB011100F83120A722A8
:10E680009DF8B40040F2A11110FB01F0664901EBC6
:10E69000C00000F562709DF8A01001EB410303EB90
:10E6A000011100EBC1004271AEE69DF8B41040F2DA
:10E6B000A11011FB00F05C4901EBC00000F5627095
:10E6C0009DF8A01001EB410202EB011110F831009E
:10E6D000042878DA00219DF8B40040F2A11210FB62
:10E6E00002F0514A02EBC0000171A1229DF8B40072
:10E6F00040F2A11110FB01F04B4901EBC00101F503
:10E7000062719DF8A00000EB400303EB001001EBE9
:10E71000C00042719DF8B41040F2A11011FB00F04E
:10E72000414901EBC00101F562719DF8A00000EBC9
:10E73000400202EB001001EBC00109910878401C77
:10E74000C1B2099801709DF8B41040F2A11011FBFC
:10E7500000F0354901EBC00000F562709DF8A01093
:10E7600001EB410202EB011110F83100042828D11D
:10E770000A229DF8B40040F2A11110FB01F02A49D1
:10E7800001EBC00101F562719DF8A00000EB4003B0
:10E7900003EB001001F83020A3229DF8B40040F2F2
:10E7A000A11110FB01F0204901EBC00000F56270DF
:10E7B0009DF8A01001EB410303EB011100EBC10038
:10E7C0004271E4E2FFE79DF8B41040F2A11011FBA2
:10E7D00000F0154901EBC00000F562709DF8A01033
:10E7E00001EB410202EB011110F8310004283BD18A
:10E7F00000219DF8B40040F2A11210FB02F00A4A79
:10E8000002EBC000017105229DF8B40040F2A11195
:10E8100010FB01F0044901EBC00101F562719DF8A4
:10E82000A00000EB400305E0584500209840002080
:10E83000F887002003EB001001F83020A3229DF898
:10E84000B40040F2A11110FB01F0FE4901EBC00041
:10E8500000F562709DF8A01001EB410303EB01117C
:10E8600000EBC100427192E29DF8B41040F2A11099
:10E8700011FB00F0F34901EBC00000F562709DF858
:10E88000A01001EB410202EB011110F83100082841
:10E8900034DC00219DF8B40040F2A11210FB02F01C
:10E8A000E84A02EBC000017109229DF8B40040F271
:10E8B000A11110FB01F0E34901EBC00101F5627108
:10E8C0009DF8A00000EB400303EB001001F830209E
:10E8D000A7229DF8B40040F2A11110FB01F0D94924
:10E8E00001EBC00000F562709DF8A01001EB410340
:10E8F00003EB011100EBC100427148E29DF8B41036
:10E9000040F2A11011FB00F0CE4901EBC00000F570
:10E9100062709DF8A01001EB410202EB011110F8AA
:10E920003100092834DC00219DF8B40040F2A11226
:10E9300010FB02F0C34A02EBC00001710A229DF8ED
:10E94000B40040F2A11110FB01F0BE4901EBC0017F
:10E9500001F562719DF8A00000EB400303EB00108D
:10E9600001F83020A3229DF8B40040F2A11110FB61
:10E9700001F0B44901EBC00101F562719DF8A000FE
:10E9800000EB400303EB001001EBC0004271FEE11D
:10E990009DF8B41040F2A11011FB00F0A94901EB61
:10E9A000C00000F562709DF8A01001EB410202EB7F
:10E9B000011110F831000D2838DC00219DF8B40059
:10E9C00040F2A11210FB02F09E4A02EBC00001715E
:10E9D0000E229DF8B40040F2A11110FB01F09949FC
:10E9E00001EBC00101F562719DF8A00000EB40034E
:10E9F00003EB001001F83020A1229DF8B40040F292
:10EA0000A11110FB01F08F4901EBC00000F562700D
:10EA10009DF8A01001EB410303EB011100EBC100D5
:10EA20004271B4E1B4E1E8E13DE21BE29DF8B410CB
:10EA300040F2A11011FB00F0824901EBC00000F58B
:10EA400062709DF8A01001EB410202EB011110F879
:10EA500031000E2834DC00219DF8B40040F2A112F0
:10EA600010FB02F0774A02EBC00001710F229DF803
:10EA7000B40040F2A11110FB01F0724901EBC0019A
:10EA800001F562719DF8A00000EB400303EB00105C
:10EA900001F83020A3229DF8B40040F2A11110FB30
:10EAA00001F0684901EBC00000F562709DF8A0100C
:10EAB00001EB410303EB011100EBC100427166E180
:10EAC0009DF8B41040F2A11011FB00F05D4901EB7C
:10EAD000C00000F562709DF8A01001EB410202EB4E
:10EAE000011110F8310010287DDC11229DF8B400CE
:10EAF00040F2A11110FB01F0524901EBC00101F5F8
:10EB000062719DF8A00000EB400303EB001001F8D8
:10EB10003020A1229DF8B40040F2A11110FB01F0B9
:10EB2000484901EBC00101F562719DF8A00000EBBE
:10EB3000400303EB001001EBC00042719DF8B400EC
:10EB400040F2A11110FB01F03E4901EBC00101F5BB
:10EB500062719DF8A00000EB400303EB001001EB95
:10EB6000C00082709DF8B41001EB410000EB011071
:10EB7000354901EB001130319DF8A00001EB001088
:10EB8000801C0990007820F080008030099908707E
:10EB90009DF8B41001EB410000EB01102A4901EB94
:10EBA000001030309DF8A01000EB0110801C09907F
:10EBB000007820F00400001D099908709DF8B41039
:10EBC00001EB410000EB01101F4901EB0010303058
:10EBD0009DF8A01000EB01108078C0F3401080B3C6
:10EBE0009DF8B41000E046E001EB410000EB01109D
:10EBF000154901EB001030309DF8A01000EB01101A
:10EC0000801C0990007820F02002099802709DF87D
:10EC1000B41001EB410000EB01100B4901EB0010B7
:10EC200030309DF8A01000EB01108078C0F3400058
:10EC3000D8B99DF8B41001EB410000EB0110024976
:10EC400004E083E0584500209840002001EB0010CC
:10EC500030309DF8A01000EB0110801C0990007866
:10EC600020F008000830099908709DF8B4100220BF
:10EC7000FBF71CFA8BE09DF8B41040F2A11011FBD9
:10EC800000F0FE4901EBC00101F562719DF8A000A2
:10EC900000EB400202EB001011F830109DF8B400B8
:10ECA00040F2A11210FB02F0F44A02EBC0004079DE
:10ECB00081426CD19DF8B41040F2A11011FB00F01C
:10ECC000114601EBC00000F562709DF8A01001EB49
:10ECD000410202EB011100EBC1008078A12836D07F
:10ECE000A3229DF8B40040F2A11110FB01F0E3490A
:10ECF00001EBC00101F562719DF8A00000EB40033B
:10ED000003EB001001EBC00042719DF8B41040F21B
:10ED1000A11011FB00F0D94901EBC00000F56270B1
:10ED20009DF8A01001EB410202EB011100EBC100C4
:10ED30008078A2282BD000209DF8B41040F2A112B8
:10ED400011FB02F1CD4A02EBC10108711FE0A122C3
:10ED50009DF8B40040F2A11110FB01F0C74901EB8E
:10ED6000C00101F562719DF8A00000EB400303EBC8
:10ED7000001001EBC000427101219DF8B40040F287
:10ED8000A11210FB02F0BD4A02EBC00001710CE4BD
:10ED9000A1229DF8B40040F2A11110FB01F0B74987
:10EDA00001EBC00101F562719DF8A00000EB40038A
:10EDB00003EB001001EBC00082709DF8B40040F23C
:10EDC000A11110FB01F0AD4901EBC00101F5627129
:10EDD0009DF8A00000EB400303EB001001EBC00026
:10EDE000427100219DF8B40040F2A11210FB02F024
:10EDF000A24A02EBC000017156E400219DF8B40064
:10EE000040F2A11210FB02F09C4A02EBC00001711B
:10EE100009229DF8B40040F2A11110FB01F09749BE
:10EE200001EBC00101F562719DF8A00000EB400309
:10EE300003EB001001F83020A7229DF8B40040F247
:10EE4000A11110FB01F08D4901EBC00000F56270CB
:10EE50009DF8A01001EB410303EB011100EBC10091
:10EE6000427121E400219DF8B40040F2A11210FB90
:10EE700002F0824A02EBC0000171A7229DF8B400A3
:10EE800040F2A11110FB01F07C4901EBC00000F53C
:10EE900062709DF8A01001EB410303EB011100EB40
:10EEA000C100427173E700219DF8B40040F2A11245
:10EEB00010FB02F0714A02EBC0000171A7229DF81D
:10EEC000B40040F2A11110FB01F06C4901EBC0014C
:10EED00001F562719DF8A00000EB400303EB001008
:10EEE00001EBC00042719DF8B41001EB4100C0EB92
:10EEF000C110634901EBC000407930287ED19DF8F4
:10EF0000B41040F2A11011FB00F05C4901EBC0010C
:10EF100001F562719DF8A00000EB400202EB0010C9
:10EF200011F830109DF8B40040F2A11210FB02F06D
:10EF3000524A02EBC000407981425FD19DF8B40093
:10EF400040F2A11110FB01F0114601EBC00000F5E9
:10EF500062709DF8A01001EB410202EB011100EB81
:10EF6000C100C078312830D19DF8B40000EB4001D9
:10EF700001EB0010434901EB001030309DF8A01068
:10EF800000EB0110801C0990007820F02002099805
:10EF9000027000229DF8B40040F2A11110FB01F0B4
:10EFA000364901EBC00000F562709DF8A01001EB3E
:10EFB000410303EB011100EBC10080F845209DF8EF
:10EFC000B4100220FBF772F857E09DF8B40040F24D
:10EFD000A11110FB01F0294901EBC00000F562709E
:10EFE0009DF8A01001EB410202EB011100EBC10002
:10EFF000C078332841D19DF8B40000E06FE000EB09
:10F00000400101EB00101F4901EB001030309DF86A
:10F01000A01000EB0110801C0990007820F0200265
:10F020000998027001229DF8B40040F2A11110FB72
:10F0300001F0124901EBC00000F562709DF8A010CC
:10F0400001EB410303EB011100EBC10080F8462006
:10F05000A9229DF8B40040F2A11110FB01F007496C
:10F0600001EBC00000F562709DF8A01001EB4103B8
:10F0700003EB011100EBC100827005E05845002050
:10F08000F8870020984000209DF8B40000EB400174
:10F0900001EB0010FE4901EB001030309DF8A0108C
:10F0A00000EB0110801C0990007820F00102099803
:10F0B00002709DF8B40000EB400101EB0010F44930
:10F0C00001EB001030309DF8A01000EB0110801C07
:10F0D0000990007820F0020209980270D6E39DF8AA
:10F0E000B40000EB4001C1EBC010EA4901EBC000E5
:10F0F000407931287ED19DF8B41040F2A11011FB67
:10F1000000F0E54901EBC00101F562719DF8A00036
:10F1100000EB400202EB001011F830109DF8B40033
:10F1200040F2A11210FB02F0DB4A02EBC000407972
:10F1300081425FD19DF8B41040F2A11011FB00F0A4
:10F14000114601EBC00000F562709DF8A01001EBC4
:10F15000410202EB011100EBC10090F8460058BBE0
:10F1600001229DF8B40040F2A11110FB01F0CA4940
:10F1700001EBC00101F562719DF8A00000EB4003B6
:10F1800003EB001001EBC00080F845209DF8B4109F
:10F1900001EB410000EB0110BD4901EB00113031E2
:10F1A0009DF8A00001EB0010801C0990007820F071
:10F1B0000100401C099908709DF8B41001EB410052
:10F1C00000EB0110B24901EB001030309DF8A010A7
:10F1D00000EB0110801C0990007820F002020998D1
:10F1E0000270AE4890F8E00790B19DF8B41001EBC2
:10F1F000410000E005E200EB0110A54901EB001021
:10F2000030309DF8A01000EB0110807A022877D1F1
:10F21000A34890F829000128F9D1A148D0F80C02A0
:10F220009F49498D88426BD29DF8B40040F2A111EC
:10F2300010FB01F0984901EBC00000F562709DF8E9
:10F24000A01001EB410202EB011100EBC10090F8AC
:10F250004500012853D19DF8B41040F2A11011FBD4
:10F2600000F08D4901EBC00000F562709DF8A01020
:10F2700001EB410202EB011100EBC10090F87F00AD
:10F28000E8BB01229DF8B40000EB400101EB001047
:10F290007F4901EB001130319DF8A00001EB001017
:10F2A000C27200229DF8B40000EB400101EB001097
:10F2B000774901EB001130319DF8A00001EB0010FF
:10F2C00042604FF010429DF8B40040F2A11110FBD3
:10F2D00001F0714901EBC00101F562719DF8A000D8
:10F2E00000EB400303EB001001EBC00082609DF8CF
:10F2F000B41001EB410000EB0110654901E071E041
:10F300006FE001EB001130319DF8A00001EB00101F
:10F3100001789DF8B40040F2A11210FB02F05E4AA1
:10F3200002EBC00041709DF8B41040F2A11011FB37
:10F3300000F0114601EBC00101F562719DF8A000DB
:10F3400000EB400202EB001011F830109DF8B40001
:10F3500040F2A11210FB02F04F4A02EBC0004079CC
:10F3600081423ED100229DF8B40040F2A11110FB71
:10F3700001F0494901EBC00101F562719DF8A0005F
:10F3800000EB400303EB001001EBC000C271A422AC
:10F390009DF8B40040F2A11110FB01F03E4901EBD1
:10F3A000C00101F562719DF8A00000EB400303EB82
:10F3B000001001EBC0008270A3229DF8B40040F25F
:10F3C000A11110FB01F0344901EBC00101F562719C
:10F3D0009DF8A00000EB400303EB001001EBC00020
:10F3E000427153E29DF8B41040F2A11011FB00F0FD
:10F3F000294901EBC00000F562709DF8A01001EBF7
:10F40000410202EB011100EBC10090F84500012818
:10F410007DD19DF8B41040F2A11011FB00F01E49FF
:10F4200001EBC00101F562719DF8A00000EB400204
:10F4300002EB001001EBC00090F8801040F2A11028
:10F4400011FB00F0144901EBC00101F562719DF858
:10F45000B40040F2A11210FB02F00F4A02EBC00010
:10F4600000F562709DF8A02002EB420303EB02124C
:10F4700000EBC20090F8810000EB400202EB0010AC
:10F4800001EBC00090F87E00032840D1022209E081
:10F4900098400020F887002058450020BC3200200A
:10F4A000BC1200209DF8B40000EB400101EB0010FD
:10F4B000F94901EB001130319DF8A00001EB00107B
:10F4C000C2724FF010429DF8B40040F2A11110FB3F
:10F4D00001F0F24901EBC00101F562719DF8A00055
:10F4E00000EB400303EB001001EBC00082609DF8CD
:10F4F000B41001EB410000EB0110E74901EB0011F2
:10F5000030319DF8A00001EB0010017800E0B0E17F
:10F510009DF8B40040F2A11210FB02F0DF4A02EBAA
:10F52000C00041709DF8B41040F2A11011FB00F032
:10F53000114601EBC00101F562719DF8A00000EBDE
:10F54000400202EB001011F830109DF8B40040F2B8
:10F55000A11210FB02F0D14A02EBC00040798142B7
:10F560003ED100229DF8B40040F2A11110FB01F041
:10F57000CA4901EBC00101F562719DF8A00000EBE2
:10F58000400303EB001001EBC000C271A4229DF800
:10F59000B40040F2A11110FB01F0C04901EBC00121
:10F5A00001F562719DF8A00000EB400303EB001031
:10F5B00001EBC0008270A3229DF8B40040F2A111BB
:10F5C00010FB01F0B54901EBC00000F562709DF839
:10F5D000A01001EB410303EB011100EBC1004271EC
:10F5E00000229DF8B40000EB400101EB0010AA4995
:10F5F00001EB001030309DF8A01000EB01104260CC
:10F6000044E19DF8B41001EB4100C0EBC110A449E6
:10F6100001EBC000407933287ED19DF8B41001EB96
:10F62000410000EB01109C4901EB001030309DF8C7
:10F63000A01000EB0110801C0990007820F0010060
:10F64000401C099908709DF8B41001EB410000EBD3
:10F650000110914901EB001030309DF8A01000EB33
:10F660000110801C0990007820F020020998027097
:10F670009DF8B41001EB410000EB0110864901EB4D
:10F68000001030309DF8A01000EB0110801C099094
:10F69000007820F00200801C099908709DF8B410D1
:10F6A00040F2A11011FB00F07C4901EBC00042794F
:10F6B0009DF8B40040F2A11110FB01F0774901EB75
:10F6C000C00000F562709DF8A01001EB410303EB50
:10F6D000011100F831209DF8B41001EB410000EB5E
:10F6E00001106D4901EB001030309DF8A01000EBC7
:10F6F0000110801C0990007820F08000803009996A
:10F7000008709DF8B41001EB410000EB0110624954
:10F7100001EB0010303000E022E09DF8A01000EB7B
:10F7200001108078C0F3400020B99DF8B410022089
:10F73000FAF7BCFCA2229DF8B40040F2A11110FB24
:10F7400001F0564901EBC00000F562709DF8A01071
:10F7500001EB410303EB011100EBC100827095E066
:10F760009DF8B41001EB4100C0EBC1104C4901EB16
:10F77000C000407934287CD19DF8B41001EB4100E1
:10F7800000EB0110444901EB001030309DF8A0104F
:10F7900000EB0110801C0990007820F020020998ED
:10F7A00002709DF8B41001EB410000EB01103A49E2
:10F7B00001EB001030309DF8A01000EB0110801C10
:10F7C0000990007820F002020998027001229DF849
:10F7D000B40040F2A11110FB01F0304901EBC00070
:10F7E00000F562709DF8A01001EB410303EB0111DD
:10F7F00000EBC10080F84620A9229DF8B40040F239
:10F80000A11110FB01F0254901EBC00000F5627069
:10F810009DF8A01001EB410303EB011100EBC100C7
:10F8200082709DF8B41040F2A11011FB00F01B494A
:10F8300001EBC00042799DF8B40040F2A11110FB29
:10F8400001F0164901EBC00000F562709DF8A010B0
:10F8500001EB410303EB011100F831209DF8B410D6
:10F8600001EB410000EB01100B4901EB00103030BF
:10F8700000E00BE09DF8A01000EB0110801C099047
:10F88000007820F0800080300999087000202E90C8
:10F890002F900021399128E0984000205845002001
:10F8A000F8870020DDE92E10000140EA11720901FD
:10F8B000CDE92E129DF8B41001EB4100C0EBC11050
:10F8C000FE4901EBC001BDF8E400801D085C303842
:10F8D000C117DDE92E34184341EA0402CDE92E02B6
:10F8E000BDF8E400401C80B23990BDF8E400062861
:10F8F000D8DB9DF8B4002E9940F2A11210FB02F063
:10F90000EF4A02EBC00202F562729DF8A00000EB24
:10F91000400303EB001002EBC000C0F81A100022F5
:10F920002E922F920021399122E0DDE92E10000164
:10F9300040EA11720901CDE92E129DF8B41001EBD5
:10F940004100C0EBC110DD4901EBC001BDF8E4008E
:10F950000D30085C3038C117DDE92E34184341EA18
:10F960000402CDE92E02BDF8E400401C80B23990BB
:10F97000BDF8E4000428D8DB9DF8B4002E9940F2CD
:10F98000A11210FB02F0CE4A02EBC00202F5627235
:10F990009DF8A00000EB400303EB001002EBC00059
:10F9A000416300222E922F920021399122E0DDE95D
:10F9B0002E10000140EA11720901CDE92E129DF8C6
:10F9C000B41001EB4100C0EBC110BC4901EBC00118
:10F9D000BDF8E4001130085C3038C117DDE92E3481
:10F9E000184341EA0402CDE92E02BDF8E400401CB0
:10F9F00080B23990BDF8E4000628D8DB9DF8B40049
:10FA00002E9940F2A11210FB02F0AD4A02EBC002A7
:10FA100002F562729DF8A00000EB400303EB0010BA
:10FA200002EBC000C0F81E109DF8B41001EB4100BD
:10FA3000C0EBC110A14901EBC00042799DF8B400B0
:10FA400040F2A11110FB01F09D4901EBC00101F54D
:10FA500062719DF8A00000EB400303EB001001EB86
:10FA6000C000C2709DF8B41001EB410000EB011022
:10FA7000944901EB001130319DF8A00001EB00101A
:10FA800082789DF8B40040F2A11110FB01F08C497E
:10FA900001EBC00101F562719DF8A00000EB40038D
:10FAA00003EB001001EBC00002769DF8B41040F2A9
:10FAB000A11011FB00F0824901EBC00101F5627158
:10FAC0009DF8A00000EB400202EB001011F830108E
:10FAD0009DF8B40040F2A11210FB02F0784A02EB4C
:10FAE000C000407981427CDA9DF8B41040F2A11048
:10FAF00011FB00F0114601EBC00000F562709DF8AB
:10FB0000A01001EB410202EB011110F831000F28A7
:10FB100067DD00219DF8B40040F2A11210FB02F055
:10FB2000674A02EBC0000171A7229DF8B40040F2C1
:10FB3000A11110FB01F0624901EBC00101F56271F6
:10FB40009DF8A00000EB400303EB001001EBC000A8
:10FB5000427101219DF8B40040F2A11210FB02F0A5
:10FB6000574A02EBC00001719DF8B41040F2A11099
:10FB700011FB00F0114601EBC00042799DF8B40082
:10FB800040F2A11110FB01F04D4901EBC00101F55C
:10FB900062719DF8A00000EB400303EB001001F838
:10FBA0003020A1229DF8B40040F2A11110FB01F019
:10FBB000434901EBC00101F562719DF8A00000EB23
:10FBC000400303EB001001EBC00042719DF8B4103C
:10FBD00001EB410000EB01103A4901EB001130311B
:10FBE00000E071E09DF8A00001EB0010801C09907E
:10FBF000007820F080008030099908709DF8B410DA
:10FC000001EB410000EB01102E4901EB00103030F8
:10FC10009DF8A01000EB0110801C0990007820F0E6
:10FC20000400001D099908709DF8B41001EB410013
:10FC300000EB0110234901EB001030309DF8A010BB
:10FC400000EB01108078C0F3401088B99DF8B41023
:10FC500001EB410000EB01101A4901EB00103030BC
:10FC60009DF8A01000EB01108078C0F3400058B35D
:10FC70009DF8B41001EB410000EB0110114901EBBC
:10FC8000001030309DF8A01000EB0110801C09908E
:10FC9000007820F02002099802709DF8B41001EB62
:10FCA000410000EB0110074901EB001030309DF8D6
:10FCB000A01000EB0110801C099006E0F8870020DE
:10FCC0005845002098400020C3E0007820F0020250
:10FCD000099802709DF8B41001EB410000EB01108F
:10FCE000FE4901EB001030309DF8A01000EB011030
:10FCF000801C0990007820F00800083009990870ED
:10FD00009DF8B4009DF8A01001EB0010C217CDE9DA
:10FD10002E029DF8B41040F2A11011FB00F0F04942
:10FD200001EBC00000F562709DF8A01001EB4102EC
:10FD300002EB011100EBC100223009902E9800EB7C
:10FD40004001E84800EB41100D301022089009995D
:10FD5000F8F77BFA9DF8B41040F2A11011FB00F007
:10FD6000DF4901EBC00101F562719DF8A00000EBD5
:10FD7000400202EB001001EBC0012E9800EB4002A4
:10FD8000D84800EB421051F81A2F40F8012F49686B
:10FD900041609DF8B41001EB410000EB0110CF4928
:10FDA00001EB001130319DF8A00001EB001001784B
:10FDB0002E9800EB4002CB4800EB421001702E98C9
:10FDC00000EB4001C74800EB4111C748026841F809
:10FDD0001D2F808888809DF8B41040F2A11011FB7F
:10FDE00000F0BF4901EBC00101F562719DF8A00070
:10FDF00000EB400202EB001001EBC000416B2E98BB
:10FE000000EB4002B74800EB4210C0F809109DF823
:10FE1000B41001EB410000EB0110B04901EB0011FF
:10FE200030319DF8A00001EB001041682E9800EBE6
:10FE30004002AC4800EB4210C0F823102E9881B26B
:10FE400008200991FAF732F99DF8B4100220FAF768
:10FE50002DF9FCE300202E902F900021399122E013
:10FE6000DDE92E10000140EA11720901CDE92E12E0
:10FE70009DF8B41001EB4100C0EBC1109B4901EBB0
:10FE8000C001BDF8E4000B30085C3038C117DDE973
:10FE90002E3440EA03022143CDE92E21BDF8E400CF
:10FEA000401C81B23991BDF8E4000A28D8DB9DF8E6
:10FEB000B400DDE92E1240F2A11310FB03F0884BD1
:10FEC00003EBC00303F562739DF8A00000EB400450
:10FED00004EB001003EBC00040F8221F4260002238
:10FEE0002E922F920021399122E0DDE92E1000019F
:10FEF00040EA11720901CDE92E129DF8B41001EB10
:10FF00004100C0EBC110794901EBC001BDF8E4002C
:10FF10001530085C3038C117DDE92E34184341EA4A
:10FF20000402CDE92E02BDF8E400401C80B23990F5
:10FF3000BDF8E4000A28D8DB9DF8B400DDE92E21E5
:10FF400040F2A11310FB03F0654B03EBC00303F574
:10FF500062739DF8A00000EB400404EB001003EB7B
:10FF6000C00022308260C16000219DF8B40040F2E0
:10FF7000A11210FB02F05A4A02EBC00001719DF879
:10FF8000B41040F2A11011FB00F0114601EBC000CB
:10FF900000F562709DF8A01001EB410202EB011127
:10FFA00010F831000C2814DC0D229DF8B40040F24A
:10FFB000A11110FB01F04A4901EBC00000F562708D
:10FFC0009DF8A01001EB410303EB011100F8312073
:10FFD0007FE39DF8B40040F2A11110FB01F040490D
:10FFE00001EBC00101F562719DF8A00000EB400239
:10FFF00002EB001011F830109DF8B40040F2A1128D
:020000040801F1
:1000000010FB02F0364A02EBC00040798142DFD19A
:100010009DF8B4009DF8A01001EB0010C217CDE9C7
:100020002E023148F53090F8E00708B39DF8B4008F
:1000300000EB400101EB0010284901EB00103030CB
:100040009DF8A01000EB0110807A022810D09DF8D6
:10005000B40000EB400101EB0010204901EB00105F
:1000600030309DF8A01000EB0110C07A00287CDD34
:1000700000229DF8B40000EB400101EB001017498D
:1000800001EB001030309DF8A01000EB0110C2729F
:100090001748D0F80C020521B0FBF1F201FB120069
:1000A00000EB400112482C3000EB41100D3009905C
:1000B0009DF8B40040F2A11110FB01F0084901EBDA
:1000C000C00000F562709DF8A01001EB410202EB48
:1000D000011100EBC100223010220BE098400020FB
:1000E00058450020D8140020C7310020F887002090
:1000F000BC120020014608900998F8F7A6F8FE48BF
:10010000D0F80C020521B0FBF1F201FB120000EB6C
:100110004001F9482C3000EB41129DF8B40040F248
:10012000A11110FB01F0F54901EBC00101F562716D
:100130009DF8A00000EB400303EB001001EBC000B2
:1001400050F81A1F42F8011F40685060EA48D0F882
:100150000C020521B0FBF1F201FB120000EB4001A3
:10016000E5482C3000EB411200E094E19DF8B4002A
:1001700000EB400101EB0010E14901EB00113031CF
:100180009DF8A00001EB001000781070DA48D0F85C
:100190000C020521B0FBF1F201FB120000EB400163
:1001A000D5482C3000EB41129DF8B40040F2A1116B
:1001B00010FB01F0D14901EBC00101F562719DF81E
:1001C000A00000EB400303EB001001EBC000406B0C
:1001D000C2F80900C848D0F80C020521B0FBF1F2C2
:1001E00001FB120000EB4001C3482C3000EB411131
:1001F000C448026841F81D2F80888880BE48D0F826
:100200000C020521B0FBF1F201FB120000EB4001F2
:10021000B9482C3000EB41129DF8B40000EB4001CE
:1002200001EB0010B64901EB001130319DF8A00040
:1002300001EB00104068C2F8230000229DF8B400D2
:1002400000EB400101EB0010AD4901EB0011303132
:100250009DF8A00001EB001042600021399154E0AC
:10026000A548D0F80C020521B0FBF1F201FB120009
:1002700000EB4001A0482C3000EB41112731BDF8C4
:10028000E4409DF8B40040F2A11210FB02F09B4A3A
:1002900002EBC00202F562729DF8A00000EB400381
:1002A00003EB001002EBC00090F8800040F2A112B6
:1002B00010FB02F0914A02EBC00202F562729DF857
:1002C000B40040F2A11310FB03F08C4B03EBC0030E
:1002D00003F562739DF8A00000EB400505EB0010EC
:1002E00003EBC00090F8810000EB400303EB00102B
:1002F00002EBC0024732BDF8E400001D105C085557
:10030000BDF8E400401C81B23991BDF8E400062834
:10031000A6DB0021399142E000239DF8B40040F2B1
:10032000A11110FB01F0754901EBC00101F56271EB
:100330009DF8A00000EB400202EB001001EBC000B2
:1003400090F8800040F2A11110FB01F06B4901EB25
:10035000C00101F562719DF8B40040F2A11210FBDA
:1003600002F0664A02EBC00202F562729DF8A0003C
:1003700000EB400404EB001002EBC00090F8810099
:1003800000EB400202EB001001EBC0014731BDF869
:10039000E4000B54BDF8E400401C81B23991BDF873
:1003A000E4000A28B8DB5448D0F80C020521B0FB61
:1003B000F1F080B2014609900220F8F789FE002191
:1003C0000620F9F773FE4C48D0F80C024A49498DD3
:1003D000884206D24848D0F80C02401C4649C1F871
:1003E0000C0200210520F9F761FE9DF8B40000EB36
:1003F000400101EB0010424901EB001030309DF844
:10040000A01000EB0110801C0990007820F0080279
:10041000099802703848D0F80C020521B0FBF1F2BF
:1004200001FB120000EB400133482C3000EB41107F
:10043000D0F823202E9800EB4001334800EB411008
:10044000C0F823200020399020E02B48D0F80C027F
:100450000521B0FBF1F201FB120000EB4001264840
:100460002C3000EB41102730BDF8E410425C2E9890
:1004700000EB4001244800EB41112731BDF8E400B6
:100480000A54BDF8E400401C81B23991BDF8E40083
:100490000628DADB64E09DF8B40000EB400101EBD4
:1004A0000010174901EB001030309DF8A01000EB50
:1004B0000110801C0990007820F00800083009998C
:1004C00008709DF8B40000EB400101EB00100C49EE
:1004D00001EB001030309DF8A01000EB01104268D5
:1004E0002E9800EB4001084800EB4110C0F8232093
:1004F0000020399030E00000BC1200205845002058
:1005000098400020C7310020D81400209DF8B40086
:1005100040F2A11110FB01F0FE4901EBC00101F511
:1005200062719DF8A00000EB400202EB001001EBAD
:10053000C0014731BDF8E4000A5C2E9800EB400191
:10054000F54800EB41112731BDF8E4000A54BDF82D
:10055000E400401C81B23991BDF8E4000628D5DBE7
:1005600000229DF8B40040F2A11110FB01F0E9490E
:1005700001EBC00101F562719DF8A00000EB4003A2
:1005800003EB001001EBC00080F846209DF8B4108A
:100590000220F9F78BFD9DF8B40040F2A11110FB89
:1005A00001F0DC4901EBC00101F562719DF8A0008A
:1005B00000EB400202EB001001EBC000223009907A
:1005C0002E9800EB4001D44800EB41110D31102270
:1005D0000891DDE90801F7F738FE9DF8B40040F214
:1005E000A11110FB01F0CB4901EBC00101F56271D3
:1005F0009DF8A00000EB400202EB001001EBC001EF
:100600002E9800EB4002C44800EB421051F81A2F1C
:1006100040F8012F496841609DF8B40000EB4001AB
:1006200001EB0010BD4901EB001130319DF8A00035
:1006300001EB001001782E9800EB4002B64800EB69
:10064000421001702E9800EB4001B34800E06BE0CF
:1006500000EB4111B248026841F81D2F8088888064
:100660009DF8B40040F2A11110FB01F0A94901EB83
:10067000C00101F562719DF8A00000EB400202EBA1
:10068000001001EBC000416B2E9800EB4002A24825
:1006900000EB4210C0F809109DF8B40000EB4001D7
:1006A00001EB00109D4901EB001130319DF8A000D5
:1006B00001EB001041682E9800EB4002964800EBD9
:1006C0004210C0F823102E9881B208200991F9F742
:1006D000EDFCA7229DF8B40040F2A11110FB01F03F
:1006E0008C4901EBC00101F562719DF8A00000EB9F
:1006F000400303EB001001EBC0004271A2229DF801
:10070000B40040F2A11110FB01F0824901EBC000DE
:1007100000F562709DF8A01001EB410303EB01119D
:1007200000EBC100827000BF00BF0DF033BD9DF82B
:10073000B40000EB4001C1EBC0107A4911F8300061
:10074000042802D1042125910CE09DF8B41001EB9E
:100750004100C0EBC110734911F83000152801D1D8
:10076000152125919DF8B41001EB4100C0EBC1109B
:100770006C4901EBC00041789DF8B40000EB4002E9
:10078000C2EBC010674A12F8300041EA002041F283
:100790003001884202D1A62125913DE09DF8B41098
:1007A00001EB4100C0EBC1105E4901EBC000417894
:1007B0009DF8B40000EB4002C2EBC010594A12F899
:1007C000300041EA002041F23101884202D1A721E4
:1007D000259121E09DF8B41001EB4100C0EBC11060
:1007E000504911F83000022816D19DF8B41001EBE1
:1007F0004100C0EBC1104B4901EBC00001799DF8ED
:10080000B40000EB4002C2EBC010464A02EBC0004D
:10081000C07841EA002125919DF8B41040F2A11062
:1008200011FB00F03B4901EBC000817828910021C9
:100830003D4A9DF8B40002EB00129DF8A00011544F
:100840003A4890F82800012815D19DF8B41001EB22
:10085000410000EB0110314901EB001030309DF8F0
:10086000A01000EB0110801C0990007820F080009F
:10087000803009990870BDF89400A7287ED007DC65
:1008800004287CD015287BD0A62841F06D8762E033
:10089000A0F55850303820B1112872D01228F4D168
:1008A000FEE39DF8B41040F2A11011FB00F01949CD
:1008B00001EBC00000F562709DF8A01001EB410251
:1008C00002EB011110F8310090BB00219DF8B4003B
:1008D00040F2A11210FB02F00E4A02EBC0000171BF
:1008E00001229DF8B40040F2A11110FB01F009496A
:1008F00001EBC00101F562719DF8A00000EB40031F
:1009000003EB001001F83020A7229DF8B40040F25C
:10091000A1110EE058450020D81400209840002076
:10092000C7310020F8870020883E0020BC1200203C
:100930000FE010FB01F0FE4901EBC00000F5627012
:100940009DF8A01001EB410303EB011100EBC10086
:10095000427101F009BF00219DF8B40040F2A112DC
:1009600010FB02F0F24A02EBC00001719DF8B410D6
:1009700040F2A11011FB00F0114603E0F9E060E144
:10098000B0E2E4E201EBC00000F562709DF8A01057
:1009900001EB410202EB011110F83100022829DCC1
:1009A00003229DF8B40040F2A11110FB01F0E049D0
:1009B00001EBC00101F562719DF8A00000EB40035E
:1009C00003EB001001F83020A9229DF8B40040F29A
:1009D000A11110FB01F0D64901EBC00000F56270D7
:1009E0009DF8A01001EB410303EB011100EBC100E6
:1009F0004271BDE09DF8B41040F2A11011FB00F06F
:100A0000CB4901EBC00000F562709DF8A01001EB2E
:100A1000410202EB011110F83100052829DC062201
:100A20009DF8B40040F2A11110FB01F0C04901EBA8
:100A3000C00101F562719DF8A00000EB400303EBDB
:100A4000001001F83020A2229DF8B40040F2A1115C
:100A500010FB01F0B64901EBC00000F562709DF893
:100A6000A01001EB410303EB011100EBC100427147
:100A70007EE09DF8B41040F2A11011FB00F0AC49EB
:100A800001EBC00000F562709DF8A01001EB41027F
:100A900002EB011100EBC1004079A52815D19DF8AA
:100AA000B41001EB410000EB0110A24901EB001072
:100AB00030309DF8A01000EB0110801C09900078E8
:100AC00020F00400001D099908709DF8B41040F250
:100AD000A11011FB00F0964901EBC00000F5627017
:100AE0009DF8A01001EB410202EB011100EBC100E7
:100AF0008078A1283CD09DF8B41040F2A11011FBE1
:100B000000F08B4901EBC00101F562719DF8A00076
:100B100000EB400202EB001001EBC00082789DF870
:100B2000B40040F2A11110FB01F0814901EBC001BA
:100B300001F562719DF8A00000EB400303EB00108B
:100B400001EBC0004271A1229DF8B40040F2A11156
:100B500010FB01F0764901EBC00000F562709DF8D2
:100B6000A01001EB410303EB011100EBC100827007
:100B7000EFE69DF8B41040F2A11011FB00F06C49B3
:100B800001EBC00000F562709DF8A01001EB41027E
:100B900002EB011100EBC1004079A42830D19DF88F
:100BA000B41001EB410000EB0110624901EB0010B1
:100BB00030309DF8A01000EB0110801C09900078E7
:100BC00020F0200120310998017000229DF8B40026
:100BD00040F2A11110FB01F0554901EBC00101F5F4
:100BE00062719DF8A00000EB400303EB001001EBE5
:100BF000C00080F845209DF8B4100220F9F756FA9D
:100C000000219DF8B40040F2A11210FB02F0484A06
:100C100002EBC0000171A1229DF8B40040F2A111C5
:100C200010FB01F0424901EBC00000F562709DF835
:100C3000A01001EB410303EB011100EBC100427175
:100C400087E69DF8B41040F2A11011FB00F038497E
:100C500001EBC00000F562709DF8A01001EB4102AD
:100C600002EB011110F83100012834DC00219DF85D
:100C7000B40040F2A11210FB02F02D4A02EBC000BA
:100C8000017102229DF8B40040F2A11110FB01F0A5
:100C9000274901EBC00101F562719DF8A00000EB4E
:100CA000400303EB001001F83020A3229DF8B400AC
:100CB00040F2A11110FB01F01D4901EBC00000F54D
:100CC00062709DF8A01001EB410303EB011100EBF2
:100CD000C100427105E19DF8B41040F2A11011FB72
:100CE00000F0134901EBC00000F562709DF8A01000
:100CF00001EB410202EB011110F83100042839DC4C
:100D000000219DF8B40040F2A11210FB02F0084A45
:100D100002EBC000017105229DF8B40040F2A11160
:100D200010FB01F0024901EBC00101F5627103E023
:100D300058450020984000209DF8A00000EB40039B
:100D400003EB001001F83020A3229DF8B40040F21C
:100D5000A11110FB01F0FE4901EBC00000F562702B
:100D60009DF8A01001EB410303EB011100EBC10062
:100D70004271B6E09DF8B41040F2A11011FB00F0F2
:100D8000F34901EBC00000F562709DF8A01001EB83
:100D9000410202EB011110F83100062815DCA122F6
:100DA0009DF8B40040F2A11110FB01F0E84901EBFD
:100DB000C00000F562709DF8A01001EB410303EB49
:100DC000011100EBC10042718BE09DF8B41040F2BC
:100DD000A11011FB00F0DE4901EBC00101F56271C9
:100DE0009DF8A00000EB400202EB001011F830105B
:100DF0009DF8B40040F2A11210FB02F0D44A02EBBD
:100E0000C000407981426CD19DF8B41040F2A1102D
:100E100011FB00F0114601EBC00000F562709DF877
:100E2000A01001EB410202EB011100EBC100807840
:100E3000A12836D0A3229DF8B40040F2A11110FBE6
:100E400001F0C34901EBC00101F562719DF8A000FA
:100E500000EB400303EB001001EBC00042719DF872
:100E6000B41040F2A11011FB00F0B94901EBC00031
:100E700000F562709DF8A01001EB410202EB011138
:100E800000EBC1008078A2282BD000209DF8B41080
:100E900040F2A11211FB02F1AD4A02EBC10108714F
:100EA0001FE0A1229DF8B40040F2A11110FB01F057
:100EB000A74901EBC00101F562719DF8A00000EBAC
:100EC000400303EB001001EBC000427101219DF8CB
:100ED000B40040F2A11210FB02F09D4A02EBC000E8
:100EE000017136E5A1229DF8B40040F2A11110FB7A
:100EF00001F0974901EBC00101F562719DF8A00076
:100F000000EB400303EB001001EBC00042719DF8C1
:100F1000B40040F2A11110FB01F08D4901EBC001BA
:100F200001F562719DF8A00000EB400303EB001097
:100F300001EBC000827000219DF8B40040F2A112C4
:100F400010FB02F0824A02EBC000017101E50021B2
:100F50009DF8B40040F2A11210FB02F07C4A02EBB3
:100F6000C0000171A7229DF8B40040F2A11110FB4E
:100F700001F0774901EBC00101F562719DF8A00015
:100F800000EB400303EB001001EBC00042719DF841
:100F9000B41001EB4100C0EBC1106E4901EBC00081
:100FA000407930287DD19DF8B41040F2A11011FB9A
:100FB00000F0674901EBC00101F562719DF8A000E6
:100FC00000EB400202EB001011F830109DF8B40065
:100FD00040F2A11210FB02F05D4A02EBC000407922
:100FE00081425ED19DF8B40000EB400101EB00109E
:100FF000A2F5986101EB001030309DF8A01000EBD5
:101000000110801C0990007820F0010209980270FC
:101010009DF8B40000EB400101EB00104E4901EBDC
:10102000001030309DF8A01000EB0110801C0990DA
:10103000007820F00202099802709DF8B40040F296
:10104000A11110FB01F0424901EBC00000F56270F4
:101050009DF8A01001EB410202EB011100EBC10071
:10106000C078312832D19DF8B40000EB400101EB8B
:101070000010394901EB001030309DF8A01000EB52
:101080000110801C0990007820F02002099802705D
:1010900000229DF8B40040F2A11110FB01F001E024
:1010A000FEE340E02A4901EBC00000F562709DF8C4
:1010B000A01001EB410303EB011100EBC10080F82C
:1010C00045209DF8B4100220F8F7F0FF9DF8B40019
:1010D00040F2A11110FB01F01D4901EBC00000F529
:1010E00062709DF8A01001EB410202EB011100EBD0
:1010F000C10090F84600012814D1A9229DF8B4003F
:1011000040F2A11110FB01F0114901EBC00000F504
:1011100062709DF8A01001EB410303EB011100EB9D
:10112000C1008270DEE39DF8B40000EB4001C1EB2A
:10113000C010084901EBC000407931287ED19DF8EC
:10114000B40040F2A11110FB01F0014906E00000DB
:1011500058450020F88700209840002001EBC0018E
:1011600001F562719DF8A00000EB400202EB001057
:1011700011F830109DF8B40040F2A11210FB02F0FB
:10118000FE4A02EBC0004079814257D19DF8B4007D
:1011900040F2A11110FB01F0114601EBC00000F577
:1011A00062709DF8A01001EB410202EB011100EB0F
:1011B000C10090F8460058BB01229DF8B40040F2EF
:1011C000A11110FB01F0ED4901EBC00101F56271C5
:1011D0009DF8A00000EB400303EB001001EBC00002
:1011E00080F845209DF8B40000EB400101EB0010B1
:1011F000E34901EB001130319DF8A00001EB001034
:10120000801C0990007820F00100401C09990870AA
:101210009DF8B40000EB400101EB0010D84901EB50
:10122000001030309DF8A01000EB0110801C0990D8
:10123000007820F002020998027000E00CE2D14828
:1012400090F8E00780B19DF8B40000EB400101EB9D
:101250000010CB4901EB001030309DF8A01000EBDE
:101260000110807A022878D1C74890F82900012817
:10127000F9D1C548D0F80C02C349498D88426CD2D7
:101280009DF8B40040F2A11110FB01F0BB4901EB45
:10129000C00000F562709DF8A01001EB410202EB66
:1012A000011100EBC10090F84500012854D19DF8D0
:1012B000B40040F2A11110FB01F0B04901EBC000F5
:1012C00000F562709DF8A01001EB410202EB0111E4
:1012D00000EBC10090F87F00F0BB01229DF8B40044
:1012E00000EB400101EB0010A54901EB001130318A
:1012F0009DF8A00001EB0010C2724FF010429DF863
:10130000B40040F2A11110FB01F09C4901EBC001B7
:1013100001F562719DF8A00000EB400303EB0010A3
:1013200001EBC00082609DF8B40000EB400101EBCE
:101330000010934901EB001130319DF8A00001EB42
:10134000001001789DF8B40040F2A11210FB02F0E9
:101350008A4A02EBC00001E070E005E141709DF8AF
:10136000B40040F2A11110FB01F0114601EBC001E5
:1013700001F562719DF8A00000EB400202EB001045
:1013800011F830109DF8B40040F2A11210FB02F0E9
:101390007A4A02EBC000407981423ED100229DF89A
:1013A000B40040F2A11110FB01F0744901EBC0013F
:1013B00001F562719DF8A00000EB400303EB001003
:1013C00001EBC000C271A4229DF8B40040F2A1114B
:1013D00010FB01F0694901EBC00101F562719DF854
:1013E000A00000EB400303EB001001EBC000827093
:1013F000A3229DF8B40040F2A11110FB01F05F4957
:1014000001EBC00000F562709DF8A01001EB4103F4
:1014100003EB011100EBC100427100229DF8B40002
:1014200000EB400101EB0010554901EB001030309A
:101430009DF8A01000EB0110426053E29DF8B4004B
:1014400040F2A11110FB01F04C4901EBC00000F586
:1014500062709DF8A01001EB410202EB011100EB5C
:10146000C10090F8450001287ED19DF8B40040F2FB
:10147000A11110FB01F0414901EBC00101F56271BE
:101480009DF8A00000EB400202EB001001EBC00051
:1014900090F8801040F2A11011FB00F0374901EBE9
:1014A000C00101F562719DF8B40040F2A11210FB79
:1014B00002F0324A02EBC00000F562709DF8A020F5
:1014C00002EB420303EB021200EBC20090F8810032
:1014D00000EB400202EB001001EBC00090F87E0030
:1014E000032841D102229DF8B40000EB400101EB3A
:1014F0000010234901EB001130319DF8A00001EBF1
:101500000010C2724FF010429DF8B40040F2A111D9
:1015100010FB01F0194901EBC00101F562719DF862
:10152000A00000EB400303EB001001EBC000826061
:101530009DF8B40000EB400101EB0010104901EBF5
:10154000001130319DF8A00001EB001001789DF8EA
:10155000B40040F2A11210FB02F0084A02EBC000F6
:1015600041709DF8B40000E09BE140F2A11110FB36
:1015700001F0114601EBC00108E0000058450020D1
:1015800098400020BC320020BC12002001F562719E
:101590009DF8A00000EB400202EB001011F83010A3
:1015A0009DF8B40040F2A11210FB02F0FE4A02EBDB
:1015B000C000407981423ED100229DF8B40040F243
:1015C000A11110FB01F0F84901EBC00101F56271B6
:1015D0009DF8A00000EB400303EB001001EBC000FE
:1015E000C271A4229DF8B40040F2A11110FB01F0D9
:1015F000ED4901EBC00101F562719DF8A00000EB1F
:10160000400303EB001001EBC0008270A3229DF8A1
:10161000B40040F2A11110FB01F0E34901EBC0005E
:1016200000F562709DF8A01001EB410303EB01117E
:1016300000EBC100427100229DF8B40000EB4001B4
:1016400001EB0010D94901EB001030309DF8A010DB
:1016500000EB0110426045E19DF8B40000EB400151
:10166000C1EBC010D24901EBC000407933287DD1D5
:101670009DF8B40000EB400101EB0010CB4901EBF9
:10168000001030309DF8A01000EB0110801C099074
:10169000007820F00100401C099908709DF8B40002
:1016A00000EB400101EB0010C04901EB00103030AD
:1016B0009DF8A01000EB0110801C0990007820F02C
:1016C0002002099802709DF8B40000EB400101EB84
:1016D0000010B64901EB001030309DF8A01000EB6F
:1016E0000110801C0990007820F00200801C0999EC
:1016F00008709DF8B40040F2A11110FB01F0AA4956
:1017000001EBC00042799DF8B40040F2A11110FB3A
:1017100001F0A54901EBC00000F562709DF8A01032
:1017200001EB410303EB011100F831209DF8B400F7
:1017300000EB400101EB00109C4901EB0010303040
:101740009DF8A01000EB0110801C0990007820F09B
:1017500080008030099908709DF8B41001EB4100B9
:1017600000EB0110914901EB001000E023E0303064
:101770009DF8A01000EB01108078C0F3400020B964
:101780009DF8B4100220F8F791FCA2229DF8B40055
:1017900040F2A11110FB01F0834901EBC00000F5FC
:1017A00062709DF8A01001EB410303EB011100EB07
:1017B000C100827096E09DF8B41001EB4100C0EBCF
:1017C000C1107B4901EBC0004079342869D19DF8F4
:1017D000B41001EB410000EB0110744901EB001063
:1017E00030309DF8A01000EB0110801C09900078AB
:1017F00020F02002099802709DF8B41001EB41001E
:1018000000EB0110694901EB001030309DF8A01089
:1018100000EB0110801C0990007820F0020209986A
:10182000027001229DF8B40040F2A11110FB01F0FA
:101830005D4901EBC00000F562709DF8A01001EB5E
:10184000410303EB011100EBC10080F84620A922FF
:101850009DF8B40040F2A11110FB01F0524901EBD8
:10186000C00000F562709DF8A01001EB410303EB8E
:10187000011100EBC10082709DF8B41040F2A1107C
:1018800011FB00F0484901EBC00042799DF8B4001B
:1018900040F2A11110FB01F0434901EBC00001E04F
:1018A000E3E21FE000F562709DF8A01001EB410338
:1018B00003EB011100F831209DF8B41001EB410059
:1018C00000EB0110394901EB001030309DF8A010F9
:1018D00000EB0110801C0990007820F0800080301F
:1018E0000999087000202E902F900021399122E054
:1018F000DDE92E10000140EA11720901CDE92E1236
:101900009DF8B41001EB4100C0EBC110284901EB78
:10191000C001BDF8E400801D085C3038C117DDE966
:101920002E34184341EA0402CDE92E02BDF8E4004A
:10193000401C80B23990BDF8E4000828D8DB9DF83F
:10194000B4002E9940F2A11210FB02F0164A02EBED
:10195000C00202F562729DF8A00000EB400303EBA9
:10196000001002EBC000C0F81A1000222E922F9235
:10197000002139912AE0DDE92E10000140EA1172C0
:101980000901CDE92E129DF8B41001EB4100C0EB26
:10199000C110074901EBC001BDF8E4000F30085C3D
:1019A0003038C11706E0000058450020984000205C
:1019B000F8870020DDE92E34184341EA0402CDE91E
:1019C0002E02BDF8E400401C80B23990BDF8E4005E
:1019D0000628D0DB9DF8B4002E9940F2A11210FB2E
:1019E00002F0FE4A02EBC00202F562729DF8A0000E
:1019F00000EB400303EB001002EBC0004163002248
:101A00002E922F920021399122E0DDE92E10000163
:101A100040EA11720901CDE92E129DF8B41001EBD4
:101A20004100C0EBC110EE4901EBC001BDF8E4007C
:101A30001530085C3038C117DDE92E24104341EA27
:101A40000402CDE92E02BDF8E400401C80B23990BA
:101A5000BDF8E4000828D8DB9DF8B4002E9940F2C8
:101A6000A11210FB02F0DD4A02EBC00202F5627225
:101A70009DF8A00000EB400303EB001002EBC00058
:101A8000C0F81E109DF8B41001EB4100C0EBC1106E
:101A9000D34901EBC00042799DF8B40040F2A11196
:101AA00010FB01F0CD4901EBC00101F562719DF819
:101AB000A00000EB400303EB001001EBC000C2707C
:101AC0009DF8B41001EB410000EB0110C54901EB9A
:101AD000001130319DF8A00001EB001082789DF8D4
:101AE000B40040F2A11110FB01F0BC4901EBC001B0
:101AF00001F562719DF8A00000EB400303EB0010BC
:101B000001EBC00002769DF8B41040F2A11011FB69
:101B100000F0B24901EBC00101F562719DF8A0002F
:101B200000EB400202EB001011F830109DF8B400F9
:101B300040F2A11210FB02F0A84A02EBC00040796B
:101B400081427DDA00219DF8B40040F2A11210FB21
:101B500002F0A24A02EBC0000171A7229DF8B40076
:101B600040F2A11110FB01F09C4901EBC00101F50D
:101B700062719DF8A00000EB400303EB001001EB45
:101B8000C000427101219DF8B40040F2A11210FB87
:101B900002F0924A02EBC00001719DF8B41040F2CD
:101BA000A11011FB00F0114601EBC00042799DF835
:101BB000B40040F2A11110FB01F0884901EBC00113
:101BC00001F562719DF8A00000EB400303EB0010EB
:101BD00001F83020A1229DF8B40040F2A11110FBC1
:101BE00001F07E4901EBC00101F562719DF8A00092
:101BF00000EB400303EB001001EBC00042719DF8C5
:101C0000B41001EB410000EB0110764901EB00112B
:101C100030319DF8A00001EB0010801C0990007885
:101C200020F080008030099908709DF8B41001EB15
:101C3000410000EB01106B4901EB0010303000E077
:101C40005BE09DF8A01000EB0110801C099000786B
:101C500020F00400001D099908709DF8B41001EBF4
:101C6000410000EB01105F4901EB001030309DF89E
:101C7000A01000EB01108078C0F34010E8B39DF88D
:101C8000B41001EB410000EB0110564901EB0010CC
:101C900030309DF8A01000EB0110801C09900078F6
:101CA00020F02002099802709DF8B41001EB410069
:101CB00000EB01104B4901EB001030309DF8A010F3
:101CC00000EB01108078C0F34000E8BB9DF8B41031
:101CD00001EB410000EB0110424901EB00103030F4
:101CE0009DF8A01000EB0110801C0990007820F0F6
:101CF000080008300999087000E0B5E09DF8B400CC
:101D00009DF8A01001EB0010C217CDE92E029DF83E
:101D1000B41040F2A11011FB00F0304901EBC000FB
:101D200000F562709DF8A01001EB410202EB011179
:101D300000EBC100223009902E9800EB40012A48A8
:101D400000EB41100D3000E089E010220890099965
:101D5000F6F77BFA9DF8B41040F2A11011FB00F0E9
:101D60001E4901EBC00101F562719DF8A00000EB76
:101D7000400202EB001001EBC0012E9800EB400284
:101D8000194800EB421051F81A2F40F8012F49680A
:101D900041609DF8B41001EB410000EB01101149C6
:101DA00001EB001130319DF8A00001EB001001782B
:101DB0002E9800EB40020C4800EB421001702E9868
:101DC00000EB4001084800EB41110848026841F867
:101DD0001D2F808888809DF8B41009E058450020A8
:101DE000F887002098400020D8140020C731002038
:101DF00040F2A11011FB00F0FE4901EBC00101F51A
:101E000062719DF8A00000EB400202EB001001EBB4
:101E1000C000416B2E9800EB4002F74800EB4210E7
:101E2000C0F809109DF8B41001EB410000EB01105F
:101E3000F24901EB001130319DF8A00001EB0010D8
:101E400041682E9800EB4002EB4800EB4210C0F8CE
:101E500023102E9881B208200991F8F727F99DF8F0
:101E6000B4100220F8F722F9FEE300202E902F9004
:101E70000021399122E0DDE92E10000140EA1172C3
:101E80000901CDE92E129DF8B41001EB4100C0EB21
:101E9000C110DB4901EBC001BDF8E4000B30085C68
:101EA0003038C117DDE92E34184341EA0402CDE988
:101EB0002E02BDF8E400401C80B23990BDF8E40069
:101EC0000C28D8DB9DF8B400DDE92E1240F2A113F6
:101ED00010FB03F0C74B03EBC00303F562739DF8DF
:101EE000A00000EB400404EB001003EBC00040F83E
:101EF000221F426000222E922F920021399122E06F
:101F0000DDE92E10000140EA11720901CDE92E121F
:101F10009DF8B41001EB4100C0EBC110B84901EBD2
:101F2000C001BDF8E4001730085C3038C117DDE9A6
:101F30002E34184341EA0402CDE92E02BDF8E40034
:101F4000401C80B23990BDF8E4000C28D8DB9DF825
:101F5000B400DDE92E2140F2A11310FB03F0A54BE4
:101F600003EBC00303F562739DF8A00000EB40048F
:101F700004EB001003EBC00022308260C16000213E
:101F80009DF8B40040F2A11210FB02F0994A02EB56
:101F9000C00001719DF8B41040F2A11011FB00F0D7
:101FA000114601EBC00000F562709DF8A01001EB36
:101FB000410202EB011110F83100032814DC042265
:101FC0009DF8B40040F2A11110FB01F0894901EB2A
:101FD000C00000F562709DF8A01001EB410303EB17
:101FE000011100F831207EE39DF8B41040F2A110F9
:101FF00011FB00F07F4901EBC00101F562719DF812
:10200000A00000EB400202EB001011F830109DF828
:10201000B40040F2A11210FB02F0764A02EBC000BD
:1020200040798142DFD19DF8B4009DF8A01001EB0A
:102030000010C217CDE92E02724890F8E00708B3ED
:102040009DF8B41001EB410000EB01106B4901EB6E
:10205000001030309DF8A01000EB0110807A0228AB
:1020600010D09DF8B41001EB410000EB0110634962
:1020700001EB001030309DF8A01000EB0110C07A89
:1020800000287DDD00229DF8B40000EB400101EB4B
:1020900000105A4901EB001030309DF8A01000EB01
:1020A0000110C2725848D0F80C020521B0FBF1F2C1
:1020B00001FB120000EB400153482C3000EB4110B3
:1020C0000D3009909DF8B40040F2A11110FB01F011
:1020D000484901EBC00000F562709DF8A01001EBCB
:1020E000410202EB011100EBC10022301022014637
:1020F00008900998F6F7A9F84348D0F80C02052192
:10210000B0FBF1F201FB120000EB40013E482C3025
:1021100000EB41129DF8B40040F2A11110FB01F058
:10212000344901EBC00101F562719DF8A00000EB9C
:10213000400303EB001001EBC00050F81A1F42F8F7
:10214000011F406850603048D0F80C020521B0FBF8
:10215000F1F201FB120000EB40012B482C3000EBA8
:1021600041129DF8B40000EB400101EB001023493F
:1021700001EB001130319DF8A00001EB001000E0F0
:1021800095E1007810702048D0F80C020521B0FBD2
:10219000F1F201FB120000EB40011B482C3000EB78
:1021A00041129DF8B40040F2A11110FB01F0114959
:1021B00001EBC00101F562719DF8A00000EB400346
:1021C00003EB001001EBC000406BC2F809000E48A1
:1021D000D0F80C020521B0FBF1F201FB120000EB7C
:1021E000400109482C3000EB41110648F5380268DF
:1021F0000CE0000058450020D81400209840002032
:10220000F8870020BC320020BC12002041F81D2FAE
:1022100080888880FE48D0F80C020521B0FBF1F2DE
:1022200001FB120000EB4001F9482C3000EB411299
:102230009DF8B40000EB400101EB0010F54901EB03
:10224000001130319DF8A00001EB00104068C2F889
:10225000230000229DF8B40000EB400101EB0010C8
:10226000EC4901EB001130319DF8A00001EB0010AA
:1022700042600021399154E0E548D0F80C02052174
:10228000B0FBF1F201FB120000EB4001E0482C3002
:1022900000EB41112731BDF8E4409DF8B40040F255
:1022A000A11210FB02F0DC4A02EBC00202F56272DE
:1022B0009DF8A00000EB400303EB001002EBC00010
:1022C00090F8800040F2A11210FB02F0D24A02EB1B
:1022D000C00202F562729DF8B40040F2A11310FB37
:1022E00003F0CD4B03EBC00303F562739DF8A00030
:1022F00000EB400505EB001003EBC00090F88100F7
:1023000000EB400303EB001002EBC0024732BDF8C4
:10231000E400001D105C0855BDF8E400401C81B2CB
:102320003991BDF8E4000628A6DB0021399142E08E
:1023300000239DF8B40040F2A11110FB01F0B64952
:1023400001EBC00101F562719DF8A00000EB4002B5
:1023500002EB001001EBC00090F8800040F2A111E8
:1023600010FB01F0AC4901EBC00101F562719DF871
:10237000B40040F2A11210FB02F0A74A02EBC00227
:1023800002F562729DF8A00000EB400404EB00101F
:1023900002EBC00090F8810000EB400202EB00105D
:1023A00001EBC0014731BDF8E4000B54BDF8E40077
:1023B000401C81B23991BDF8E4000A28B8DB94488A
:1023C000D0F80C020521B0FBF1F080B20146099073
:1023D0000220F6F77DFE00210620F7F767FE8C4805
:1023E000D0F80C028A49498D884206D28848D0F834
:1023F0000C02401C8649C1F80C0200210520F7F7A9
:1024000055FE9DF8B41001EB410000EB011081492D
:1024100001EB001030309DF8A01000EB0110801C83
:102420000990007820F00802099802707848D0F8E6
:102430000C020521B0FBF1F201FB120000EB4001A0
:1024400073482C3000EB4110D0F823202E9800EB7D
:102450004001724800EB4110C0F823200020399061
:1024600020E06B48D0F80C020521B0FBF1F201FB33
:10247000120000EB400166482C3000EB4110273081
:10248000BDF8E410425C2E9800EB4001634800EB7D
:1024900041112731BDF8E4000A54BDF8E400401CA6
:1024A00081B23991BDF8E4000628DADB59E09DF8E5
:1024B000B41001EB410000EB0110564901EB001094
:1024C00030309DF8A01000EB0110801C09900078BE
:1024D00020F008000830099908709DF8B41001EB4D
:1024E000410000EB01104B4901EB001030309DF82A
:1024F000A01000EB011042682E9800EB4001474805
:1025000000EB4110C0F823200020399025E09DF811
:10251000B41040F2A11011FB00F03F4901EBC001E3
:1025200001F562719DF8A00000EB400202EB001083
:1025300001EBC0014731BDF8E4000A5C2E9800EBC6
:102540004001364800EB41112731BDF8E4000A5440
:10255000BDF8E400401C81B23991BDF8E4000628C2
:10256000D5DB00229DF8B40040F2A11110FB01F070
:10257000294901EBC00101F562719DF8A00000EB53
:10258000400303EB001001EBC00080F846209DF8EB
:10259000B4100220F7F78AFD9DF8B40040F2A111B3
:1025A00010FB01F01C4901EBC00101F562719DF8BF
:1025B000A00000EB400202EB001001EBC000223053
:1025C00009902E9800EB4001144800EB41110D31A9
:1025D00010220891DDE90801F5F737FE9DF8B410E7
:1025E00040F2A11011FB00F00B4901EBC00101F515
:1025F00062719DF8A00000EB400202EB001001EBBD
:10260000C0012E9800EB4002044800EB421007E0A6
:10261000BC1200209840002058450020D81400200B
:1026200051F81A2F40F8012F496841609DF8B41005
:1026300001EB410000EB0110F94901EB00113031D1
:102640009DF8A00001EB001001782E9800EB4002ED
:10265000F44800EB421001702E9800EB4001F14865
:1026600000EB4111F04800E07EE0026841F81D2FC8
:10267000808888809DF8B41040F2A11011FB00F012
:10268000EA4901EBC00101F562719DF8A00000EB81
:10269000400202EB001001EBC000416B2E9800EBF2
:1026A0004002E04800EB4210C0F809109DF8B41059
:1026B00001EB410000EB0110D94901EB0011303171
:1026C0009DF8A00001EB001041682E9800EB40023D
:1026D000D44800EB4210C0F823102E9881B2082095
:1026E0000991F7F7E3FC00229DF8B40040F2A11134
:1026F00010FB01F0CD4901EBC00101F562719DF8BD
:10270000A00000EB400303EB001001EBC00080F8D9
:102710004620A7229DF8B40040F2A11110FB01F061
:10272000C24901EBC00101F562719DF8A00000EB08
:10273000400303EB001001EBC0004271A2229DF8A0
:10274000B40040F2A11110FB01F0B84901EBC00147
:1027500001F562719DF8A00000EB400303EB00104F
:1027600001EBC000827000BF00BF0BF013BD002161
:10277000AF4A9DF8B40002EB00129DF8A00011547E
:102780009DF8B41001EB4100C0EBC110A94901EB69
:10279000C000407870280ED19DF8B41001EB4100C4
:1027A000C0EBC110A34901EBC0008078FA2802D128
:1027B000B121259142E09DF8B41001EB4100C0EB3E
:1027C000C1109C4901EBC000407800F0F000C02827
:1027D0000ED19DF8B41001EB4100C0EBC11095493A
:1027E00001EBC0008078FA2802D1B621259125E0BE
:1027F0009DF8B41001EB4100C0EBC1108D4911F8F8
:10280000300000F0F000502818D19DF8B41001EB12
:102810004100C0EBC110874901EBC000407800F0D7
:10282000F00030280AD19DF8B41001EB4100C0EB54
:10283000C110804901EBC000817825919DF8B4104A
:1028400040F2A11011FB00F0784901EBC000817843
:1028500028910021764A9DF8B40002EB00129DF801
:10286000A0001154744890F82800012815D19DF853
:10287000B41001EB410000EB0110694901EB0010BD
:1028800030309DF8A01000EB0110801C09900078FA
:1028900020F08000803009990870BDF89400652808
:1028A00074D004DC012809D0032805D17FE0B128C9
:1028B00002D0B62800D100E08BE18AE19DF8B41087
:1028C00001EB4100C0EBC1105A4901EBC000007997
:1028D000012806D0022805D0032804D0052864D199
:1028E00002E062E061E060E09DF8B41040F2A11007
:1028F00011FB00F04D4901EBC00000F562709DF83E
:10290000A01001EB410202EB011110F83100E0BB15
:1029100000219DF8B40040F2A11210FB02F0434ADE
:1029200002EBC000017101229DF8B40040F2A11138
:1029300010FB01F03D4901EBC00101F562719DF80A
:10294000A00000EB400303EB001001F83020B6229A
:102950009DF8B40040F2A11110FB01F0334901EBE6
:10296000C00101F562719DF8A00000EB400303EB8C
:10297000001001EBC0004271B2229DF8B40040F299
:10298000A11110FB01F0294901E00DE037E001EB56
:10299000C00000F562709DF8A01001EB410303EB4D
:1029A000011100EBC100827000BF00BF11E19DF872
:1029B000B41001EB4100C0EBC1101E4901EBC00097
:1029C000C1791E4880F8031D9DF8B41001EB410049
:1029D00000EB0110124901EB001130319DF8A0000D
:1029E00001EB0010801C0990144890F8030DC208F8
:1029F0000998007862F3000009990870E9E09DF8F1
:102A0000B41001EB4100C0EBC1100A4901EBC0005A
:102A1000007900F0F00098B9B821259112E000008B
:102A200098400020D8140020C731002058450020CD
:102A3000883E0020F8870020BC120020BC22002025
:102A4000B92125910021399120E09DF8B41001EBC6
:102A5000410000EB0110FE4901EB00113031BDF8DF
:102A6000E40001EB001041789DF8B40000EB400257
:102A7000C2EBC010F74A12F830005038814200D142
:102A800012E0BDF8E400401C81B239919DF8B41009
:102A900001EB410000EB0110ED4901EB0010C179A1
:102AA000BDF8E4008142D0DC00BF9DF8B41040F2D4
:102AB000A11011FB00F0E84901EBC00000F56270C5
:102AC0009DF8A01001EB410202EB011110F831005A
:102AD000012834D100219DF8B40040F2A11210FB6E
:102AE00002F0DD4A02EBC000017102229DF8B40041
:102AF00040F2A11110FB01F0D74901EBC00101F533
:102B000062719DF8A00000EB400303EB001001F898
:102B10003020B9229DF8B40040F2A11110FB01F061
:102B2000CD4901EBC00000F562709DF8A01001EBEB
:102B3000410303EB011100EBC100427148E09DF835
:102B4000B41040F2A11011FB00F0C34901EBC0002A
:102B500000F562709DF8A01001EB410202EB01113B
:102B600010F83100012833D100219DF8B40040F263
:102B7000A11210FB02F0B84A02EBC0000171022260
:102B80009DF8B40040F2A11110FB01F0B24901EB35
:102B9000C00101F562719DF8A00000EB400303EB5A
:102BA000001001F83020B9229DF8B40040F2A111C4
:102BB00010FB01F0A84901EBC00000F562709DF820
:102BC000A01001EB410303EB011100EBC1004271C6
:102BD00000BF00BFC9E59DF8B41001EB410000EB58
:102BE00001109B4901EB0010007B20B101287CD033
:102BF00002287BD1EBE299499DF8B40031F810002E
:102C0000801F81B209919DF8B41001EB4100C0EB27
:102C1000C110904901EBC000401C08900999F6F7DB
:102C200093FE0022CDE930029DF8B41001EB410083
:102C3000C0EBC110874901EBC00288489DF8B41071
:102C400030F81100401F11180991042109981FF054
:102C500003F9C217CDE92E022FA819C82E995940A1
:102C6000604001437ED17E4A9DF8B40002EB001023
:102C700001709DF8B41001EB4100C0EBC110754923
:102C800001EBC00001792591BDF89400312802D0F4
:102C9000452868D1FBE071489DF8B41030F8110068
:102CA0001838412190FBF1F0C217C1B2CDE92E02D4
:102CB0006C4880F8AC1000203990DEE09DF8B4102C
:102CC00001EB4100C0EBC110624901EBC001BDF84E
:102CD000E40000EB801014300A5C6249AD31BDF8AD
:102CE000E4000A549DF8B41001E0D3E06EE201EB79
:102CF0004100C0EBC110574901EBC001BDF8E40031
:102D000000EB80101A3001440991082109981FF046
:102D100061F88DED0E0A534AB932BDF8E4000E9900
:102D200002EB001041609DF8B41001EB4100C0EBD4
:102D3000C110484901EBC001BDF8E40000EB801070
:102D4000323001440991082109981FF043F88DEDB4
:102D50000E0A444AB932BDF8E4000E9902EB0010A5
:102D6000016001E095E093E09DF8B41001EB4100B3
:102D7000C0EBC110374901EBC001BDF8E40000EB26
:102D800080103A3001440991082109981FF022F877
:102D90008DED0E0A334AB932BDF8E4000E9902EB0C
:102DA000001081609DF8B40000EB4001C1EBC01041
:102DB000284901EBC001BDF8E40000EB801042306F
:102DC00001440991082109981FF004F88DED0E0ABD
:102DD000244AB932BDF8E4000E9902EB0010C1603C
:102DE0009DF8B40000EB400101EB0010184901EB25
:102DF00000113031BDF8E40001EB0010801C099097
:102E0000007820F080008030099908709DF8B400A7
:102E100000EB4001C1EBC0100E4901EBC0020F48AE
:102E20009DF8B41030F81100401E125C9DF8B400FB
:102E300040F2A11110FB01F0074901EBC00000F5C1
:102E400062709DF8A01001EB410303EB01110BE050
:102E500098400020F887002058450020787900200D
:102E6000883E0020BC32002000EBC10080F84420E6
:102E7000BDF8E400401C80B23990BDF8E4000021A8
:102E8000DDE92E34C01AA141FFF618AF00E000BF03
:102E900000BFB4E29DF8B40000EB4001C1EBC010EC
:102EA000FE4901EBC000407D9DF8B41001EB4102EA
:102EB000C2EBC111F94A02EBC101897D40EA012050
:102EC000C217CDE92E029DF8B40000EB4001C1EB22
:102ED000C010F24901EBC001099115210998F6F7DC
:102EE00017FD0022CDE930022FA819C82E995940AC
:102EF000604001437ED19DF8B40000EB4001C1EB7E
:102F0000C010E64911F83000401EC1B228910021DE
:102F1000E34A9DF8B40002EB00129DF8A0001154A2
:102F2000E04A9DF8A00011549FEDDF0A10EE101A40
:102F30000C329DF8A00002EB001041609DF8B40037
:102F400000EB4001C1EBC010D44901EBC000817916
:102F50009DF8B40000EB4002C2EBC010CF4A02EB78
:102F6000C000407941EA002000EE100AB8EEC00A25
:102F70009FEDCE1AC0EE010A9DF8B40000EB4001AF
:102F8000C1EBC010114601EBC00001799DF8B400FF
:102F900000EB4002C2EBC010C04A02EBC000C07898
:102FA00041EA002000EE100AB8EEC00A30EE800AB6
:102FB00010EE101ABB4A0C329DF8A00002EB001074
:102FC00001609DF8B40000EB4001C1EBC010B349B3
:102FD00001EBC000817A9DF8B40000EB4002C2EB27
:102FE000C010AE4A02EBC000407A41EA002000EE79
:102FF000100A00E0EAE0B8EEC00A9FEDAC1AC0EE9D
:10300000010A9DF8B40000EB4001C1EBC01011466D
:1030100001EBC000017A9DF8B40000EB4002C2EB66
:10302000C0109E4A02EBC000C07941EA002000EEC9
:10303000100AB8EEC00A30EE800A10EE101A994A53
:103040000C329DF8A00002EB001081609DF8B400E6
:1030500000EB4001C1EBC010904901EBC000C07A09
:1030600000F0800038BB9DF8B40000EB4001C1EBDC
:10307000C0108A4901EBC000017B9DF8B40000EB51
:103080004002C2EBC010854A02EBC000C07A41EAA0
:10309000002000EE100AF8EEC00AB3EE001A80EE2F
:1030A000810A10EE100A7F4A0C329DF8A01002EB44
:1030B0000111C86047E09DF8B40000EB4001C1EB8E
:1030C000C011764800EBC100017B9DF8B40000EB15
:1030D0004002C2EBC010714A02EBC000C07A41EA64
:1030E0000020404280B200EE100AB8EEC00A8DED1A
:1030F000030A0398F5F712FB9FED6D0B53EC102BB1
:10310000CDE904019DED040B51EC100BF5F7EAF944
:103110009FED690B53EC102BCDE906019DED060BDD
:1031200051EC100BF5F769F9CDE908019DED080B9D
:1031300051EC100BF5F705FB5A4A0C329DF8A01024
:1031400002EB0111C8609DF8B40000EB400101EBF7
:1031500000105B4901EB001030309DF8A01000EB2F
:103160000110801C0990007820F0800080300999BF
:1031700008709DF8B40000EB4001C1EBC010474956
:1031800001EBC000C27D9DF8B40040F2A11110FB1C
:1031900001F04C4901EBC00000F562709DF8A010F1
:1031A00001EB410303EB011100EBC10080F8442067
:1031B0009DF8B41001EB410000EB0110404901EB18
:1031C0000010C1793748AD3880F8AC1017E19DF890
:1031D000B41001EB4100C0EBC110304901EBC0005D
:1031E000C0799DF8B41001EB4102C2EBC1112B4A2A
:1031F00002EBC101097A40EA0120C217CDE92E0293
:103200009DF8B41001EB4100C0EBC110234901EB64
:10321000C001099107210998F6F77AFB0022CDE950
:103220003002DDE93042DDE92E10614050400143BB
:103230007ED19DF8B41001EB4100C0EBC1101749DD
:1032400011F83000401EC1B228910021144A9DF8A7
:10325000B40002EB00100170124A9DF8A000115456
:103260009DF8B41001EB4100C0EBC1100B4901EB1C
:10327000C000817908460191F5F7CAF9CDE902014C
:103280009DED021B9FED100B22F08AFC8DED060BCD
:103290009DF8B41001EB41001AE00000F88700200F
:1032A000883E0020693300200000000000FF7F47B7
:1032B000000000000000304000000000000000009E
:1032C00098400020584500200000000000002440E5
:1032D000C0EBC110F64901EBC00001799DF8B400C4
:1032E00000EB4002C2EBC010F14A02EBC000C07814
:1032F00041EA002000EE100AB8EEC00A8DED030A84
:103300000398F5F70BFACDE904019DED060B53EC9C
:10331000102B9DED040B51EC100BF5F7E3F8CDE904
:1033200008019DED080B51EC100BF5F70AFA00E0CF
:1033300064E0E04A9DF8A01002EB011148601FED27
:10334000260A10EE100A9DF8A01002EB0111086089
:103350001FED2B0A10EE100A9DF8A01002EB0111D0
:1033600088601FED2F0A10EE100A9DF8A01002EBE6
:103370000111C8609DF8B41001EB410000EB011091
:1033800002F6235101EB001030309DF8A01000EB45
:103390000110801C0990007820F08000803009998D
:1033A00008709DF8B41001EB4100C0EBC110C0499A
:1033B00001EBC000427A9DF8B40040F2A11110FB6D
:1033C00001F0BD4901EBC00000F562709DF8A0104E
:1033D00001EB410303EB011100EBC10080F8442035
:1033E0009DF8B41001EB410000EB0110B34901EB73
:1033F0000010C179AF48B93880F8AC1000BF00BFE9
:103400000AF0C8BE9DF8B41001EB4100C0EBC1103A
:10341000A74901EBC000C1789DF8B40000EB400261
:10342000C2EBC010A24A02EBC000807841EA002142
:1034300029919DF8B41001EB4100C0EBC110114679
:1034400001EBC001BDF8A400401C095C9DF8B4006C
:1034500000EB4002C2EBC010954A02EBC002BDF87F
:10346000A400105C41EA0020C217CDE92E029DF8AD
:10347000B41001EB4100C0EBC1108D4901EBC0005D
:103480000990BDF8A410F6F743FA0022CDE9300206
:10349000DDE93042DDE92E1061405040014341F04A
:1034A00067869DF8B41001EB4100C0EBC110804964
:1034B00001EBC00041782891002139911CE09DF872
:1034C000B41001EB410000EB01107C4901EB00114D
:1034D0003031BDF8E40001EB001041789DF8A00008
:1034E000814204D1BDF8E400C1B2289112E0BDF8D8
:1034F000E400401C81B239919DF8B41001EB410009
:1035000000EB01106D4901EB0010C179BDF8E4003A
:103510008142D4DC00BF9DF8B41001EB410000EB08
:103520000110664901EB001030309DF8A01000EB4F
:103530000110801C0990007820F0800080300999EB
:1035400008709DF8B41001EB4100C0EBC110584960
:1035500001EBC000007925900020594A9DF8B41075
:1035600002EB01129DF8A0105054BDF89400F3280E
:103570007DD009DC05287BD006280ED0F12878D034
:10358000F22841F0F485F7E3F42873D0F62872D0DE
:10359000F72871D0F828F4D1EFE30621109100212B
:1035A0003691EBE3BDF84000401C81B210919DF8CC
:1035B000B41001EB4100C0EBC1103D4901EBC0016B
:1035C000BDF84000095C2591BDF84000401C81B267
:1035D0001091BDF89400F12804D0F22872D0F3289D
:1035E00071D1FDE39DF8B41001EB4100C0EBC110B7
:1035F0002F4901EBC001BDF84000095C2991BDF8DD
:103600004000401C81B210919DF8B41001EB4100C4
:1036100000EB0110294901EB001130319DF8A02089
:10362000BDF8D800104401EB0010407A00F0010012
:10363000E8B39DF8B41040F2A11011FB00F01E4950
:1036400001EBC00101F562719DF8A020BDF8D80022
:10365000104400EB400202EB001001EBC00090F8B8
:10366000900000F0010010BB9DF8B41005E0FDE3F0
:10367000FDE3FDE3FDE3FDE3FDE340F2A11011FBFB
:1036800000F00D4901EBC00101F562719DF8A02029
:10369000BDF8D800104400EB400202EB001001EB33
:1036A000C00090F8820010B1002139913CE09EE00A
:1036B000F8870020753300205845002098400020EE
:1036C000883E0020FCE3FAE39DF8B41040F2A1101C
:1036D00011FB00F0FC4901EBC00101F562719DF89E
:1036E000A020BDF8D800104400EB400202EB00100F
:1036F00001EBC00000F18301BDF8E4000A5C9DF815
:10370000B40000EB400101EB0010F04901EB0010A8
:103710000E30BDF8E410405C824200D008E0BDF8F5
:10372000E400401C81B23991BDF8E4000428CBDBF1
:1037300000BFBDF8E400042859D1042139912FE0DD
:103740009DF8B41040F2A11011FB00F0DE4901EB2E
:10375000C00101F562719DF8A020BDF8D8001044A9
:1037600000EB400202EB001001EBC00000F183010E
:10377000BDF8E4000A5C9DF8B40000EB400101EBE9
:103780000010D24901EB00100E30BDF8E410405C8F
:10379000824200D008E0BDF8E400401C81B23991BB
:1037A000BDF8E4000A28CBDB00BFBDF8E4000A281E
:1037B0001DD09DF8B41040F2A11011FB00F0C249D9
:1037C00001EBC00101F562719DF8A020BDF8D800A1
:1037D000104400EB400202EB001001EBC0009030FF
:1037E0000990007820F00100401C09990870BDF88C
:1037F000A4000F287ED19DF8B41001EB410000EB2E
:103800000110B24901EB001130319DF8A020BDF844
:10381000D800104401EB0010801C0990007820F0C3
:103820000400001D09990870002039902DE09DF8D2
:10383000B41001EB4100C0EBC110A54901EBC00180
:10384000BDF84020BDF8E40010440A5C9DF8B400C7
:1038500040F2A11110FB01F09B4901EBC00101F501
:1038600062719DF8A030BDF8D800184400EB400309
:1038700003EB001001EBC0014731BDF8E4000A542E
:10388000BDF8E400401C81B23991BDF8E4000A287B
:10389000CDDBBDF840000A3081B210910021399192
:1038A0002FE09DF8B41001EB4100C0EBC110884936
:1038B00001EBC001BDF84020BDF8E40010440A5CF3
:1038C0009DF8B40040F2A11110FB01F07E4901EB1C
:1038D000C00101F562719DF8A030BDF8D800184410
:1038E00000EB400303EB001001EBC0016031BDF8B9
:1038F000E40000E078E20A54BDF8E400401C81B224
:103900003991BDF8E4000228CBDBBDF84000801CF3
:1039100081B210919DF8B41001EB4100C0EBC110D1
:103920006B4901EBC001BDF84000085C01049DF843
:10393000B40000EB4002C2EBC010654A02EBC002CB
:10394000BDF84000401C105C41EA00219DF8B40025
:1039500000EB4002C2EBC0105D4A02EBC002BDF8B2
:103960004000801C105C01439DF8B40040F2A1129D
:1039700010FB02F0544A02EBC00202F562729DF89D
:10398000A030BDF8D800184400EB400303EB001052
:1039900002EBC0004167BDF84000C01C81B210912D
:1039A0004C4890F8E007E8BB0021399120E09DF8F1
:1039B000B41040F2A11011FB00F0434901EBC0012B
:1039C00001F562719DF8A020BDF8D800104400EB0D
:1039D000400202EB001001EBC0004730BDF8E410DC
:1039E000405C00B108E0BDF8E400401C81B23991B0
:1039F000BDF8E4000A28DADB00BFBDF8E4000A28BD
:103A00001BD140229DF8B40040F2A11110FB01F03F
:103A10002D4901EBC00101F562719DF8A030BDF8A0
:103A2000D80000E05AE0184400EB400303EB00101C
:103A300001EBC00080F87E2066E19DF8B41040F2F2
:103A4000A11011FB00F0204901EBC00101F56271EA
:103A50009DF8A020BDF8D800104400EB400202EB16
:103A6000001001EBC00090F87E00B8BB00212A9145
:103A700021E10021379137E09DF8B41040F2A11008
:103A800011FB00F0104901EBC00101F562719DF8D6
:103A9000A020BDF8D800104400EB400202EB00105B
:103AA00001EBC0014731BDF8DC00001D095C9DF849
:103AB000A80000EB4002084800EB4202BDF8DC0021
:103AC000105C81420BD013E0584500209840002044
:103AD000F8870020BC3200208834002014E1BDF8B3
:103AE000DC00401C81B23791BDF8DC000628C3DB46
:103AF00000BFBDF8DC0006287ED103229DF8B4008B
:103B000040F2A11110FB01F0FE4901EBC00101F5EB
:103B100062719DF8A030BDF8D800184400EB400356
:103B200003EB001001EBC00080F87E209DF8B4107C
:103B300001EB410000EB0110F34901EB00113031C2
:103B40009DF8A020BDF8D800104401EB0010801CA7
:103B50000990007820F00402099802700020399042
:103B60001FE020229DF8B40040F2A11110FB01F0EB
:103B7000E44901EBC00101F562719DF8A030BDF888
:103B8000D800184400EB400303EB001001EBC00128
:103B90005131BDF8E4000A54BDF8E400401C81B284
:103BA0003991BDF8E4000F28DBDB002139911FE0DB
:103BB00020229DF8B40040F2A11110FB01F0D14980
:103BC00001EBC00101F562719DF8A030BDF8D8008D
:103BD000184400EB400303EB001001EBC00163311C
:103BE000BDF8E4000A54BDF8E400401C81B23991EC
:103BF000BDF8E4000A2800E058E0D9DB00229DF877
:103C0000B40040F2A11110FB01F0BE4901EBC0016C
:103C100001F562719DF8A030BDF8D800184400EBA2
:103C2000400303EB001001EBC00080F87820002176
:103C300039911FE000229DF8B40040F2A11110FB61
:103C400001F0B04901EBC00101F562719DF8A030AF
:103C5000BDF8D800184400EB400303EB001001EB63
:103C6000C0017931BDF8E4000A54BDF8E400401CFD
:103C700081B23991BDF8E4000528DBDB9DF8B41072
:103C800040F2A11011FB00F09E4901EBC00101F5CB
:103C900062719DF8A020BDF8D800104400EB4002EE
:103CA00002EB001001EBC000406F0CE09DF8A80093
:103CB000401CC1B22A919548B0F8CA019DF8A810DD
:103CC00088423FF7D6AE00BF9048B0F8CA019DF8D1
:103CD000A810884218D140229DF8B40040F2A111EA
:103CE00010FB01F0874901EBC00101F562719DF8FD
:103CF000A030BDF8D800184400EB400303EB0010DF
:103D000001EBC00080F87E209DF8B41040F2A110B5
:103D100011FB00F07B4901EBC00101F562719DF8D8
:103D2000A020BDF8D800104400EB400202EB0010C8
:103D300001EBC00090F87E00032804D011281ED0AB
:103D4000402850D134E0F2229DF8B40040F2A11195
:103D500010FB01F06B4901EBC00101F562719DF8A8
:103D6000A030BDF8D800184400EB400303EB00106E
:103D700001EBC000427136E0F1E3F1E316E1F3221A
:103D80009DF8B40040F2A11110FB01F05D4901EB78
:103D9000C00101F562719DF8A030BDF8D80018444B
:103DA00000EB400303EB001001EBC00042711AE08E
:103DB000F2229DF8B40040F2A11110FB01F051492C
:103DC00001EBC00101F562719DF8A030BDF8D8008B
:103DD000184400EB400303EB001001EBC00000E0CF
:103DE000C5E0427100BF6AE09DF8B41001EB4100EC
:103DF00000EB0110444901EB001130319DF8A02087
:103E0000BDF8D800104401EB0010801C0990007828
:103E100020F00401099801709DF8B41040F2A1103F
:103E200011FB00F0374901EBC00101F562719DF80B
:103E3000A020BDF8D800104400EB400202EB0010B7
:103E400001EBC00090F8900000F00100B8B3002230
:103E50009DF8B40040F2A11110FB01F0294901EBDB
:103E6000C00101F562719DF8A03005E0FDE3FDE3BE
:103E7000ACE0FCE3FCE3FCE3BDF8D800184400EB45
:103E8000400303EB001001EBC000A0F88E200522D8
:103E90009DF8B40040F2A11110FB01F0194901EBAB
:103EA000C00101F562719DF8A030BDF8D80018443A
:103EB00000EB400303EB001001EBC00042716FE028
:103EC000FFE79DF8B41040F2A11011FB00F00D497E
:103ED00001EBC00101F562719DF8A020BDF8D8008A
:103EE000104400EB400202EB001001EBC00090F820
:103EF0007E00402821D100229DF8B40040F2A1119B
:103F000006E000005845002098400020BC32002008
:103F100010FB01F0FE4901EBC00101F562719DF853
:103F2000A030BDF8D800184400EB400303EB0010AC
:103F300001EBC00080F87E2000BF00BFF1229DF899
:103F4000B40040F2A11110FB01F0F14901EBC001F6
:103F500001F562719DF8A030BDF8D800184400EB5F
:103F6000400303EB001001EBC000427118E0F122A6
:103F70009DF8B40040F2A11110FB01F0E44901EBFF
:103F8000C00101F562719DF8A030BDF8D800184459
:103F900000EB400303EB001001EBC000427100BFD7
:103FA00000BFBDF8D800401C81B236919DF8B41016
:103FB00001EB4100C0EBC110D64901EBC0004179D3
:103FC000BDF8D80081423FF7EDAAF4E39DF8B410A4
:103FD00040F2A11011FB00F0CD4901EBC00000F54B
:103FE00062709DF8A01001EB410202EB011110F884
:103FF000310048BB01229DF8B40040F2A11110FB32
:1040000001F0C34901EBC00101F562719DF8A00008
:1040100000EB400303EB001001F83020F4229DF880
:10402000B40040F2A11110FB01F0B94901EBC0004E
:1040300000F562709DF8A01001EB410303EB011144
:1040400000EBC1004271CDE09DF8B41001EB4100DE
:1040500000EB0110B04901EB001030309DF8A010CA
:1040600000EB0110407A00F0010080B39DF8B4101D
:1040700040F2A11011FB00F0A54901EBC00000F5D2
:1040800062709DF8A01001EB410202EB011100EB00
:10409000C10090F8900000F00100C0B99DF8B41084
:1040A00040F2A11011FB00F0994901EBC00000F5AE
:1040B00062709DF8A01001EB410202EB011100EBD0
:1040C000C10090F8820010B1002139912DE089E003
:1040D0009DF8B41040F2A11011FB00F08C4901EBE7
:1040E000C00101F562719DF8A00000EB400202EBF7
:1040F000001001EBC00000F18301BDF8E4000A5C90
:104100009DF8B40000EB400101EB0010824901EB87
:1041100000100E30BDF8E410405C824200D008E090
:10412000BDF8E400401C81B23991BDF8E4000428D8
:10413000CEDB00BFBDF8E400042853D1042139913F
:104140002CE09DF8B41040F2A11011FB00F0704972
:1041500001EBC00101F562719DF8A00000EB400287
:1041600002EB001001EBC00000F18301BDF8E40098
:104170000A5C9DF8B40000EB400101EB00106649B9
:1041800001EB00110E31BDF8E400085C824200D062
:1041900008E0BDF8E400401C81B23991BDF8E400AC
:1041A0000A28CEDB00BFBDF8E4000A281AD09DF82B
:1041B000B41040F2A11011FB00F0554901EBC00012
:1041C00000F562709DF8A01001EB410202EB0111B5
:1041D00000EBC10090300990007820F00100401CF5
:1041E00009990870BDF8A400112877D19DF8B41082
:1041F00001EB410000EB0110474901EB00103030AA
:104200009DF8A01000EB0110801C0990007820F0B0
:104210000400001D099908700020399028E09DF8DD
:10422000B41001EB4100C0EBC1103A4901EBC001F1
:10423000BDF8E400401D0A5C9DF8B40040F2A111F5
:1042400010FB01F0324901EBC00101F562719DF8EC
:10425000A00000EB400303EB001001EBC00147316D
:10426000BDF8E4000A54BDF8E400401C81B2399165
:10427000BDF8E4000A28D2DB0021399128E09DF83E
:10428000B41001EB4100C0EBC110224901EBC001A9
:10429000BDF8E4000F300A5C9DF8B40040F2A111B3
:1042A00010FB01F01A4901EBC00101F562719DF8A4
:1042B000A00000EB400303EB001001EBC0016031F4
:1042C000BDF8E4000A54BDF8E400401C81B2399105
:1042D000BDF8E4000228D2DBB0E2FFE7BDF8A4009D
:1042E00014287DD19DF8B40000EB400101EB0010D3
:1042F000094901EB001030309DF8A01000EB0110CF
:10430000801C0990007820F00400001D099905E048
:1043100058450020F88700209840002008700020B1
:10432000399028E09DF8B40000EB4001C1EBC010CB
:10433000F84901EBC001BDF8E400401D0A5C9DF89E
:10434000B40040F2A11110FB01F0F34901EBC001F0
:1043500001F562719DF8A00000EB400303EB001033
:1043600001EBC0014731BDF8E4000A54BDF8E40098
:10437000401C81B23991BDF8E4000A28D2DB00214B
:10438000399128E09DF8B40000EB4001C1EBC0106A
:10439000E04901EBC001BDF8E4000F300A5C9DF874
:1043A000B40040F2A11110FB01F0DB4901EBC001A8
:1043B00001F562719DF8A00000EB400303EB0010D3
:1043C00001EBC0016031BDF8E4000A54BDF8E4001F
:1043D000401C81B23991BDF8E4000228D2DB00E034
:1043E0002DE29DF8B40000EB4001C1EBC010C949BB
:1043F00001EBC000407C01049DF8B40000EB4002DA
:10440000C2EBC010C34A02EBC000807C41EA00212D
:104410009DF8B40000EB4002C2EBC010BD4A02EBB5
:10442000C000C07C01439DF8B40040F2A11210FB13
:1044300002F0B94A02EBC00000F562709DF8A020BE
:1044400002EB420303EB021200EBC2004167B348E8
:1044500090F8E007F0BB002139911DE09DF8B40011
:1044600040F2A11110FB01F0AB4901EBC00101F5D5
:1044700062719DF8A00000EB400202EB001001EB1E
:10448000C0004730BDF8E410405C00B108E0BDF862
:10449000E400401C81B23991BDF8E4000A28DDDB5C
:1044A00000BFBDF8E4000A2818D140229DF8B400EE
:1044B00040F2A11110FB01F0974901EBC00000F59B
:1044C00062709DF8A01001EB410303EB011100EBBA
:1044D000C10000E045E080F87E2050E19DF8B40086
:1044E00040F2A11110FB01F08B4901EBC00000F577
:1044F00062709DF8A01001EB410202EB011100EB8C
:10450000C10090F87E0060BB00212A9111E10021DA
:1045100037912CE09DF8B40040F2A11110FB01F09E
:104520007D4901EBC00101F562719DF8A00000EB2F
:10453000400202EB001001EBC0014731BDF8DC0086
:10454000001D095C9DF8A80000EB4002744800EBD8
:104550004202BDF8DC00105C814203D00BE0FDE3B9
:10456000FDE30CE1BDF8DC00401C81B23791BDF8E1
:10457000DC000628CEDB00BFBDF8DC00062879D1C0
:1045800003229DF8B40040F2A11110FB01F0624932
:1045900001EBC00101F562719DF8A00000EB400342
:1045A00003EB001001EBC00080F87E209DF8B40002
:1045B00000EB400101EB00105A4901EB00113031D2
:1045C0009DF8A00001EB0010801C0990007820F0FD
:1045D000040209980270002039901CE020229DF806
:1045E000B40040F2A11110FB01F04B4901EBC001F6
:1045F00001F562719DF8A00000EB400303EB001091
:1046000001EBC0015131BDF8E4000A54BDF8E400EB
:10461000401C81B23991BDF8E4000F28DEDB002197
:1046200039911CE020229DF8B40040F2A11110FB4A
:1046300001F0394901EBC00101F562719DF8A0005C
:1046400000EB400303EB001001EBC0016331BDF848
:10465000E4000A54BDF8E400401C81B23991BDF871
:10466000E4000A28DEDB002205E0FCE3FCE3FCE3D7
:10467000FCE3E9E358E09DF8B40040F2A11110FB1F
:1046800001F0254901EBC00101F562719DF8A00020
:1046900000EB400303EB001001EBC00080F8782032
:1046A000002139911CE000229DF8B40040F2A111D4
:1046B00010FB01F0184901EBC00101F562719DF892
:1046C000A00000EB400303EB001001EBC0017931C7
:1046D000BDF8E4000A54BDF8E400401C81B23991F1
:1046E000BDF8E4000528DEDB9DF8B40040F2A1111E
:1046F00010FB01F0084901EBC00000F562709DF865
:10470000A01001EB410202EB011100EBC100406F70
:1047100017E00000F887002058450020BC32002038
:1047200088340020984000209DF8A800401CC1B2A9
:104730002A91FE48B0F8CA019DF8A81088423FF7B8
:10474000E6AE00BFF948B0F8CA019DF8A81088424B
:1047500015D140229DF8B40040F2A11110FB01F0E8
:10476000F34901EBC00000F562709DF8A01001EB69
:10477000410303EB011100EBC10080F87E209DF89E
:10478000B40040F2A11110FB01F0E94901EBC000B7
:1047900000F562709DF8A01001EB410202EB0111DF
:1047A00000EBC10090F87E00032805D0112819D035
:1047B000402843D12CE045E3F2229DF8B40040F2BA
:1047C000A11110FB01F0DA4901EBC00000F56270A5
:1047D0009DF8A01001EB410303EB011100EBC100B8
:1047E00042712BE0F3229DF8B40040F2A11110FBBE
:1047F00001F0CF4901EBC00000F562709DF8A010F8
:1048000001EB410303EB011100EBC100427115E024
:10481000F2229DF8B40040F2A11110FB01F0C4494E
:1048200001EBC00000F562709DF8A01001EB4103A0
:1048300003EB011100EBC100427100BF02E3BDF8C0
:10484000A40006287DD19DF8B40000EB4001C1EB27
:10485000C010B84901EBC0004079012872D1032093
:10486000B5490870F7229DF8B40040F2A11110FB81
:1048700001F0AF4901EBC00101F562719DF8A000A4
:1048800000EB400303EB001001EBC00042719DF808
:10489000B40040F2A11110FB01F0A54901EBC001E9
:1048A00001F562719DF8A00000EB400202EB0010E0
:1048B00001EBC00090F8800000EB400101EB00101C
:1048C0009E4901EB001130319DF8B40040F2A11275
:1048D00010FB02F0964A02EBC00000F562709DF8F2
:1048E000A02002EB420303EB021200EBC20090F89F
:1048F000810001EB00108078C0F34000F0B39DF818
:10490000B41040F2A11011FB00F0894901EBC00086
:1049100000F562709DF8A01001EB410202EB01115D
:1049200000EBC10090F8801001EB410000EB01109A
:10493000824901EB00108079012804D00A287CD13B
:104940003FE027E2CDE0BA239DF8B40040F2A11188
:1049500010FB01F0764901EBC00101F562719DF891
:10496000A00000EB400202EB001001EBC00090F849
:10497000800040F2A11110FB01F000E03AE16C4927
:1049800001EBC00101F562719DF8B40040F2A11283
:1049900010FB02F0664A02EBC00000F562709DF861
:1049A000A02002EB420404EB021200EBC20090F8DC
:1049B000810000EB400202EB001001EBC0004371EC
:1049C0003BE00B239DF8B40040F2A11110FB01F075
:1049D000574901EBC00101F562719DF8A00000EBA1
:1049E000400202EB001001EBC00090F8800040F2A2
:1049F000A11110FB01F04E4901EBC00101F56271FC
:104A00009DF8B40040F2A11210FB02F0484A02EBFC
:104A1000C00000F562709DF8A02002EB420404EB98
:104A2000021200EBC20090F8810000EB400202EBA2
:104A3000001001EBC000437100BF00BF9DF8B4102F
:104A400040F2A11011FB00F0394901EBC00101F562
:104A500062719DF8A00000EB400202EB001001EB38
:104A6000C00090F8801001EB410000EB01103349C9
:104A700001EB001130319DF8B40040F2A11210FB9F
:104A800002F02B4A02EBC00202F562729DF8A00010
:104A900000EB400303EB001002EBC00090F8810034
:104AA00001EB001002789DF8B40040F2A11110FB58
:104AB00001F01F4901EBC00000F562709DF8A010E5
:104AC00001EB410303EB011100EBC10090F8800002
:104AD00040F2A11110FB01F0154901EBC00042703A
:104AE000B0E19DF8B41001EB4100C0EBC1101149D9
:104AF00001EBC000407902287CD104200E490870E7
:104B0000F8229DF8B40040F2A11110FB01F0084911
:104B100001EBC00101F562719DF8A00000EB4003BC
:104B200003EB001001EBC000427109E0BC32002031
:104B300058450020F88700201902002098400020E6
:104B40009DF8B41040F2A11011FB00F0F94901EBFF
:104B5000C00101F562719DF8A00000EB400202EB7C
:104B6000001001EBC00090F8801001EB410000EB59
:104B70000110F14901EB001130319DF8B40040F211
:104B8000A11210FB02F0EB4A02EBC00000F56270CC
:104B90009DF8A02002EB420303EB021200EBC200DF
:104BA00090F8810001EB00108078C0F3400008B35A
:104BB0009DF8B41040F2A11011FB00F0DD4901EBAB
:104BC000C00000F562709DF8A01001EB410202EBFD
:104BD000011100EBC10090F8801001EB410000EBE7
:104BE0000110D54901EB00108079012803D00A2873
:104BF00079D13CE026E1B3239DF8B40040F2A11145
:104C000010FB01F0CB4901EBC00101F562719DF889
:104C1000A00000EB400202EB001001EBC00090F896
:104C2000800040F2A11110FB01F0C24901EBC0016C
:104C300001F562719DF8B40040F2A11210FB02F080
:104C4000BC4A02EBC00000F562709DF8A02002EBA8
:104C5000420404EB021200EBC20090F8810000EB6A
:104C6000400202EB001001EBC00043713BE00C235B
:104C70009DF8B40040F2A11110FB01F0AD4901EB29
:104C8000C00101F562719DF8A00000EB400202EB4B
:104C9000001001EBC00090F8800040F2A11110FB61
:104CA00001F0A44901EBC00101F562719DF8B40067
:104CB00040F2A11210FB02F09E4A02EBC00000F588
:104CC00062709DF8A02002EB420404EB021200EB9C
:104CD000C20090F8810000EB400202EB001001EBF3
:104CE000C000437100BF00BF9DF8B41040F2A11096
:104CF00011FB00F08F4901EBC00101F562719DF8D5
:104D0000A00000EB400202EB001001EBC00090F8A5
:104D1000801001EB410000EB0110874901EB00110D
:104D200030319DF8B40040F2A11210FB02F0814A2C
:104D300002EBC00202F562729DF8A00000EB400396
:104D400003EB001002EBC00090F8810001EB0010B3
:104D500002789DF8B40040F2A11101E08FE072E00A
:104D600010FB01F0734901EBC00000F562709DF883
:104D7000A01001EB410303EB011100EBC10090F81F
:104D8000800040F2A11110FB01F06A4901EBC00064
:104D9000427057E09DF8B41001EB410000EB0110A8
:104DA000654901EB001030309DF8A01000EB0110B8
:104DB000801C0990007820F00402099802709DF888
:104DC000B41040F2A11011FB00F05A4901EBC000F1
:104DD00000F562709DF8A01001EB410202EB011199
:104DE00000EBC10090F8900000F0010050B30022E9
:104DF0009DF8B40040F2A11110FB01F04D4901EB08
:104E0000C00101F562719DF8A00000EB400303EBC7
:104E1000001001EBC000A0F88E2005229DF8B40020
:104E200040F2A11110FB01F0424901EBC00000F576
:104E300062709DF8A01001EB410303EB011100EB40
:104E4000C100427193E100BFF1229DF8B40040F22D
:104E5000A11110FB01F0374901EBC00000F56270B1
:104E60009DF8A01003E04FE005E191E066E001EB62
:104E7000410303EB011100EBC100427177E19DF8A2
:104E8000B41040F2A11011FB00F02A4901EBC00060
:104E900000F562709DF8A01001EB410202EB0111D8
:104EA00000EBC10090F87E00402816D100229DF84A
:104EB000B40040F2A11110FB01F01E4901EBC0004B
:104EC00000F562709DF8A01001EB410303EB0111A6
:104ED00000EBC10080F87E2000BF00BFF1229DF8EA
:104EE000B40040F2A11110FB01F0124901EBC00027
:104EF00000F562709DF8A01001EB410303EB011176
:104F000000EBC100427132E1F1229DF8B40040F2A1
:104F1000A11110FB01F0074901EBC00000F5627020
:104F20009DF8A01001EB410303EB011100EBC10060
:104F300042711CE1584500209840002003229DF852
:104F4000B40040F2A11110FB01F0FE4901EBC001D9
:104F500001F562719DF8A00000EB400303EB001027
:104F600001F83020F1229DF8B40040F2A11110FBAD
:104F700001F0F44901EBC00000F562709DF8A0104B
:104F800001EB410303EB011100EBC1004271EEE0C4
:104F900002229DF8B40040F2A11110FB01F0E94992
:104FA00001EBC00101F562719DF8A00000EB400328
:104FB00003EB001001F83020F6229DF8B40040F217
:104FC000A11110FB01F0DF4901EBC00101F5627195
:104FD0009DF8A00000EB400303EB001001EBC000C4
:104FE000427101229DF8B40040F2A11110FB01F0C2
:104FF000D44901EBC00101F562719DF8A00000EBFE
:10500000400303EB001001EBC00080F88220002178
:10501000399129E09DF8B41001EB4100C0EBC110BB
:10502000C94901EBC001BDF8E400401D0A5C9DF8D0
:10503000B40040F2A11110FB01F0C24901EBC00124
:1050400001F562719DF8A00000EB400303EB001036
:1050500001EBC00000F18301BDF8E4000A54BDF883
:10506000E400401C81B23991BDF8E4000A28D1DB8C
:10507000BDF8A4007BE09DF8B41001EB4100C0EB4B
:10508000C110B14901EBC00081799DF8B40000EB7B
:105090004002C2EBC010AC4A02EBC000407941EACA
:1050A00000229DF8B40040F2A11110FB01F0A549C7
:1050B00001EBC00101F562719DF8A00000EB400317
:1050C00003EB001001EBC000A0F88E209DF8B41097
:1050D00040F2A11011FB00F09A4901EBC00101F56B
:1050E00062719DF8A00000EB400202EB001001EBA2
:1050F000C000B0F88E109DF8B40000EB400202EB47
:105100000010924A02EB0010408B81422EDBF1220C
:105110009DF8B40040F2A11110FB01F0894901EBA8
:10512000C00101F562719DF8A00000EB400303EBA4
:10513000001001EBC00042719DF8B40040F2A111D3
:1051400010FB01F07F4901EBC00101F562719DF890
:10515000A00000EB400202EB001001EBC000903019
:105160000990007820F001020998027000BF00BF8A
:1051700009F010B89DF8B40000EB4001C1EBC0107D
:10518000714901EBC00001792891002136911CE0A2
:105190009DF8B40000EB400101EB00106B4901EBFE
:1051A00000113031BDF8D80001EB001041789DF8B6
:1051B000A000814204D1BDF8D800C1B2289112E00C
:1051C000BDF8D800401C81B236919DF8B40000EBC8
:1051D000400101EB00105D4901EB0010C179BDF801
:1051E000D8008142D4DC00BF9DF8B40000EB400140
:1051F000C1EBC010544901EBC000C1782591BDF846
:105200009400172834D2DFE800F0330C0F33121566
:10521000181B1E33333333333321242733332A2DE2
:1052200030000721299123E00721299120E0062160
:1052300029911DE0062129911AE00621299117E004
:105240001220299014E00721299111E009212991C8
:105250000EE0062129910BE00621299108E00B219F
:10526000299105E00B21299102E02A21299100BF13
:1052700000BFBDF8A400001FC1B209919DF8B400A1
:1052800000EB4001C1EBC0102F4901EBC000C01C76
:1052900008900999F4F71EF937909DF8B40000EBD7
:1052A0004001C1EBC010284901EBC001BDF8A400CA
:1052B000401E095CBDF8DC00814270D19DF8B4004D
:1052C00000EB4001C1EBC0101F4901EBC00040786A
:1052D000002864DD9DF8B40000EB4001C1EBC01074
:1052E000194901EBC001BDF8A4000A5C9DF8B400A7
:1052F00040F2A11110FB01F0124901EBC00101F5D0
:1053000062719DF8A00000EB400303EB001001EB7D
:10531000C00080F8442000210D4A9DF8B40002EB43
:1053200000129DF8A00011540A4890F828000128A6
:1053300021D19DF8B40000EB400101EB00100349BE
:105340000AE0000058450020F8870020984000201F
:10535000883E0020BC12002001EB001030309DF888
:10536000A01000EB0110801C0990007820F0800054
:10537000803009990870BDF8940007287ED00ADCB7
:1053800007287CD2DFE810F07B006806CA067B00A5
:1053900052061506CE0C10380728F2D200E0FCE3C6
:1053A000DFE810F02E0D180D6D006D0007000800ED
:1053B000F30600BFBDF8940014287DD19DF8B40019
:1053C00000EB4001C1EBC010FE4901EBC000407989
:1053D00001069DF8B40000EB4002C2EBC010F94A90
:1053E00002EBC000807941EA00419DF8B40000EB77
:1053F0004002C2EBC010F34A02EBC000C07941EAA0
:1054000000219DF8B40000EB4002C2EBC010ED4A51
:1054100002EBC000007A01439DF8B40040F2A112F3
:1054200010FB02F0E84A02EBC00202F562729DF83E
:10543000A00000EB400303EB001002EBC000C0F83B
:105440001A109DF8B40040F2A11110FB01F0DE49E2
:1054500001EBC00101F562719DF8A00000EB400274
:1054600002EB001001EBC000D0F81A1008460991B9
:10547000002111F0CDFBCDE92E0101E0F1E3F1E3D4
:105480009DF8B40000EB400101EB0010CF4901EBA7
:105490000010007F00F003019DF8B40000EB400213
:1054A00002EB0010C94A02EB0010007FC0F30110AC
:1054B00001449DF8B40000E06FE000EB400202EB15
:1054C0000010C24A02EB0010007FC0F38100091AED
:1054D00008460591F3F78BF8CDE906019DED061B13
:1054E0009FEDBB0B20F05CFB8DED080B9DED080BD9
:1054F00051EC100BF3F7EDF8CDE930019DF8B40055
:1055000040F2A11110FB01F0AF4901EBC00101F520
:1055100062719DF8A00000EB400202EB001001EB6D
:10552000C000416B08460791002111F071FBDDE9D5
:105530002E32A0FB034501FB035100FB02150222A2
:105540000023DDE93001F2F73DFE231845EB0100B1
:10555000CDE90830DDE93023DDE90801F2F732FE5C
:10556000CDE92E01DDE92E0112F006F901469DF884
:10557000B40040F2A11210FB02F0934A02EBC0000B
:1055800000F562709DF8A02002EB420303EB0212CB
:1055900000EBC200C0F81E1046E0BDF894001528CC
:1055A00042D19DF8B40000EB4001C1EBC010854929
:1055B00001EBC000407901069DF8B40000EB400209
:1055C000C2EBC0107F4A02EBC000807941EA004183
:1055D0009DF8B40000EB4002C2EBC010794A02EB28
:1055E000C000C07941EA00219DF8B40000EB400200
:1055F000C2EBC010734A02EBC000007A01439DF871
:10560000B40040F2A11210FB02F06F4A02EBC0009E
:1056100000F562709DF8A02002EB420303EB02123A
:1056200000EBC200C0F81E109DF8B40000EB400172
:10563000C1EBC010634901EBC000427A9DF8B40091
:1056400040F2A11110FB01F05F4901EBC00101F52F
:1056500062719DF8A00000EB400303EB001001EB2A
:10566000C00080F894209DF8B40000EB400101EBED
:105670000010564901EB001130319DF8A00001EBFC
:105680000010801C09909DF8B40040F2A11110FB9D
:1056900001F24D4800EBC20000F562709DF8A010C9
:1056A00001EB410202EB011100EBC10090F8940004
:1056B000C2090998007862F30000099908709DF802
:1056C000B40040F2A11110FB01F03F4901EBC00012
:1056D00000F562709DF8A01001EB410202EB011190
:1056E00000EBC10090F8940000F00300012818D0EE
:1056F0009DF8B40040F2A11110FB01F0324901EB1A
:10570000C00000F562709DF8A01001EB410202EBB1
:10571000011100EBC10090F8940000F00300032891
:105720002BD19DF8B40000EB400101EB001027499C
:1057300001EB001030309DF8A01000EB0110801C30
:105740000990007820F00200801C099908709DF8EB
:10575000B40000EB400101EB00101C4901EB00100C
:1057600030309DF8A01000EB0110801C09900078EB
:1057700020F020020998027014E09DF8B40000EBBC
:10578000400101EB0010114901EB001030309DF891
:10579000A01000EB0110801C0990007820F002029C
:1057A000099802709DF8B40000EB400101EB001075
:1057B000064901EB001130319DF8A00001EB00100B
:1057C000807809E0F88700205845002098400020A4
:1057D0000000000000002440C0F340029DF8B40027
:1057E00040F2A11110FB01F0FE4901EBC00000F5F1
:1057F00062709DF8A01001EB410303EB011100EB77
:10580000C100007EC0F3400082426CD09DF8B4001D
:1058100040F2A11110FB01F0F24901EBC00000F5CC
:1058200062709DF8A01001EB410202EB011100EB48
:10583000C100183009909DF8B40000EB400101EB65
:105840000010E94901EB001030309DF8A01000EB8A
:105850000110807842080998007862F341000999A4
:1058600008709DF8B40000EB400101EB0010DE4928
:1058700001EB001030309DF8A01000EB0110807893
:10588000C0F3400050BB9DF8B40000EB400101EBB9
:105890000010D54901EB001030309DF8A01000EB4E
:1058A0000110801C0990007820F0200209980270F5
:1058B00001229DF8B40040F2A11110FB01F0C9498A
:1058C00001EBC00000F562709DF8A01001EB4103F0
:1058D00003EB011100EBC10080F846209DF8B410E5
:1058E0000220F4F7E3FB9DF8B40000EB400101EB6C
:1058F0000010BD4901EB001130319DF8A00001EB13
:105900000010807800F001029DF8B40040F2A1116F
:1059100010FB01F0B34901EBC00000F562709DF887
:10592000A01001EB410303EB011100EBC100007E6D
:1059300000F00100824265D09DF8B40040F2A11150
:1059400010FB01F0A74901EBC00000F562709DF863
:10595000A01001EB410202EB011100EBC100183075
:1059600009909DF8B40000EB400101EB00109E4946
:1059700001EB001030309DF8A01000EB0110817891
:105980000998027861F3000202709DF8B40000EB00
:10599000400101EB0010944901EB001030309DF8FC
:1059A000A01000EB0110807800F0010058BB9DF8BA
:1059B000B40000EB400101EB00108B4901EB00103B
:1059C00030309DF8A01000EB0110801C0990007889
:1059D00020F020020998027000229DF8B40040F2E5
:1059E000A11110FB01F07F4901EBC00000F56270CE
:1059F0009DF8A01001EB410303EB011100EBC10086
:105A000080F8452014E29DF8B40040F2A11110FB8B
:105A100001F0744901EBC00000F562709DF8A01020
:105A200001EB410202EB011100EBC10090F84600CE
:105A3000B0B901229DF8B40040F2A11110FB01F0B1
:105A4000684901EBC00000F562709DF8A01001EB01
:105A5000410303EB011100EBC10080F845202AE06F
:105A600000229DF8B40040F2A11110FB01F05D4945
:105A700001EBC00101F562719DF8A00000EB40034D
:105A800003EB001001EBC00080F845209DF8B40046
:105A900000EB400101EB0010534901EB00113031E4
:105AA0009DF8A00001EB0010801C0990007820F008
:105AB0000102099802704D4890F8E00780B19DF806
:105AC000B40000EB400101EB0010474901EB00106E
:105AD00030309DF8A01000EB0110807A022876D1BA
:105AE000434890F82900012872D14148D0F80C02AF
:105AF0003F49498D88426BD29DF8B40040F2A11114
:105B000010FB01F0374901EBC00000F562709DF811
:105B1000A01001EB410202EB011100EBC10090F873
:105B20004500012853D19DF8B40040F2A11110FBAB
:105B300001F02C4901EBC00000F562709DF8A01047
:105B400001EB410202EB011100EBC10090F87F0074
:105B5000E8BB01229DF8B40000EB400101EB00100E
:105B6000214901EB001130319DF8A00001EB00103C
:105B7000C2729DF8B40000EB400101EB00101A491D
:105B800001EB001130319DF8A00001EB001001780D
:105B90009DF8B40040F2A11200E0FCE310FB02F01B
:105BA000104A02EBC000417005229DF8B40040F29B
:105BB000A11110FB01F00B4901EBC00101F562716D
:105BC0009DF8A00000EB400303EB001001E001E1B1
:105BD0006BE001EBC000427100229DF8B40000EBC5
:105BE000400107E05845002098400020BC320020CA
:105BF000BC12002001EB0010FE4901EB0011303116
:105C00009DF8A00001EB001042609DF8B410022046
:105C1000F4F74CFA002139911CE000229DF8B40001
:105C200040F2A11110FB01F0F34901EBC00101F5B5
:105C300062719DF8A00000EB400303EB001001EB44
:105C4000C0014731BDF8E4000A54BDF8E400401C2F
:105C500081B23991BDF8E4001428DEDB00203990D0
:105C60001EE06DE359E200229DF8B40040F2A1115C
:105C700010FB01F0E04901EBC00101F562719DF8F4
:105C8000A00000EB400303EB001001EBC001633107
:105C9000BDF8E4000A54BDF8E400401C81B239911B
:105CA000BDF8E4000A28DEDBC2E09DF8B40040F253
:105CB000A11110FB01F0D04901EBC00000F56270AA
:105CC0009DF8A01001EB410202EB011100EBC100B5
:105CD00090F8450001287DD19DF8B40040F2A11153
:105CE00010FB01F0C44901EBC00101F562719DF8A0
:105CF000A00000EB400202EB001001EBC00090F8A6
:105D0000800040F2A11110FB01F0BB4901EBC00182
:105D100001F562719DF8B40040F2A11210FB02F08F
:105D2000B54A02EBC00000F562709DF8A02002EBBE
:105D3000420303EB021200EBC20090F8810000EB7B
:105D4000400202EB001001EBC00090F87E00032837
:105D50006ED102229DF8B40000EB400101EB00106F
:105D6000A44901EB001130319DF8A00001EB0010B7
:105D7000C2729DF8B40000EB400101EB00109D4998
:105D800001EB001130319DF8A00001EB001001780B
:105D90009DF8B40040F2A11210FB02F0964A02EB0B
:105DA000C00041709DF8B40040F2A11110FB01F059
:105DB000114601EBC00101F562719DF8A00000EBF6
:105DC000400202EB001011F830109DF8B40040F2D0
:105DD000A11200E02CE010FB02F0874A02EBC000A9
:105DE0004079814214D105229DF8B40040F2A111FE
:105DF00010FB01F0804901EBC00000F562709DF8D6
:105E0000A01001EB410303EB011100EBC100427153
:105E100000229DF8B40000EB400101EB0010754931
:105E200001EB001030309DF8A01000EB0110426033
:105E30009DF8B40040F2A11110FB01F06E4901EB96
:105E4000C00000F562709DF8A01001EB410202EB6A
:105E5000011110F83100012814DC02229DF8B40071
:105E600040F2A11110FB01F0634901EBC00000F505
:105E700062709DF8A01001EB410303EB011100F8E3
:105E8000312095E09DF8B40040F2A11110FB01F023
:105E9000594901EBC00000F562709DF8A01001EBBC
:105EA000410202EB011110F83100022834DC00211C
:105EB0009DF8B40040F2A11210FB02F04E4A02EB32
:105EC000C000017103229DF8B40040F2A11110FB43
:105ED00001F0494901EBC00101F562719DF8A00094
:105EE00000EB400303EB001001F8302007229DF87F
:105EF000B40040F2A11110FB01F03F4901EBC000DA
:105F000000F562709DF8A01001EB410303EB011155
:105F100000EBC10042714BE09DF8B40040F2A111CA
:105F200010FB01F0344901EBC00101F562719DF8ED
:105F3000A00000EB400202EB001011F830109DF8B9
:105F4000B40040F2A11210FB02F02B4A02EBC00099
:105F5000407981422CD19DF8B40040F2A11110FB90
:105F600001F0114601EBC00000F562709DF8A01031
:105F700001EB410202EB011100EBC10090F894002B
:105F8000C0F34010A0B116229DF8B40040F2A11158
:105F900010FB01F0184901EBC00000F562709DF89C
:105FA000A01001EB410303EB011100EBC1004271B2
:105FB000B3E014229DF8B40040F2A11110FB01F0EF
:105FC0000D4901EBC00101F562719DF8A00000EBE5
:105FD000400303EB001001EBC000427101219DF86A
:105FE000B40040F2A11210FB02F0034A02EBC00021
:105FF000017103E098400020584500209DF8B4004E
:1060000000EB400101EB0010A2F5986101EB0011DB
:1060100030319DF8A00001EB0010801C0990007841
:1060200020F0200020300999087076E014229DF8B5
:10603000B40040F2A11110FB01F0FE4901EBC000D9
:1060400000F562709DF8A01001EB410303EB011114
:1060500000EBC100427160E09DF8B40040F2A11174
:1060600010FB01F0F34901EBC00000F56270BDF8D0
:10607000D81001EB410202EB011100EBC100807965
:1060800001282AD100229DF8B40040F2A11110FB92
:1060900001F0E84901EBC00101F56271BDF8D800DB
:1060A00000EB400303EB001001EBC00082711422EF
:1060B0009DF8B40040F2A11110FB01F0DD4901EBA5
:1060C000C00000F562709DF8A01001EB410303EBE6
:1060D000011100EBC10042711FE000219DF8B400E6
:1060E00040F2A11210FB02F0D24A02EBC000017193
:1060F00005229DF8B40040F2A11110FB01F0CD493A
:1061000001EBC00000F562709DF8A01001EB4103A7
:1061100003EB011100EBC1004271FDE301219DF889
:10612000B40040F2A11210FB02F0C24A02EBC00020
:10613000017114229DF8B40040F2A11110FB01F08E
:10614000BC4901EBC00101F562719DF8A00000EBB4
:10615000400303EB001001EBC00042719DF8B40056
:1061600000EB400101EB0010B34901EB00113031AD
:106170009DF8A00001EB0010801C0990007820F031
:106180000400001D09990870C6E300202E902F908E
:10619000002139911EE0DDE92E10000240EA116273
:1061A0000902CDE92E129DF8B40000EB4001C1EBCD
:1061B000C010A24901EBC001BDF8E400401D085C1D
:1061C000DDE92E341843CDE92E04BDF8E400401C6F
:1061D00080B23990BDF8E4000328DCDBDDE92E0154
:1061E00011F0CAFA01469DF8B40040F2A11210FB6A
:1061F00002F0904A02EBC00202F562729DF8A00024
:1062000000EB400303EB001002EBC000C0F81E10CF
:1062100000222E922F92002139911FE0DDE92E10ED
:10622000000240EA11620902CDE92E129DF8B40085
:1062300000EB4001C1EBC010804901EBC001BDF88B
:10624000E4000830085CDDE92E3440EA0302CDE9C1
:106250002E24BDF8E400401C81B23991BDF8E40061
:106260000328DBDBDDE92E0111F086FA01469DF8FB
:10627000B40040F2A11210FB02F06E4A02EBC00221
:1062800002F562729DF8A00000EB400303EB0010E2
:1062900002EBC000C0F81A1000222E922F920021AB
:1062A00039911EE0DDE92E10000240EA1162090278
:1062B000CDE92E129DF8B40000EB4001C1EBC010F7
:1062C0005E4901EBC001BDF8E4001330085CDDE974
:1062D0002E341843CDE92E04BDF8E400401C80B2F2
:1062E0003990BDF8E4000328DCDB9DF8B4002E995A
:1062F00040F2A11210FB02F04E4A02EBC00202F57E
:1063000062729DF8A00000EB400303EB001002EB6B
:10631000C000416307229DF8B40040F2A11110FBB8
:1063200001F0444901EBC00000F562709DF8A01037
:1063300001EB410303EB011100EBC1004271EBE201
:1063400000202E902F90002139911FE0DDE92E10C2
:10635000000240EA11620902CDE92E129DF8B40054
:1063600000EB4001C1EBC010344901EBC001BDF8A6
:10637000E400401D085CDDE92E3440EA0302CDE96B
:106380002E24BDF8E400401C81B23991BDF8E40030
:106390000428DBDB00E0FCE3DDE92E0111F0ECF981
:1063A0009DF8B42040F2A11312FB03F2214B03EB42
:1063B000C20303F562739DF8A02002EB420404EBD4
:1063C000021203EBC20222329060D16000212E91B2
:1063D0002F91002039901EE0DDE92E10000240EAE6
:1063E00011620902CDE92E129DF8B40000EB4001C4
:1063F000C1EBC010114901EBC001BDF8E400093048
:10640000085CDDE92E341843CDE92E04BDF8E40024
:10641000401C80B23990BDF8E4000428DCDBDDE9E3
:106420002E0111F0A9F99DF8B42040F2A11312FB3E
:1064300003F205E05845002098400020F88700202E
:10644000FE4B03EBC20303F562739DF8A02002EB41
:10645000420404EB021203EBC20242F8220F516025
:106460009DF8B40040F2A11110FB01F0F34901EBDB
:10647000C00000F562709DF8A01001EB410202EB34
:10648000011110F831009DF8B41040F2A11211FB77
:1064900002F1EA4A02EBC101497988427ED19DF8B6
:1064A000B40040F2A11110FB01F0114601EBC00055
:1064B00000F562709DF8A01001EB410202EB0111A2
:1064C00000EBC10090F89400C0F34010A8B117226F
:1064D0009DF8B40040F2A11110FB01F0D74901EB87
:1064E000C00000F562709DF8A01001EB410303EBC2
:1064F000011100EBC100427114E014229DF8B400B8
:1065000040F2A11110FB01F0CC4901EBC00000F5F5
:1065100062709DF8A01001EB410303EB011100EB49
:10652000C10042719DF8B4009DF8A01001EB00106D
:10653000C217CDE92E02C24890F8E00708B39DF8D3
:10654000B40000EB400101EB0010BE4901EB00106C
:1065500030309DF8A01000EB0110807A022810D096
:106560009DF8B40000EB400101EB0010B54901EBD0
:10657000001030309DF8A01000EB0110C07A002808
:106580007EDD00229DF8B40040F2A11110FB01F065
:10659000AA4901EBC00101F5627100E02DE39DF80D
:1065A000A00000EB400303EB001001EBC00080F8FB
:1065B00046209DF8B40000EB400101EB0010A1491A
:1065C00001EB001130319DF8A00001EB0010C27208
:1065D0009D48D0F80C020521B0FBF1F201FB12003E
:1065E00000EB400198482C3000EB41100D30099031
:1065F0009DF8B41040F2A11011FB00F08F4901EB9F
:10660000C00000F562709DF8A01001EB410202EBA2
:10661000011100EBC10022301022014608900998B8
:10662000F1F713FE8848D0F80C020521B0FBF1F217
:1066300001FB120000EB400183482C3000EB4112BB
:106640009DF8B40040F2A11110FB01F07B4901EB71
:10665000C00101F562719DF8A00000EB400303EB5F
:10666000001001EBC00050F81A1F42F8011F4068EB
:1066700050607548D0F80C020521B0FBF1F200E043
:10668000A8E101FB120000EB40016F482C3000EB49
:1066900041129DF8B40000EB400101EB0010694984
:1066A00001EB001130319DF8A00001EB00100078E3
:1066B00010706548D0F80C020521B0FBF1F201FB27
:1066C000120000EB400160482C3000EB41129DF8B5
:1066D000B40040F2A11110FB01F0584901EBC001D8
:1066E00001F562719DF8A00000EB400303EB001080
:1066F00001EBC000406BC2F809005348D0F80C020F
:106700000521B0FBF1F201FB120000EB40014E4805
:106710002C3000EB41114A48F538026841F81D2F32
:10672000808888804848D0F80C020521B0FBF1F23F
:1067300001FB120000EB400143482C3000EB4112FA
:106740009DF8B40000EB400101EB00103D4901EB66
:10675000001130319DF8A00001EB00104068C2F834
:10676000230000229DF8B40000EB400101EB001073
:10677000344901EB001130319DF8A00001EB00100D
:1067800042600021399154E02F48D0F80C020521D5
:10679000B0FBF1F201FB120000EB40012A482C3063
:1067A00000EB41112731BDF8E4409DF8B40040F200
:1067B000A11210FB02F0214A02EBC00202F5627244
:1067C0009DF8A00000EB400303EB001002EBC000BB
:1067D00090F8800040F2A11210FB02F0174A02EB81
:1067E000C00202F562729DF8B40040F2A11310FBE2
:1067F00003F0124B03EBC00303F562739DF8A00096
:1068000000EB400505EB001003EBC00090F88100A1
:1068100000EB400303EB001002EBC0024732BDF86F
:10682000E400001D105C0855BDF8E400401C81B276
:106830003991BDF8E4000628A6DB07E058450020A2
:10684000BC32002098400020BC120020002039906B
:1068500042E000239DF8B40040F2A11110FB01F0CA
:10686000FE4901EBC00101F562719DF8A00000EB4B
:10687000400202EB001001EBC00090F8800040F2F3
:10688000A11110FB01F0F54901EBC00101F56271A6
:106890009DF8B40040F2A11210FB02F0EF4A02EBA7
:1068A000C00202F562729DF8A00000EB400404EB08
:1068B000001002EBC00090F8810000EB400202EBF8
:1068C000001001EBC0014731BDF8E4000B54BDF8E6
:1068D000E400401C81B23991BDF8E4000A28B8DB1D
:1068E000DF48D0F80C020521B0FBF1F080B2014680
:1068F00009900220F2F7ECFB00210620F3F7D6FB0B
:10690000D748D0F80C02D649498D884208D2D448DD
:10691000D0F80C02401C00E003E2D149C1F80C029F
:1069200000210520F3F7C2FB9DF8B40000EB400105
:1069300001EB0010CB4901EB001030309DF8A010A6
:1069400000EB0110801C0990007820F008020998E3
:106950000270C348D0F80C020521B0FBF1F201FB34
:10696000120000EB4001BE482C3000EB4110D0F883
:1069700023202E9800EB4001BB4800EB4110C0F8EB
:1069800023200020399020E0B548D0F80C020521E2
:10699000B0FBF1F201FB120000EB4001B0482C30DB
:1069A00000EB41102730BDF8E410425C2E9800EB5C
:1069B0004001AD4800EB41112731BDF8E4000A5415
:1069C000BDF8E400401C81B23991BDF8E40006280E
:1069D000DADB6FE000229DF8B40040F2A11110FB59
:1069E00001F09E4901EBC00101F562719DF8A00024
:1069F00000EB400303EB001001EBC00080F84620E1
:106A00009DF8B40000EB400101EB0010954901EB4B
:106A1000001130319DF8A00001EB0010801C09909E
:106A2000007820F008000830099908709DF8B4003B
:106A300000EB400101EB00108A4901EB00103030FF
:106A40009DF8A01000EB011042682E9800EB400169
:106A5000854800EB4110C0F823200020399025E044
:106A60009DF8B40040F2A11110FB01F07B4901EB4D
:106A7000C00101F562719DF8A00000EB400202EB3D
:106A8000001001EBC0014731BDF8E4000A5C2E980C
:106A900000EB4001744800EB41112731BDF8E400E0
:106AA0000A54BDF8E400401C81B23991BDF8E400FD
:106AB0000628D5DB9DF8B4100220F3F7F7FA9DF80D
:106AC000B40040F2A11110FB01F0644901EBC000D9
:106AD00000F562709DF8A01001EB410202EB01117C
:106AE00000EBC100223009902E9800EB40015E4877
:106AF00000EB41100D30102208900999F1F7A5FB29
:106B00009DF8B40040F2A11110FB01F0534901EBD4
:106B1000C00101F562719DF8A00000EB400202EB9C
:106B2000001001EBC0012E9800EB40024E4800EB34
:106B3000421051F81A2F40F8012F496841609DF822
:106B4000B40000EB400101EB0010464901EB0011DD
:106B500030319DF8A00001EB001001782E9800EB79
:106B60004002414800EB421001702E9800EB4001BA
:106B70003D4800EB41113D48026841F81D2F8088D7
:106B800088809DF8B40040F2A11110FB01F0334958
:106B900000E04CE101EBC00101F562719DF8A0003D
:106BA00000EB400202EB001001EBC000416B2E989D
:106BB00000EB40022C4800EB4210C0F809109DF891
:106BC000B40000EB400101EB0010264901EB00117D
:106BD00030319DF8A00001EB001041682E9800EBC9
:106BE0004002214800EB4210C0F823102E9881B2D9
:106BF00008200991F3F75AFA93E09DF8B40040F2A7
:106C0000A11110FB01F0154901EBC00101F5627102
:106C10009DF8A00000EB400202EB001011F83010CC
:106C20009DF8B40040F2A11210FB02F00B4A02EBF7
:106C3000C0004079814274DA9DF8B40000EB400155
:106C400001EB0010074901EB001030309DF8A01057
:106C500000EB0110801C0990007809E058450020E5
:106C6000BC12002098400020D8140020C73100201A
:106C700020F00400001D099908709DF8B40000EB95
:106C8000400101EB0010A2F5986101EB00103030DB
:106C90009DF8A01000EB0110801C0990007820F0F6
:106CA000800080300999087001209DF8B41040F2EE
:106CB000A11211FB02F1FE4A02EBC10108719DF81D
:106CC000B40040F2A11110FB01F0114601EBC0002D
:106CD00042799DF8B40040F2A11110FB01F0F44993
:106CE00001EBC00000F562709DF8A01001EB4103BC
:106CF00003EB011100F8312014229DF8B40040F29A
:106D0000A11110FB01F0EA4901EBC00000F562702F
:106D10009DF8A01001EB410303EB011100EBC10052
:106D2000427183E00121E34880F804179DF8B40024
:106D300040F2A11110FB01F0DD4901EBC00101F5AA
:106D400062719DF8A00000EB400202EB001011F808
:106D500030109DF8B40040F2A11210FB02F0D44AAA
:106D600002EBC0004079814233DA00219DF8B40083
:106D700040F2A11210FB02F0CD4A02EBC0000171FB
:106D800001229DF8B40040F2A11110FB01F0C849A6
:106D900001EBC00101F562719DF8A00000EB40031A
:106DA00003EB001001F8302014229DF8B40040F2EB
:106DB000A11110FB01F0BE4901EBC00000F56270AB
:106DC0009DF8A01001EB410303EB011100EBC100A2
:106DD00042712BE014229DF8B40040F2A11110FB87
:106DE00001F0B34901EBC00101F562719DF8A0000B
:106DF00000EB400303EB001001EBC000427115E013
:106E000014229DF8B40040F2A11110FB01F0A84932
:106E100001EBC00000F562709DF8A01001EB41038A
:106E200003EB011100EBC100427100BF00BF07F08E
:106E3000B1B99DF8B40040F2A11110FB01F09C49DA
:106E400001EBC000817828919DF8B40000EB40016F
:106E5000C1EBC010984911F8301029919DF8B40089
:106E600040F2A11110FB01F0914901EBC00101F5C5
:106E700062719DF8A00000EB400202EB001001EBF4
:106E8000C000417925919DF8B40000EB4001C1EBB1
:106E9000C010894901EBC0010991BDF8A4100998FF
:106EA000F3F79CFE37909DF8B40000EB4001C1EB76
:106EB000C010814901EBC001BDF8A400095CBDF818
:106EC000DC00814241F067879DF8B40000EB40018F
:106ED000C1EBC010784901EBC0004078002841F3B5
:106EE0005A870021754A9DF8B40002EB00129DF804
:106EF000A0001154BDF8940089287DD00EDC142820
:106F000001F0298705DC082877D0102841F0428756
:106F1000FDE3152872D08028F8D1FAE38B286ED0D3
:106F20008C286DD08E286CD08F28EFD1BDF8A400AE
:106F30000D2867D19DF8B40000EB4001C1EBC010F3
:106F40005D4901EBC00041785D4880F8041D9DF863
:106F5000B40000EB4001C1EBC010574901EBC00089
:106F6000C17A574880F8051D9DF8B40040F2A11180
:106F700010FB01F04E4901EBC00000F562709DF876
:106F8000A01001EB410202EB011110F831000328BF
:106F90007EDC4B4890F8050D00287ADD9DF8B400A2
:106FA00040F2A11110FB01F0414901EBC00101F5D4
:106FB00062719DF8A00000EB400202EB001001EBB3
:106FC000C00109910878401CC1B2099801709DF870
:106FD000B40040F2A11110FB01F0354901EBC000F3
:106FE00000F562709DF8A01001EB410202EB011167
:106FF00010F83100042806E0FEE3FEE3FEE3FEE3C2
:10700000FEE3FEE3FEE344DB9DF8B40000EB400149
:1070100001EB00102B4901EB001030309DF8A0105F
:1070200000EB0110801C0990254890F8050DC0F375
:107030000010C0F101000999097860F30001099876
:1070400001701F4890F8040DC0F3C00078BB9DF894
:10705000B40000EB400101EB00101A4901EB0010F5
:1070600030309DF8A01000EB01108078C0F3401084
:10707000E8B19DF8B40000EB400101EB00101149AC
:1070800001EB001030309DF8A01000EB011001E082
:107090006BE006E1801C0990007820F00200801C63
:1070A000099908709DF8B40040F2A1110CE027E0A6
:1070B00058450020BC320020F8870020883E002080
:1070C000BC2200209840002010FB01F0FE4901EB9B
:1070D000C00000F562709DF8A01001EB410202EBC8
:1070E000011100EBC10018300990007820F0020077
:1070F000801C099908709DF8B4100220F2F7D6FFA1
:1071000000219DF8B40040F2A11210FB02F0EE4AFB
:1071100002EBC000017104229DF8B40040F2A111FD
:1071200010FB01F0E84901EBC00101F562719DF827
:10713000A00000EB400303EB001001F830208C228C
:107140009DF8B40040F2A11110FB01F0DE4901EB03
:10715000C00000F562709DF8A01001EB410303EB45
:10716000011100EBC10042719BE09DF8B40040F2B8
:10717000A11110FB01F0D44901EBC00101F56271CE
:107180009DF8A00000EB400202EB001011F8301057
:107190009DF8B40040F2A11210FB02F0CA4A02EBC3
:1071A000C000407981427CD19DF8B40000EB4001E1
:1071B00001EB0010A2F5986101EB001030309DF852
:1071C000A01000EB0110801C0990C04890F8050D3C
:1071D000C0F30010C0F1010009990A7860F30002C1
:1071E0000A709DF8B40000EB400101EB0010B849B3
:1071F00001EB001030309DF8A01000EB0110801C56
:107200000990B24890F8040DC2080998007862F31A
:107210004100099908709DF8B40000EB400101EBB2
:107220000010AB4901EB001030309DF8A01000EBCE
:1072300001108078C0F340029DF8B40040F2A11123
:1072400010FB01F0A04901EBC00000F562709DF851
:10725000A01001EB410303EB011100EBC100007E24
:10726000C0F3400082426DD09DF8B40040F2A111FD
:1072700010FB01F0944901EBC00000F562709DF82D
:10728000A01001EB410202EB011100EBC10018302C
:1072900009909DF8B40000EB400101EB00108C490F
:1072A00000E0C9E301EB001030309DF8A01000EBC6
:1072B0000110807842080998007862F3410009992A
:1072C00008709DF8B40000EB400101EB001080490C
:1072D00001EB001030309DF8A01000EB0110807819
:1072E000C0F3400048BB01229DF8B40040F2A11158
:1072F00010FB01F0744901EBC00101F562719DF8CA
:10730000A00000EB400303EB001001EBC000427350
:107310009DF8B40040F2A11110FB01F06A4901EBA5
:10732000C00000F562709DF8A01001EB410303EB73
:10733000011100EBC10080F846209DF8B410022036
:10734000F2F7B4FE9DF8B40000EB400101EB001031
:107350005F4901EB001130319DF8A00001EB0010F6
:10736000807800F001029DF8B40040F2A11110FBFA
:1073700001F0554901EBC00000F562709DF8A010C6
:1073800001EB410303EB011100EBC100007E00F0B3
:107390000100824279D09DF8B40040F2A11110FBA7
:1073A00001F0494901EBC00000F562709DF8A010A2
:1073B00001EB410202EB011100EBC1001830099012
:1073C0009DF8B40000EB400101EB0010404901EBD7
:1073D000001030309DF8A01000EB01108178099862
:1073E000027861F3000202709DF8B40000EB4001E6
:1073F00001EB0010364901EB001030309DF8A01071
:1074000000EB0110807800F00100E8BB9DF8B400AB
:1074100000EB400101EB00102D4901EB0010303072
:107420009DF8A01000EB01108078C0F3401068B305
:107430009DF8B40040F2A11110FB01F0224901EBCC
:10744000C00000F562709DF8A01001EB410202EB54
:10745000011100EBC10090F84600B8B99DF8B400E6
:1074600040F2A11110FB01F0174901EBC00000F53B
:1074700062709DF8A01001EB410202EB011100EBDC
:10748000C100407B10B902E05BE05FE242E09DF8A2
:10749000B40000EB400101EB00100D4901EB0010BE
:1074A00030309DF8A01000EB01108078C0F3400050
:1074B00080BB01229DF8B40040F2A11110FB01F045
:1074C000014901EBC00105E058450020BC22002025
:1074D0009840002001F562719DF8A00000EB400388
:1074E00003EB001001EBC00042739DF8B40040F2C2
:1074F000A11110FB01F0FE4901EBC00000F5627024
:107500009DF8A01001EB410303EB011100EBC1005A
:1075100080F8462000229DF8B40040F2A11110FB33
:1075200001F0F34901EBC00000F562709DF8A01076
:1075300001EB410303EB011100EBC10080F8452092
:10754000FFE19DF8B40040F2A11110FB01F0E84901
:1075500001EBC00000F562709DF8A01001EB410244
:1075600002EB011100EBC10090F84600B0B9012216
:107570009DF8B40040F2A11110FB01F0DC4901EBD1
:10758000C00000F562709DF8A01001EB410303EB11
:10759000011100EBC10080F845202AE000229DF88F
:1075A000B40040F2A11110FB01F0D14901EBC00180
:1075B00001F562719DF8A00000EB400303EB0010A1
:1075C00001EBC00080F845209DF8B40000EB4001BD
:1075D00001EB0010C74901EB001130319DF8A0000C
:1075E00001EB0010801C0990007820F0010209983E
:1075F0000270C14890F8E00780B19DF8B40000EB3C
:10760000400101EB0010BB4901EB001030309DF848
:10761000A01000EB0110807A022879D1B74890F8C9
:107620002900012874D1B548D0F80C02B349498D1E
:1076300088426DD29DF8B40040F2A11110FB01F018
:10764000AB4901EBC00000F562709DF8A01001EBA2
:10765000410202EB011100EBC10090F84500012846
:1076600054D19DF8B40040F2A11110FB01F0A049E3
:1076700001EBC00000F562709DF8A01001EB410223
:1076800002EB011100EBC10090F87F00F0BB01227A
:107690009DF8B40000EB400101EB0010954901EBAF
:1076A000001130319DF8A00001EB0010C2729DF86E
:1076B000B40000EB400101EB00108E4901EB00111A
:1076C00030319DF8A00001EB001001789DF8B40066
:1076D00040F2A11210FB02F0854A02EBC00041709B
:1076E00008229DF8B40040F2A11110FB01F080497E
:1076F00001EBC00101F562719DF8A00000EB4003B1
:1077000003EB001001EBC000427103E060E024E3F2
:10771000F6E0FDE300229DF8B40000EB400101EB30
:107720000010744901EB001130319DF8A00001EB0D
:10773000001042609DF8B4100220F2F7B7FC00215F
:1077400039911CE000229DF8B40040F2A11110FB19
:1077500001F0674901EBC00101F562719DF8A000DD
:1077600000EB400303EB001001EBC0014731BDF813
:10777000E4000A54BDF8E400401C81B23991BDF820
:10778000E4001428DEDB002039901CE000229DF884
:10779000B40040F2A11110FB01F0554901EBC0010A
:1077A00001F562719DF8A00000EB400303EB0010AF
:1077B00001EBC0016331BDF8E4000A54BDF8E400F8
:1077C000401C81B23991BDF8E4000A28DEDBB8E044
:1077D0009DF8B40040F2A11110FB01F0444901EB07
:1077E000C00000F562709DF8A01001EB410202EBB1
:1077F000011100EBC10006E0C9E281E2FEE32CE3E7
:1078000093E3FCE37BE290F84500012878D19DF8F2
:10781000B40040F2A11110FB01F0354901EBC001A9
:1078200001F562719DF8A00000EB400202EB001030
:1078300001EBC00090F8800040F2A11110FB01F0B4
:107840002B4901EBC00101F562719DF8B40040F2D3
:10785000A11210FB02F0264A02EBC00000F5627094
:107860009DF8A02002EB420303EB021200EBC200E2
:1078700090F8810000EB400202EB001001EBC00029
:1078800090F87E0003285CD102229DF8B40000EB42
:10789000400101EB0010174901EB001130319DF858
:1078A000A00001EB0010C2729DF8B40000EB400193
:1078B00001EB00100F4901EB001130319DF8A000E1
:1078C00001EB001001789DF8B40040F2A11210FB0A
:1078D00002F0074A02EBC000417008229DF8B40094
:1078E00040F2A11110FB01F0014901EBC00108E0D9
:1078F0005845002098400020BC320020BC120020D7
:107900001FE001F562719DF8A00000EB400303EB5E
:10791000001001EBC000427100229DF8B40000EBA2
:10792000400101EB0010FE4901EB001130319DF8E0
:10793000A00001EB001042609DF8B4100220F2F7A5
:10794000B5FB9DF8B4100220F2F7B0FB9DF8B4002F
:1079500040F2A11110FB01F0F24901EBC00000F56B
:1079600062709DF8A01001EB410202EB011100EBE7
:10797000C1008078802838D19DF8B40000EB400128
:1079800001EB0010E64901EB001030309DF8A0102B
:1079900000EB01108078C0F3400030BB9DF8B400CC
:1079A00000EB400101EB0010DD4901EB001030302D
:1079B0009DF8A01000EB01108078C0F34010A0B932
:1079C00015229DF8B40040F2A11110FB01F0D54939
:1079D00001EBC00000F562709DF8A01001EB4103BF
:1079E00003EB011100EBC10042719DF8B40000EB04
:1079F000400101EB0010CA4901EB001030309DF846
:107A0000A01000EB01108078C0F34000A8B18F22D5
:107A10009DF8B40040F2A11110FB01F0C14901EB47
:107A2000C00000F562709DF8A01001EB410303EB6C
:107A3000011100EBC10042714AE09DF8B40040F230
:107A4000A11110FB01F0B74901EBC00000F5627015
:107A50009DF8A01001EB410202EB011100EBC10007
:107A6000807B012834D100229DF8B40040F2A1119E
:107A700010FB01F0AB4901EBC00101F562719DF80B
:107A8000A00000EB400303EB001001EBC000827389
:107A90008C229DF8B40040F2A11110FB01F0A14925
:107AA00001EBC00101F562719DF8A00000EB4003FD
:107AB00003EB001001EBC000427100219DF8B400FF
:107AC00040F2A11210FB02F0964A02EBC0000171D5
:107AD0009DF8B40000EB400101EB0010904901EB70
:107AE0000010007BF0BB9DF8B40000EB4001C1EB3F
:107AF000C0108D4901EBC000807801049DF8B400EE
:107B000000EB4002C2EBC010874A02EBC000C07815
:107B100041EA00219DF8B40000EB4002C2EBC01026
:107B2000814A02EBC00000790843C117CDE9080182
:107B30000FF022FE9DF8B41040F2A11211FB02F1E9
:107B4000784A02EBC10202F562729DF8A01001EBC7
:107B5000410303EB011102EBC101C1F81E009DF8C6
:107B6000B40000E03AE000EB4001C1EBC0106E4908
:107B700001EBC000407900049DF8B41001EB410214
:107B8000C2EBC111684A02EBC101897940EA0120C8
:107B90009DF8B41001EB4102C2EBC111624A02EB45
:107BA000C101C9790843C117CDE908010FF0E4FD0F
:107BB0009DF8B41040F2A11211FB02F1594A02EBF8
:107BC000C10101F562719DF8A02002EB420303EBB5
:107BD000021201EBC201C1F81A0090E09DF8B40056
:107BE00000EB4001C1EBC0104F4901EBC0008078B1
:107BF00001069DF8B40000EB4002C2EBC0104A4AF7
:107C000002EBC000C07841EA00419DF8B40000EBEF
:107C10004002C2EBC010444A02EBC000007941EAC6
:107C200000219DF8B40000EB4002C2EBC0103E4AB8
:107C300002EBC00040790843C117CDE908010FF0FD
:107C40009BFD01469DF8B40040F2A11210FB02F02A
:107C5000344A02EBC00202F562729DF8A00000EB0C
:107C6000400303EB001002EBC000C0F81E109DF8AB
:107C7000B40000EB4001C1EBC0102B4901EBC00088
:107C8000807901069DF8B40000EB4002C2EBC01001
:107C9000254A02EBC000C07941EA00419DF8B400DA
:107CA00000EB4002C2EBC0101F4A02EBC000007A9A
:107CB00041EA00219DF8B40000EB4002C2EBC01085
:107CC000194A02EBC000407A0843C117CDE9080108
:107CD0000FF052FD9DF8B41040F2A11211FB02F119
:107CE000104A02EBC10101F562719DF8A02002EB80
:107CF000420303EB021201EBC201C1F81A0023E2B6
:107D0000BDF8A400032827D18F229DF8B40040F2CB
:107D1000A11110FB01F0034901EBC00106E00000D6
:107D20009840002058450020F887002001F5627136
:107D30009DF8A00000EB400303EB001001EBC00036
:107D4000427101219DF8B40040F2A11210FB02F033
:107D5000FE4A02EBC0000171F6E1BDF8A400032861
:107D600014D18F229DF8B40040F2A11110FB01F054
:107D7000F64901EBC00000F562709DF8A01001EB20
:107D8000410303EB011100EBC1004271DCE1BDF8DE
:107D9000A400032860D19DF8B40040F2A11110FBAB
:107DA00001F0EA4901EBC00000F56270BDF8D8109F
:107DB00001EB410202EB011100EBC10080790128C7
:107DC0002AD100229DF8B40040F2A11110FB01F06D
:107DD000DE4901EBC00101F56271BDF8D80000EB8E
:107DE000400303EB001001EBC00082718F229DF86D
:107DF000B40040F2A11110FB01F0D44901EBC00026
:107E000000F562709DF8A01001EB410303EB011136
:107E100000EBC10042711FE008229DF8B40040F25F
:107E2000A11110FB01F0C94901EBC00101F562711C
:107E30009DF8A00000EB400303EB001001EBC00035
:107E4000427100219DF8B40040F2A11210FB02F033
:107E5000BE4A02EBC000017176E1BDF8A400032820
:107E600062D19DF8B40040F2A11110FB01F0B749B6
:107E700001EBC00000F56270BDF8D81001EB4102C3
:107E800002EB011100EBC100807901282AD1002208
:107E90009DF8B40040F2A11110FB01F0AB4901EBD9
:107EA000C00101F56271BDF8D80000EB400303EB9F
:107EB000001001EBC00082718F229DF8B40040F2E7
:107EC000A11110FB01F0A14901EBC00000F56270A7
:107ED0009DF8A01001EB410303EB011100EBC10081
:107EE000427121E008229DF8B40040F2A11110FB7C
:107EF00001F0964901EBC00101F562719DF8A00007
:107F000000EB400303EB001001EBC000427100E006
:107F100020E100219DF8B40040F2A11210FB02F014
:107F20008A4A02EBC00001710EE1BDF8A4000828E6
:107F300066D19DF8B40000EB4001C1EBC01084494C
:107F400001EBC000807801069DF8B40000EB400210
:107F5000C2EBC0107E4A02EBC000C07841EA00418B
:107F60009DF8B40000EB4002C2EBC010784A02EB6F
:107F7000C000007941EA00219DF8B40000EB400206
:107F8000C2EBC010724A02EBC00040790843C1172F
:107F9000CDE908010FF0F0FB9DF8B41040F2A112FA
:107FA00011FB02F1694A02EBC10202F562729DF80F
:107FB000A01001EB410303EB011102EBC101486387
:107FC0009DF8B40040F2A11110FB01F05F4901EBF4
:107FD000C00000F562709DF8A01001EB410202EBB9
:107FE000011110F831009DF8B41040F2A11211FBFC
:107FF00002F1564A02EBC101497902E0FEE3E3E0F7
:10800000A2E0884234DA00219DF8B40040F2A112C7
:1080100010FB02F04D4A02EBC000017105229DF8F1
:10802000B40040F2A11110FB01F0484901EBC0017E
:1080300001F562719DF8A00000EB400303EB001016
:1080400001F830208E229DF8B40040F2A11110FBFF
:1080500001F03E4901EBC00000F562709DF8A010F0
:1080600001EB410303EB011100EBC10042716BE036
:108070009DF8B40040F2A11110FB01F0334901EB6F
:10808000C00000F56270BDF8D81001EB410202EBB0
:10809000011100EBC1008079012835D100229DF843
:1080A000B40040F2A11110FB01F0284901EBC0011E
:1080B00001F56271BDF8D80000EB400303EB00103E
:1080C00001EBC00082718F229DF8B40040F2A11133
:1080D00010FB01F01D4901EBC00101F562719DF833
:1080E000A00000EB400303EB001001EBC000427165
:1080F00001219DF8B40040F2A11210FB02F0134AD6
:1081000002EBC00001711FE08E229DF8B40040F226
:10811000A11110FB01F00D4901EBC00101F56271E5
:108120009DF8A00000EB400303EB001001EBC00042
:10813000427100219DF8B40040F2A11210FB02F040
:10814000024A02EBC0000171FDE300005845002027
:10815000F8870020BDF8A400032834D100219DF841
:10816000B40040F2A11210FB02F0FE4A02EBC00084
:10817000017101229DF8B40040F2A11110FB01F041
:10818000F84901EBC00101F56271BDF8D80000EBC0
:10819000400303EB001001EBC00082718C229DF8BC
:1081A000B40040F2A11110FB01F0EE4901EBC00058
:1081B00000F562709DF8A01001EB410303EB011183
:1081C00000EBC1004271BEE3BDF8A4000F287DD1D1
:1081D0009DF8B40000EB400101EB0010E24901EB17
:1081E0000010007BE8BB00202E902F9000213991D9
:1081F0001FE0DDE92E10000240EA11620902CDE91C
:108200002E129DF8B40000EB4001C1EBC010D7491D
:1082100001EBC001BDF8E400C0F10600085CDDE937
:108220002E341843CDE92E04BDF8E400401C80B282
:108230003990BDF8E4000528DBDB9DF8B400DDE9EA
:108240002E1240F2A11310FB03F0C64B03EBC00348
:1082500003F562739DF8A00000EB400404EB0010EE
:1082600000E049E003EBC00040F8221F426000221A
:108270002E922F92002139911FE0DDE92E1000028D
:1082800040EA11620902CDE92E129DF8B41001EB0B
:108290004100C0EBC110B54901EBC001BDF8E400DD
:1082A000C0F10B00085CDDE92E341843CDE92E0443
:1082B000BDF8E400401C80B23990BDF8E400052808
:1082C000DBDB9DF8B400DDE92E1200E0FDE340F2B7
:1082D000A11310FB03F0A34B03EBC00000F5627089
:1082E0009DF8A03003EB430404EB031300EBC30041
:1082F00022308160C26084E000202E902F90002107
:1083000039911FE0DDE92E10000240EA11620902F6
:10831000CDE92E129DF8B41001EB4100C0EBC11065
:10832000924901EBC001BDF8E400C0F10700085C10
:10833000DDE92E240243CDE92E24BDF8E400401CE3
:1083400081B23991BDF8E4000628DBDB9DF8B4006A
:10835000DDE92E1240F2A11310FB03F0814B03EB79
:10836000C00303F562739DF8A00000EB400404EB2A
:10837000001003EBC00040F8221F426000222E9242
:108380002F920021399120E0DDE92E10000240EA11
:1083900011620902CDE92E129DF8B41001EB4100E3
:1083A000C0EBC110714901EBC001BDF8E400C0F1A0
:1083B0000D00085CDDE92E3440EA0302CDE92E24ED
:1083C000BDF8E400401C81B23991BDF8E4000628F4
:1083D000DADB9DF8B400DDE92E1240F2A11310FBA8
:1083E00003F0604B03EBC00000F562709DF8A03015
:1083F00003EB430404EB031300EBC3002230816062
:10840000C2609DF8B41040F2A11011FB00F0554974
:1084100001EBC00101F562719DF8A00000EB400284
:1084200002EB001011F830109DF8B40040F2A112D8
:1084300010FB02F04B4A02EBC000407981427DD133
:108440009DF8B4009DF8A01001EB0010C217CDE913
:108450002E02474890F8E00708B39DF8B41001EBEE
:10846000410000EB0110404901EB001030309DF855
:10847000A01000EB0110807A022810D09DF8B410F3
:1084800001EB410000EB0110374901EB00103030E7
:108490009DF8A01000EB0110C07A00286CDD0022CE
:1084A0009DF8B40000EB400101EB00102E4901EBF8
:1084B000001030309DF8A01000EB0110C2722D4862
:1084C000D0F80C020521B0FBF1F201FB120000EB29
:1084D000400128482C3000EB41100D3009909DF8E8
:1084E000B41040F2A11011FB00F11E4800EBC100D6
:1084F00000F562709DF8A01001EB410202EB011142
:1085000000EBC10022301022014608900998EFF7D5
:108510009CFE1848D0F80C020521B0FBF1F201FBDB
:10852000120000EB400113482C3000EB41129DF883
:10853000B40040F2A11110FB01F000E0F8E209499B
:1085400001EBC00101F562719DF8A00000EB400352
:1085500003EB001001EBC00050F81A1F42F8011F96
:1085600040680AE05845002098400020F887002025
:10857000BC320020BC120020A5E15060FE48D0F8BB
:108580000C020521B0FBF1F201FB120000EB4001EF
:10859000F9482C3000EB41129DF8B40000EB40018B
:1085A00001EB0010F54901EB001130319DF8A000FE
:1085B00001EB001000781070EF48D0F80C02052194
:1085C000B0FBF1F201FB120000EB4001EA482C3055
:1085D00000EB4111EA48026841F81D2F808888802D
:1085E000E548D0F80C020521B0FBF1F201FB1200C6
:1085F00000EB4001E0482C3000EB41129DF8B40044
:1086000040F2A11110FB01F0DE4901EBC00101F5C0
:1086100062719DF8A00000EB400303EB001001EB3A
:10862000C000406BC2F80900D348D0F80C02052105
:10863000B0FBF1F201FB120000EB4001CE482C3000
:1086400000EB41129DF8B40000EB400101EB00107B
:10865000CA4901EB001130319DF8A00001EB001078
:108660004068C2F8230000229DF8B40000EB4001EE
:1086700001EB0010C14901EB001130319DF8A00061
:1086800001EB001042600021399154E0BA48D0F863
:108690000C020521B0FBF1F201FB120000EB4001DE
:1086A000B5482C3000EB41112731BDF8E4409DF86E
:1086B000B40040F2A11210FB02F0B24A02EBC00279
:1086C00002F562729DF8A00000EB400303EB00107E
:1086D00002EBC00090F8800040F2A11210FB02F003
:1086E000A84A02EBC00202F562729DF8B40040F2A3
:1086F000A11310FB03F0A34B03EBC00303F562735C
:108700009DF8A00000EB400505EB001003EBC00056
:1087100090F8810000EB400303EB001002EBC00275
:108720004732BDF8E400001D105C0855BDF8E400B8
:10873000401C81B23991BDF8E4000628A6DB002078
:10874000399042E000239DF8B40040F2A11110FBE3
:1087500001F08C4901EBC00101F562719DF8A000A8
:1087600000EB400202EB001001EBC00090F880002B
:1087700040F2A11110FB01F0824901EBC00101F5AB
:1087800062719DF8B40040F2A11210FB02F07D4A24
:1087900002EBC00202F562729DF8A00000EB4004FB
:1087A00004EB001002EBC00090F8810000EB4002E7
:1087B00002EB001001EBC0014731BDF8E4000B549F
:1087C000BDF8E400401C81B23991BDF8E4000A28EC
:1087D000B8DB6948D0F80C020521B0FBF1F080B29B
:1087E000014609900220F0F773FC00210620F1F702
:1087F0005DFC6148D0F80C025F4900E002E2498D5F
:10880000884206D25C48D0F80C02401C5A49C1F894
:108810000C0200210520F1F749FC9DF8B41001EB92
:10882000410000EB0110554901EB001030309DF87C
:10883000A01000EB0110801C0990007820F00802C5
:10884000099802704C48D0F80C020521B0FBF1F2F7
:1088500001FB120000EB400147482C3000EB4110B7
:10886000D0F823202E9800EB4001474800EB411040
:10887000C0F823200020399020E03F48D0F80C02B7
:108880000521B0FBF1F201FB120000EB40013A4878
:108890002C3000EB41102730BDF8E410425C2E98DC
:1088A00000EB4001384800EB41112731BDF8E400EE
:1088B0000A54BDF8E400401C81B23991BDF8E400CF
:1088C0000628DADB66E09DF8B41001EB410000EB0E
:1088D00001102A4901EB001030309DF8A01000EB88
:1088E0000110801C0990007820F0080008300999D8
:1088F00008709DF8B41001EB410000EB01101F4916
:1089000001EB001030309DF8A01000EB0110426820
:108910002E9800EB40011C4800EB4110C0F82320CA
:108920000020399027E09DF8B41040F2A11011FB0F
:1089300000F0144901EBC00101F562719DF8A0003F
:1089400000EB400200E005E202EB001001EBC00189
:108950004731BDF8E4000A5C2E9800EB40010A485C
:1089600000EB41112731BDF8E4000A54BDF8E400E2
:10897000401C81B2399109E0BC12002098400020CF
:10898000C731002058450020D8140020BDF8E4006D
:108990000628C8DB9DF8B41001EB410000EB011084
:1089A000FE4901EB001030309DF8A01000EB0110E3
:1089B000801C0990007820F02002099802709DF830
:1089C000B4100220F1F772FB9DF8B41040F2A11030
:1089D00011FB00F0F24901EBC00000F562709DF858
:1089E000A01001EB410202EB011100EBC1002230AB
:1089F00009902E9800EB4001EA4800EB41100D3041
:108A0000102208900999EFF720FC9DF8B41040F26D
:108A1000A11011FB00F0E24901EBC00101F5627108
:108A20009DF8A00000EB400202EB001001EBC0013A
:108A30002E9800EB4002DB4800EB421051F81A2F51
:108A400040F8012F496841609DF8B41001EB4100E6
:108A500000EB0110D14901EB001130319DF8A0006D
:108A600001EB001001782E9800EB4002CD4800EB9E
:108A7000421001702E9800EB4001CA4800EB4111F2
:108A8000C948026841F81D2F808888809DF8B4008D
:108A900040F2A11110FB01F0C14901EBC00101F549
:108AA00062719DF8A00000EB400202EB001001EBA8
:108AB000C000416B2E9800EB4002BA4800EB421018
:108AC000C0F809109DF8B40000E09AE000EB400106
:108AD00001EB0010B14901EB001130319DF8A0000D
:108AE00001EB001041682E9800EB4002AD4800EB0E
:108AF0004210C0F823102E9881B208200991F1F796
:108B0000D5FA00229DF8B40040F2A11110FB01F04B
:108B1000A34901EBC00000F562709DF8A01001EBC5
:108B2000410303EB011100EBC10080F8462053E044
:108B30009DF8B40000EB400101EB0010974901EBF8
:108B4000001030309DF8A01000EB0110801C09903F
:108B5000007820F00401091D099801709DF8B40007
:108B600000EB400101EB00108C4901EB00113031AA
:108B70009DF8A00001EB0010801C0990007820F007
:108B8000800080300999087001209DF8B41040F2EF
:108B9000A11211FB02F1824A02EBC10108719DF89A
:108BA000B40040F2A11110FB01F0114601EBC0002E
:108BB00042799DF8B40040F2A11110FB01F0784910
:108BC00001EBC00000F562709DF8A01001EB4103BD
:108BD00003EB011100F831208F229DF8B40040F220
:108BE000A11110FB01F06E4901EBC00101F56271AA
:108BF0009DF8A00000EB400303EB001001EBC00068
:108C00004271C7E0BDF8A400032857D1012166488E
:108C1000F53080F804179DF8B40040F2A11110FB64
:108C200001F05F4901EBC00101F562719DF8A00000
:108C300000EB400202EB001011F830109DF8B40078
:108C400040F2A11210FB02F0554A02EBC00040793D
:108C5000814234DA00219DF8B40040F2A11210FBE9
:108C600002F04F4A02EBC000017101229DF8B400EE
:108C700040F2A11110FB01F0494901EBC00101F5DF
:108C800062719DF8A00000EB400303EB001001F8B7
:108C900030208F229DF8B40040F2A11110FB01F0AA
:108CA0003F4901EBC00000F562709DF8A01001EB98
:108CB000410303EB011100EBC10042714AE09DF852
:108CC000B40040F2A11110FB01F0354901EBC000E6
:108CD00000F562709DF8A01001EB410202EB01115A
:108CE00000EBC1008078802834D100219DF8B400C9
:108CF00040F2A11210FB02F0294A02EBC000017100
:108D000080229DF8B40040F2A11110FB01F024492B
:108D100001EBC00101F562719DF8A00000EB40037A
:108D200003EB001001EBC000427100229DF8B4007B
:108D300040F2A11110FB01F0194901EBC00000F550
:108D400062709DF8A01001EB410303EB011100EBF1
:108D5000C10082701EE0BDF8A400032819D10021D3
:108D60001148F53080F804178F229DF8B40040F2C6
:108D7000A11110FB01F00A4901EBC00000F562707F
:108D80009DF8A01001EB410303EB011100EBC100C2
:108D9000427100BF00BF05F0FDB9000098400020FF
:108DA00058450020D8140020C73100209DF8B40099
:108DB00000EB4001C1EBC010FE4911F8300004285F
:108DC00001D125900BE09DF8B40000EB4001C1EB10
:108DD000C010F84911F83000152800D125909DF8F1
:108DE000B40000EB4001C1EBC010F24901EBC00040
:108DF00041789DF8B40000EB4002C2EBC010ED4A90
:108E000012F8300041EA002041F23001884202D1DC
:108E1000A62025903DE09DF8B40000EB4001C1EB99
:108E2000C010E44901EBC00041789DF8B40000EBAC
:108E30004002C2EBC010DF4A12F8300041EA0020C5
:108E400041F23101884202D1A720259021E09DF80E
:108E5000B40000EB4001C1EBC010D64911F830005E
:108E6000022816D19DF8B40000EB4001C1EBC01000
:108E7000D04901EBC00001799DF8B40000EB40023D
:108E8000C2EBC010CB4A02EBC000C07841EA00211F
:108E900025919DF8B40040F2A11110FB01F0C649E4
:108EA00001EBC000C17827919DF8B40040F2A111F8
:108EB00010FB01F0C04901EBC00108319DF89C0096
:108EC000C0EBC00001EBC00082789DF8B40040F216
:108ED000A11110FB01F0B84901EBC00108319DF868
:108EE0009C00C0EBC00001EBC000C0781044C1B2D0
:108EF00028910021B14A9DF8B40002EB00129DF8C0
:108F00009C00115439913AE09DF8B40040F2A1114F
:108F100010FB01F0A84901EBC00108319DF89C004D
:108F2000C0EBC00001EBC00002799DF8B40040F234
:108F3000A11110FB01F0A04901EBC00108319DF81F
:108F40009C00C0EBC00001EBC0008178BDF8E400DC
:108F5000084400EB400101EB00119DF8B40040F221
:108F6000A11310FB03F0944B03EBC00000F56270FB
:108F700000F83120BDF8E400401C81B239919DF821
:108F8000B40040F2A11110FB01F08B4901EBC001CC
:108F900008319DF89C00C0EBC00011F83010BDF8FE
:108FA000E4008142B0DCBDF8941043F23002881A2C
:108FB00091427DD009DC04297BD015297AD0A629DD
:108FC00010D0A72942F0798450E1B0F5C06F72D07B
:108FD000A0F2016000286FD001286ED00428F1D1E2
:108FE00001F0A2BF00219DF8B40040F2A11210FBD5
:108FF00002F0714A02EBC00001719DF8B40040F22A
:10900000A11110FB01F0114601EBC00008309DF8E2
:109010009C10C1EBC10100EBC1000079052824DCE4
:1090200006229DF8B40040F2A11110FB01F0624944
:1090300001EBC00108319DF89C00C0EBC00001EBC2
:10904000C0000271A8229DF8B40040F2A11110FBEB
:1090500001F0594901EBC00008309DF89C10C1EBAC
:10906000C10100EBC1004271FEE09DF8B40040F286
:10907000A11110FB01F0504901EBC00008309DF830
:109080009C10C1EBC10100EBC10000790A282BDC68
:109090000B229DF8B40040F2A11110FB01F04649EB
:1090A00001EBC00108319DF89C00C0EBC00005E059
:1090B00094E112E2FDE3FDE3FDE3FDE301EBC0001B
:1090C0000271A9229DF8B40040F2A11110FB01F039
:1090D000394901EBC00008309DF89C10C1EBC1017B
:1090E00000EBC1004271BFE09DF8B40040F2A11155
:1090F00010FB01F0304901EBC00008309DF89C10D6
:10910000C1EBC10100EBC10000790F2824DC102263
:109110009DF8B40040F2A11110FB01F0264901EBCB
:10912000C00108319DF89C00C0EBC00001EBC000FD
:109130000271A2229DF8B40040F2A11110FB01F0CF
:109140001D4901EBC00008309DF89C10C1EBC10126
:1091500000EBC100427187E09DF8B40040F2A1111C
:1091600010FB01F0144901EBC00008309DF89C1081
:10917000C1EBC10100EBC1004079A5282DD19DF8BC
:10918000B40040F2A11110FB01F00B4901EBC0014A
:1091900008319DF89C00C0EBC00001EBC000C17815
:1091A0009DF8B40000EB400202EB0010044A02EB11
:1091B000001007E0F887002058450020883E002076
:1091C00098400020303000EB0110801C099000789E
:1091D00020F00400001D099908709DF8B40040F2C9
:1091E000A11110FB01F0FC4901EBC00008309DF813
:1091F0009C10C1EBC10100EBC1008079A12833D0E4
:109200009DF8B40040F2A11110FB01F0F24901EB0E
:10921000C00108319DF89C00C0EBC00001EBC0000C
:1092200082799DF8B40040F2A11110FB01F0EA49E7
:1092300001EBC00108319DF89C00C0EBC00001EBC0
:10924000C0004271A1229DF8B40040F2A11110FBB0
:1092500001F0E14901EBC00008309DF89C10C1EB22
:10926000C10100EBC100827102F027BB00219DF813
:10927000B40040F2A11210FB02F0D74A02EBC0008A
:1092800001719DF8B40040F2A11110FB01F01146EC
:1092900001EBC00008309DF89C10C1EBC10100EB50
:1092A000C100007908281DDC00219DF8B40040F2BF
:1092B000A11210FB02F0C84A02EBC00001710822A3
:1092C0009DF8B40040F2A11110FB01F0C24901EB7E
:1092D000C00008309DF89C10C1EBC10100EBC1003B
:1092E000027124E09DF8B40040F2A11110FB01F0DE
:1092F000B94901EBC00008309DF89C10C1EBC101D9
:1093000000EBC10000790B2811DC0C229DF8B400A1
:1093100040F2A11110FB01F0AF4901EBC000083091
:109320009DF89C10C1EBC10100EBC10002719DF8DA
:10933000B40040F2A11110FB01F0A74901EBC000FD
:1093400008309DF89C10C1EBC10100EBC1004079D1
:10935000A42830D19DF8B40000EB400101EB0010CF
:109360009E4901EB001030309DF8A01000EB011079
:10937000801C0990007820F02000203009990870A6
:1093800000229DF8B40040F2A11110FB01F09249B7
:1093900001EBC00101F562719DF8A00000EB4003F4
:1093A00003EB001001EBC00080F845209DF8B410DD
:1093B0000220F0F77BFEA1229DF8B40040F2A1113B
:1093C00010FB01F0844901EBC00008309DF89C10AF
:1093D000C1EBC10100EBC100427145E700203990AB
:1093E00015E09DF8B40000EB4001C1EBC0107C49D2
:1093F00001EBC001BDF8E400C01C095C16AABDF871
:10940000E4001154BDF8E400401C81B23991BDF86C
:10941000E4000628E5DB062116A81DF065FD002105
:10942000CDE93001DDE93021100A40EA0160134640
:10943000319AC01842EB21214FF480724FF00003A3
:10944000CDE90801EEF7BEFE9DF8B40040F2A1118F
:1094500010FB01F0604901EBC00000F562709DF85F
:109460009C1001EB410303EB011100EBC100027101
:1094700000209DF8B41040F2A11211FB02F1564AEF
:1094800002EBC101087104229DF8B40040F2A11161
:1094900010FB01F0504901EBC00000F562709DF82F
:1094A0009C1001EB410303EB011100F83120A722CE
:1094B0009DF8B40040F2A11110FB01F0464901EB08
:1094C000C00000F562709DF89C1001EB410303EBB6
:1094D000011100EBC1004271C6E69DF8B40040F2F4
:1094E000A11110FB01F03C4901EBC00008309DF8D0
:1094F0009C10C1EBC10100EBC1000079042872DAB5
:1095000000219DF8B40040F2A11210FB02F0324A93
:1095100002EBC0000171A1229DF8B40040F2A1113C
:1095200010FB01F02C4901EBC00108319DF89C00B3
:10953000C0EBC00001EBC00042719DF8B40040F2E6
:10954000A11110FB01F0244901EBC00008309DF887
:109550009C10C1EBC10100EBC100001D0990007817
:10956000401CC2B2099802709DF8B40040F2A111EB
:1095700010FB01F0184901EBC00008309DF89C1069
:10958000C1EBC10100EBC1000079042823D10A22FC
:109590009DF8B40040F2A11110FB01F00E4901EB5F
:1095A000C00108319DF89C00C0EBC00001EBC00079
:1095B0000271A3229DF8B40040F2A11110FB01F04A
:1095C000054901EBC00008309DF89C10C1EBC101BA
:1095D00000EBC1004271EAE25845002098400020AB
:1095E000F8870020FFE79DF8B40040F2A11110FBBE
:1095F00001F0FE4901EBC00008309DF89C10C1EB62
:10960000C10100EBC100007904282FD100219DF891
:10961000B40040F2A11210FB02F0F44A02EBC000C9
:10962000017105229DF8B40040F2A11110FB01F078
:10963000EE4901EBC00108319DF89C00C0EBC00071
:1096400001EBC0000271A3229DF8B40040F2A11109
:1096500010FB01F0E54901EBC00008309DF89C10BB
:10966000C1EBC10100EBC1004271A0E29DF8B40062
:1096700040F2A11110FB01F0DC4901EBC000083001
:109680009DF89C10C1EBC10100EBC10000790828D6
:109690002FDC00219DF8B40040F2A11210FB02F073
:1096A000D24A02EBC000017109229DF8B40040F2D9
:1096B000A11110FB01F0CD4901EBC00108319DF86B
:1096C0009C00C0EBC00001EBC0000271A7229DF816
:1096D000B40040F2A11110FB01F0C44901EBC0003D
:1096E00008309DF89C10C1EBC10100EBC100427134
:1096F0005DE29DF8B40040F2A11110FB01F0BB49FE
:1097000001EBC00008309DF89C10C1EBC10100EBDB
:10971000C100007909282FDC00219DF8B40040F237
:10972000A11210FB02F0B14A02EBC00001710A2243
:109730009DF8B40040F2A11110FB01F0AB4901EB20
:10974000C00108319DF89C00C0EBC00001EBC000D7
:109750000271A3229DF8B40040F2A11110FB01F0A8
:10976000A24901EBC00008309DF89C10C1EBC1017B
:1097700000EBC10042711AE29DF8B40040F2A11161
:1097800010FB01F0994901EBC00008309DF89C10D6
:10979000C1EBC10100EBC10000790D282FDC0021D5
:1097A0009DF8B40040F2A11210FB02F08F4A02EBC8
:1097B000C00001710E229DF8B40040F2A11110FB0F
:1097C00001F08A4901EBC00108319DF89C00C0EB13
:1097D000C00001EBC0000271A1229DF8B40040F26C
:1097E000A11110FB01F0814901EBC00008309DF888
:1097F0009C10C1EBC10100EBC1004271D7E19DF8A3
:10980000B40040F2A11110FB01F0784901EBC00057
:1098100008309DF89C10C1EBC10100EBC10000793C
:109820000E282FDC00219DF8B40040F2A11210FB9D
:1098300002F06E4A02EBC00001710F229DF8B400E5
:1098400040F2A11110FB01F0684901EBC0010831A1
:109850009DF89C00C0EBC00001EBC0000271A32288
:109860009DF8B40040F2A11110FB01F05F4901EB3B
:10987000C00008309DF89C10C1EBC10100EBC10095
:10988000427194E19DF8B40040F2A11110FB01F087
:10989000564901EBC00008309DF89C10C1EBC10196
:1098A00000EBC100007910287DDC11229DF8B40086
:1098B00003E07DE1ABE1F8E1D9E140F2A11110FB59
:1098C00001F04A4901EBC00108319DF89C00C0EB52
:1098D000C00001EBC0000271A1229DF8B40040F26B
:1098E000A11110FB01F0414901EBC00108319DF8C5
:1098F0009C00C0EBC00001EBC00042719DF8B400B9
:1099000040F2A11110FB01F0384901EBC001083110
:109910009DF89C00C0EBC00001EBC00082710021EB
:10992000399156E09DF8B40040F2A11110FB01F00E
:109930002E4901EBC00108319DF89C00C0EBC0002E
:1099400001EBC0008178BDF8E40001449DF8B4004B
:1099500000EB400202EB0010254A02EB0010303011
:1099600000EB0110801C0990007820F0800080300E
:10997000099908709DF8B40040F2A11110FB01F0A4
:109980001A4901EBC00008309DF89C10C1EBC101E1
:1099900000EBC1008078BDF8E41042189DF8B400D7
:1099A00000EB400100E084E001EB0010104901EB06
:1099B0000010303000EB0210801C0990007820F07D
:1099C0000400001D09990870BDF8E400401C80B235
:1099D00039909DF8B40040F2A11110FB01F0034949
:1099E00001EBC00108319DF89C0003E058450020C0
:1099F00098400020C0EBC00011F83010BDF8E40022
:109A000081428FDC9DF8B40000EB400101EB0010B7
:109A1000FE4901EB001030309DF8A01000EB011062
:109A20008078C0F34010E8B39DF8B40000EB40012B
:109A300001EB0010F54901EB001030309DF8A0104B
:109A400000EB0110801C0990007820F0200209989A
:109A500002709DF8B40000EB400101EB0010EB49EF
:109A600001EB001030309DF8A01000EB0110807861
:109A7000C0F34000A8B99DF8B40000EB400101EB31
:109A80000010E24901EB001030309DF8A01000EB0F
:109A90000110801C0990007820F008000830099916
:109AA000087000E065E09DF8B4100220F0F7FEFABF
:109AB0007DE09DF8B40040F2A11110FB01F0D44903
:109AC00001EBC00108319DF89C00C0EBC00001EB28
:109AD000C00001799DF8B40040F2A11210FB02F021
:109AE000CB4A02EBC0004079814260D19DF8B400BE
:109AF00040F2A11110FB01F0114601EBC00008304B
:109B00009DF89C10C1EBC10100EBC1008079A12838
:109B100030D0A3229DF8B40040F2A11110FB01F057
:109B2000BB4901EBC00108319DF89C00C0EBC000AF
:109B300001EBC00042719DF8B40040F2A11110FB8E
:109B400001F0B34901EBC00008309DF89C10C1EB57
:109B5000C10100EBC1008079A22828D000219DF826
:109B6000B40040F2A11210FB02F0A94A02EBC000BF
:109B700001711CE0A1229DF8B40040F2A11110FB7C
:109B800001F0A34901EBC00108319DF89C00C0EB36
:109B9000C00001EBC000427101219DF8B40040F209
:109BA000A11210FB02F09A4A02EBC000017114E40A
:109BB000A1229DF8B40040F2A11110FB01F09449DC
:109BC00001EBC00108319DF89C00C0EBC00001EB27
:109BD000C00082719DF8B40040F2A11110FB01F0A9
:109BE0008B4901EBC00108319DF89C00C0EBC0001F
:109BF00001EBC000427100219DF8B40040F2A112B7
